:020000040800F2
:1000000000500020DD51010859E90008C53B0108F6
:1000100057E9000855E9000853E90008000000000E
:1000200000000000000000000000000051E900088E
:100030004FE90008000000004DE900082BDF000830
:100040007D5201087D5201087D5201087D52010850
:100050007D5201087D52010829C2000827C200080C
:100060007D5201087D5201087D5201087D52010830
:100070007D5201087D5201083DC200087D520108F1
:10008000599300087D5201087D5201087D520108F4
:10009000B9E900087D5201087D52010825C2000817
:1000A0007D5201080DBE00087D5201081DBE0008EA
:1000B000FDBD0008EDBD0008DDBD00083F53000890
:1000C00043530008395300083D5300087D5201088E
:1000D0007D52010835C200087D5201082BC200087C
:1000E00039DF00087D520108B53B0108000000001F
:1000F0000000000000000000000000000000000000
:0C01000000000000000000005FF808F1A3
:100110002DE9F04F684B694EA1B033600023736046
:1001200011F0EAFB18B911F009FC08F0B1F908F078
:1001300051FA634A634D1378634F43F00103137020
:100140000023089309930A934FF4E0130B932B6851
:10015000B87B43F480332B60AB6943F01003AB6191
:100160002B6803F400330993089B01330893099B20
:100170001BB9089BB3F5A06FF2D12B68514913F45A
:10018000003301D0022315E00A6842F001020A6040
:1001900008932B6803F002030993089B013308932B
:1001A000099B1BB9089BB3F5A06FF2D12B689A0786
:1001B00039D501230A93454B45491A6842F010028C
:1001C0001A601A6822F003021A601A6842F00202EA
:1001D0001A606B686B606B686B606B6843F480637C
:1001E0006B603C4B1A68043B22F070425A603A4AFA
:1001F0001160696821F47C116960596841F000411F
:100200005960D96821F40041D9609B681B0449BF3B
:10021000324B4FF4E01313604FF480130B930A9B9F
:10022000012B01D117E0FEE7022B18D168B10B9B1F
:10023000B3F5801F02D14FF4A01305E00B9BB3F57B
:10024000E01F02D14FF400130B930B996B680B4323
:1002500043F4803302E06B6843F460136B602B68F7
:1002600043F080732B602968164B8C01FBD55968CD
:1002700021F003015960596841F0020159606B682F
:10028000104903F00C03082BF9D14B68DFF85480B8
:1002900003F00C03042B03D0082B03D00C4B29E0F4
:1002A000136827E04B684868C3F38343C00303F136
:1002B000020319D40A4A1CE0777C00087801002068
:1002C0007630002000100240B026002000200240BE
:1002D00000127A000410014048000020001BB70003
:1002E00000093D000401002049681268890348BFE5
:1002F00052085343C8F800306B68DFF83091C3F3FD
:1003000003134B441A7BD8F8003020ACD340C8F814
:1003100000303A4A3A4BDFF818B19360394B4FF04E
:10032000000AD360AB69039243F00103AB616B6ACF
:100330003548B3606B6A43F080736B62AB6943F01E
:100340001C03AB614FF6FF7324F82C3D21468DF85A
:1003500056A00EF0E1FF584621460EF0DDFF2B4877
:1003600021460EF0D9FF2A4920464B6843F000731E
:100370004B600DF043F9159B2649039AB3FBF1F34B
:1003800025490B60254B4FF47A71C3F800A0D8F8CB
:100390000030DFF89480B3FBF1F32149013B4B605F
:1003A000F02382F823300723C1F808A00B60BB6854
:1003B000DFF880A0CAF8003009F11C0393E80300BD
:1003C000AB6984E8030043F00803AB610823CBF872
:1003D0001030159816A90EF09FFFDAF800301B07B1
:1003E00030D598F89231012B2CD80E4B98F89321E8
:1003F0009B6813F0805800F0C78523E000ED00E013
:10040000000000080005FA05000801400010014046
:100410000000014040420F001C1E0020201E002052
:1004200010E000E078010020B0260020F89E0108CE
:10043000000C014050260020B44B002283F8932189
:1004400008F094FA64200DF066FDA022B048002167
:1004500017F06DFAAF4A536823F4406343F07063BA
:1004600043F400635360EB69002243F00703EB6140
:10047000AB6943F4006343F00C03AB61A64B4FF050
:10048000000B03F10C0102F801B001320C2AF5D186
:10049000FF221A765A769A76DA76A04BA04A594607
:1004A0001A60A0483022DAF8005017F040FA594696
:1004B000C5F3801804239C4A9A4811F802E00C22E4
:1004C0004A4302F800E0B8F1000F09D1BEF11E0F57
:1004D00001BF4FF0FF0E03F1FF3302F800E0DBB283
:1004E00001310429E7D1914A97F805A01370904B88
:1004F000904983F800A0904B874AF361C0330B60AA
:100500008E4BA80603EBCA035B7848BF0123136236
:10051000002340F2DC518A4A22F813100133082BE1
:10052000F7D11C220EA8002117F001FA15F4007271
:100530001DBF844B149403930392BAF10E0F03D0A2
:100540000AF0EF03082B02D101238DF84A30C5F3DE
:1005500040038DF83E30C5F340338DF83830C5F395
:10056000C0338DF83B3015F400638DF8408004D023
:1005700097F88631591E4B424B418DF83C30C5F3FC
:1005800000438DF84130131C18BF01238DF8423011
:10059000336AB7F84821003318BF01238DF8433080
:1005A000C5F300538DF84430B7F84A31ADF84E200A
:1005B000ADF84830EA04B7F8563148BF534AADF8B1
:1005C0004630C5F3804348BFB2F850218DF83F3024
:1005D000B7F8543148BFADF84E20B3F5FA7FADF807
:1005E0004C3084BF0023ADF84E3097F8CE31564AD8
:1005F00086F82430002386F8253053709DF84A3061
:1006000005F00100002BC5F3C0018DF839008DF80D
:100610003A100CBF0023022300B901B1013309EBEA
:100620008309D9F824304FF00009A3F1020A1633E8
:1006300004934FF6FF723AF8023F934200F0B881FC
:100640009DF83D10DDB21B0ADAB219B1A91E0129CD
:1006500040F2AA819DF8401031B13C482901405830
:100660003B49884200F0A0819DF8411031B13748E4
:10067000290140583649884200F096819DF83E1085
:1006800051B13248334F00EB05104168B94203D1F4
:100690000189012900F088819DF83B1051B12B4858
:1006A0002C4F00EB05104168B94203D101890229A2
:1006B00000F07A819DF83C1051B12448264F00EBA0
:1006C00005104168B94203D10189022900F06C810B
:1006D000DDF850E0BEF1000F12D01C4FDEF8001024
:1006E00007EB0517786888420AD13989BEF80400FB
:1006F000884200F05981BEF80600884200F054811B
:10070000022B2BD19DF838302CE000BFB026002002
:10071000341E002000000140780100200C2600203B
:100720009828002010260020B0DF0108E1100020EA
:1007300090090020501F0020C42600208CC701080B
:100740004C100020F89E01089D01002064C20108A1
:100750000004004000080140000C0140012B04D1BE
:100760009DF83930002B00F01F819DF8443033B1E3
:100770009DF84A301BB92B1F032B98BF0422C24B94
:100780009DF838102D015F19A1B1D11EC9B2012900
:1007900008D85B59B3F1804F00F00681BB498B420A
:1007A0005DD101E1022A40F0E2805A59B84B9A42E9
:1007B00057D1F9E0012A52D19DF83F20DFF8E082BD
:1007C00032B15A59B24B9A4204BF032388F82730FA
:1007D000AD4AFF23511991F80DE088F86C3088F884
:1007E0006D30486801F1080309894FF0000BADF83E
:1007F000541002218DF8571088F870B015A9C8F868
:100800007C708DF856E00692059388F828B0C8F8F9
:100810002CB0C8F830B0C8F834B0C8F868B088F860
:100820006EB088F86FB00EF077FD059B069A997848
:1008300050595A4608F0E1FB3846594601220BF060
:100840004DFC944B9449C8F88030944BC8F888B05C
:10085000C8F8843038460A1D0BF088FCA4E0022A50
:100860004CD15FFA89F31C2101FB03FC8C4B4FF048
:10087000000803EB0C0B01238BF870300693824BBE
:100880008BF87190591991F80DE001F10802486850
:1008900009898BF87280ADF8541002218DF8571039
:1008A0008BF87A8015A9CBF87C70CDF81CC08DF838
:1008B00056E005920EF030FD734B059A5859917829
:1008C000424608F09AFB069B38461A4641460BF012
:1008D00005FC744A724BDDF81CC0CBF8802003EB9A
:1008E0000C01714A8031CBF88420CBF888803846DF
:1008F0000A1D0BF03BFC09F1010955E0032A39D12F
:100900009DF83F30664DDFF8D4813BB195F826B0B5
:10091000384608214FF6FF7200231CE0BDF84C203A
:1009200095F826B0B2F5FA7F0DD9604B3846B3FB87
:10093000F2F20821BDF84E3092B208F0B3FB5C4BE6
:1009400048F82B000CE05B4B3846B3FBF2F2BDF8E5
:100950004E30012192B208F0A5FB574B48F82B000E
:10096000C36095F82630013385F826301CE0012A53
:100970003FF422AF042A17D1BDF846204D4B484D15
:1009800093FBF2F23846BDF84830012192B295F857
:10099000258008F087FB95F8253005EB88080133A2
:1009A000C8F8500185F82530049B9A457FF441AE84
:1009B00096F82520414B86F87021414A002592F88F
:1009C00000801D70A8F11702022A354F99461AD8E7
:1009D000FB690021585903EB050A13F0AFFB10B176
:1009E000336A6BBB27E0374B05EB030E9AE80F0029
:1009F0008EE80F0099F8003010350133C02D89F8CA
:100A00000030E5D1ECE7304B13F838C003EBC803F6
:100A1000D3F804A089F800C0BAF1000FE0D0654512
:100A2000DEDA284A2B0103EB020E53440FCB0135CB
:100A30008EE80F00F3E7254E3368DD0452D41DE045
:100A4000234B244A13F8380003EBC8035D68107089
:100A5000002DF0D000238342EDDAC3EBC3016A1806
:100A6000D2F800C0DFF878E0013341F80EC001EBA6
:100A70000E069188B1809279B271ECE708F0EF032D
:100A8000082B154B53D155E064C201080004004007
:100A9000000800406D8A0008F8010020598B00080A
:100AA0007801002035900008438A000800127A007F
:100AB000798B000840420F00698B0008002000205D
:100AC00090090020CC0800208CC701085026002087
:100AD0006CAD0108DC1E0020241100200420002041
:100AE000DD1E002099F80030012BC7D91A4D05EB07
:100AF000031303F1100910354D45BFD055F8100C04
:100B00004FF07C5113F086F94FF07C5145F8100CF2
:100B100055F8140C13F07EF94FF07C5145F8140C85
:100B200055F80C0C13F076F945F80C0CE3E7B8F126
:100B30000E0F09D11A78B8F1180F42F010021A708E
:100B40000CD10DF057FC09E01A78B8F1190F22F01A
:100B500010021A70F4E700BFD40800200DF02EFC3C
:100B60003368BE4D58035EBFBD4B01221A70BD4AAB
:100B70004FF002091378214643F0040313704FF439
:100B80000043ADF8543014238DF85630AB698DF81E
:100B9000579043F00403AB61B3480EF0BDFBB34A7A
:100BA000B34B00201A600DF0CFF9B24B4FF00308A1
:100BB00093E80300AB6984E8030043F00803AB61EA
:100BC000159816A90EF0A8FBAB69182243F48053C0
:100BD000AB61EB68A44843F48053EB602146A0234B
:100BE0008DF8562005924FF0040AADF854308DF878
:100BF00057800EF091FB40239B482146ADF85430BE
:100C00008DF856A00EF088FB102397482146ADF8CA
:100C100054308DF8563004930EF07EFBE9684FF0A7
:100C2000070B41F48051E960E968059A21F480518D
:100C3000E9609149088800F4415040F4457040EA69
:100C400008000880888B20F400600004000C888372
:100C5000A1F810B0088880B240F040000880E9692F
:100C600041F48041E961296941F4804129618DF8AD
:100C70005780DFF80C828DF8562040464FF4204212
:100C80002146ADF854200EF047FB4FF48042404619
:100C90002146ADF854208DF856A00EF03DFB049B84
:100CA0004FF4805A404621468DF85630ADF854A096
:100CB0000EF032FB2B69714A43F480432B612B69A0
:100CC000484623F480432B61138803F4415343F4D3
:100CD000457343F003031380938B23F400631B04D9
:100CE0001B0C9383A2F810B013889BB243F040030F
:100CF0001380C8F810A00CF0EBFF002801F0B782B9
:100D00004388002B01F0B382DFF88C81002140463C
:100D10001022346816F00BFE4FF6FF73ADF8343036
:100D2000022304F4004A04F400694FF0000B1C4055
:100D30008DF836308DF837B00FD0012420A921F876
:100D40004C4D49480CF0C8FD072388F800B088F8DE
:100D500001B088F8024088F80330BAF1000F12D0D1
:100D6000022320A921F84C3D3F480CF0B5FD01239A
:100D7000E21888F8043088F80630072388F8054020
:100D800088F80730D4B2B9F1000F13D0022320A99C
:100D900021F84C3D3A480CF09FFD0923012288F8C8
:100DA0000C3088F80E20631C072288F80D4088F864
:100DB0000F20DCB26B68334843F440436B606B69CF
:100DC000DFF8C09043F001036B61AB6943F400733B
:100DD000AB610CF09BFB2C4B012C15932B4B4FF074
:100DE0000005169394BF2B4680231A934FF480730B
:100DF0001B934FF480631C93202315A91D93484631
:100E00004FF4005318941E93179519951F950CF0E5
:100E10005FFBD9F800301E4A43F00103C9F80030E7
:100E20005368012C23F4702394BF0021012123F483
:100E3000807343EA012353609168164B013C0B40D9
:100E400043F4602343F002039360D36AE4B223F4D3
:100E5000700343EA0454D46201231FE000100240EF
:100E6000F80D00207630002000080140E9DB000882
:100E7000843000202C9F01080030014000380040E1
:100E8000000C0140080002404C240140541D002089
:100E900000240140FDF7F1FF441D002008EB05028E
:100EA000917800295BD018F80500591C0928C9B2AF
:100EB000D278C04C11D9A0F10A0CD4F80C900CEBEC
:100EC0004C0C4FF0070E0EFA0CFE29EA0E0E02FA39
:100ED0000CF24EEA0202E2600EE0D4F810C000EB21
:100EE00040094FF0070E0EFA09FE2CEA0E0E02FA28
:100EF00009F24EEA02022261062BAE4C0ED8013BEB
:100F0000626B03EB83034FF01F0E0EFA03FE22EA1F
:100F10000E0200FA03F3134363631FE00C2B0ED899
:100F2000DA1FD4F830C002EB82021F2393402CEA70
:100F3000030E00FA02F34EEA030323630EE0A3F16B
:100F40000D02D4F82CC002EB82021F2393402CEA3E
:100F5000030E00FA02F34EEA0303E3620B46043584
:100F6000102D9BD1934B9A6842F480729A609A68D4
:100F700042F001029A609A6842F008029A60996809
:100F80008C4A090731D5FAE7531E092B3FF65AAAB6
:100F9000D9F840002146206058460EF0BDF94FF4C4
:100FA0000063CBF810303C200CF0B5FF97F893317C
:100FB0009845BFF641AADFF840B208224FF400631B
:100FC000CBF8102078200492CBF8143003930CF067
:100FD00097FF049A039BCBF814207820CBF81030AD
:100FE0000CF08EFF08F10108E0E7936843F004037A
:100FF0009360704B9A6812F00409FAD16E4C9A68AB
:10100000B4F85C0142F4A0029A60002841F03481F7
:10101000B4F95E31002B41F02F81B4F96031002B1F
:1010200041F02A8133689B031FD5C8200CF073FF61
:10103000AE200EF0F2FA08B10EF0F4FA5F4D87F828
:101040007101C8200CF067FF5D4B00210C2228467F
:10105000C7F8743116F06BFC0223EB700FF09DFDA6
:101060000CF034FF574B0344AB60574B00211B6817
:101070000C22B3F8563055480493B4F8646194F8E0
:1010800063A194F86B8194F86C51B4F80CB0E47BD4
:1010900016F04DFC14224E48002116F048FC4D4B32
:1010A00000221A7097F8783133B10022A7F87A211C
:1010B00053B904F035FA07E0059304F087FA059B6D
:1010C000002800F0F782F0E7B6F5807F0ED0BB2E47
:1010D0000ED8612E0ED8292E0ED8132E0ED8092E1A
:1010E0000ED8002E14BF062200220AE0002208E0DB
:1010F000012206E0022204E0032202E0042200E0D2
:101100000522354905920B88192023F040031B0462
:101110001B0C0B800B8823F038031B041B0C43F0C3
:1011200030030B800B889BB243F040030B8097F891
:101130007C1104F0DFF901200CF0E2FE059A1A2080
:10114000114604F0D7F901200CF0DAFE15A804F0DE
:101150009FF99DF95630013303D19DF95430013385
:1011600003D0B7F87A319BB21BB10023A7F87A31CC
:10117000A0E2174B194A64201A60194A5A60194AAA
:10118000DA60194A1A610CF0C6FE5146114B04226E
:101190001A70164B06221A70154A136843F00103A1
:1011A0001360144B002209291A709A4626D9114659
:1011B000F7E700BF00240140B0260020881C002073
:1011C0003A280020404B4C005C10002044200020B6
:1011D000C42400207A0E002000300140395000085D
:1011E000915400080D54000890C1793D0001002081
:1011F00020110020A0300020000C014040F20232FB
:1012000001238B401A4042BB13F0FD0F25D097F805
:10121000783133B10022A7F87A2153B904F080F96C
:1012200007E00693059104F0D1F90599069BA0B15A
:10123000F0E7CB4BCB4A64201A60CB4A5A600CF0E3
:101240006AFE04238AF80030C84B07225A70C84A45
:10125000136843F00203136003E0012901D9002160
:101260009FE7042D00F24981DFE815F005005001E9
:10127000680005000D010A200CF04DFE7720A0212A
:1012800001220DAB03F036FF002857D01E210122AA
:10129000772003F0EFFF4FF42F600CF031FE0027B2
:1012A000A7F160010025C9B2022215AB77208DF8A5
:1012B00054508DF8555003F01DFF9DF855309DF8A2
:1012C000542043EA0222AB4B03F5BF717A52023736
:1012D000102FE5D1B3F88C11012701F00F0001F4B4
:1012E0007F41A3F88C112B46DFF888E223F001023E
:1012F0007244B2F87E21002A18BF002713F0010FB4
:1013000003D0D2B25540082202E085EA1225FAE75E
:1013100015F4004F18BF85F4C055013A4FEA450552
:10132000F6D10133102BDFD1924A0143A2F88C1180
:1013300027B9C5F30333984200F074878D4D95F8B3
:101340008E31002B40F0B88714200CF0E4FD77209C
:10135000D02101220DAB03F0CDFE002800F09380D8
:101360009DF834300322552B85F8A731A5F8B0211C
:1013700040F08980D12101220DAB772003F0BAFE25
:101380009DF83430772003F00F021B0985F8A8215F
:1013900085F8A931162215ABAA2103F0ABFE9DF802
:1013A00054209DF8553043EA0223A5F890319DF86A
:1013B00056209DF8573043EA0223A5F892319DF854
:1013C00058209DF8593043EA0223A5F894319DF83E
:1013D0005A209DF85B3043EA0223A5F896319DF828
:1013E0005C209DF85D3043EA0223A5F898319DF812
:1013F0005E209DF85F3043EA0223A5F89A319DF8FC
:1014000060209DF8613043EA0223A5F89C319DF8E5
:1014100062209DF8633043EA0223A5F89E319DF8CF
:1014200064209DF8653043EA0223A5F8A0319DF8B9
:1014300066209DF8673043EA0223A5F8A2319DF8A3
:1014400068209DF8693043EA0223A5F8A4310123FE
:1014500085F88E3141F27073A5F8B43146F67813F1
:10146000A5F8B631444BC5F8B831444BC5F8BC318A
:10147000434BC5F8C031434BC5F8C431424BC5F8A6
:10148000C83100F019BF3B4F97F8CC51002D40F008
:10149000E18614200CF03FFD07F2CD137620D02119
:1014A000012203F027FE97F8CD31582B2ED107F5F6
:1014B000E87388211822762003F01CFE7620F421A0
:1014C000312203F0D7FE012387F8CC312F4BA7F848
:1014D000B451C7F8BC312E4BC7F8B83145F6D81314
:1014E000A7F8B6312B4BC7F8C0312B4BC7F8C43126
:1014F0002A4BC7F8C83100F0ADBE012D06D01B4BFA
:101500001B4A9D70136843F004031360184D2B6849
:101510009F0702D5124B1B689847F6B2154F204A19
:10152000002C4CD02B684EB940F2596113F0020FD9
:1015300040F2712318BF0B467D2108E09C0759BF7C
:101540004FF47A7319464FF4FA634FF47A719B455E
:1015500028DBBBF57A6FA8BF4FF47A6B23E000BF9E
:1015600044200020295000082B54000800010020CE
:101570002011002078010020315300084D5200084E
:10158000195300080D5200084D4F0008494F00083C
:101590004B4F000811530008C1510008E54C0008EA
:1015A000DC2200209B464B1E5B44B3FBF1F3013B66
:1015B000DBB203FB011187F87C31116003E087F88F
:1015C0007C41C2F800B02F4B44461B6898472E4E12
:1015D0000023337014B1022C40F03F864FF0000816
:1015E00020AB03F82C8D1E200A210122C7F8EC81C4
:1015F00003F080FD002800F062869DF85430482BEF
:101600000CD1224B224A1A60224A5A60224B0222F3
:10161000DA702B6843F008032B6002E0404600F0CC
:101620004EBE1E4B93F858210AB11D490A7093F81B
:1016300059210AB11B490A7093F85A3103B133702A
:101640002B68194D13F0080F19D0BDF910706426DE
:1016500097FBF6F4204612F089FB804606FB1470D7
:1016600000B212F083FB114912F0D4FB0146404650
:1016700012F0C8FA0E4912F0CDFB28601DE00023DD
:101680002B601AE0C4240020A130002010070020A5
:101690007DF30008E9F0000800010020B0260020DA
:1016A0007A0E0020A0300020F01D00208988883CA0
:1016B0000000204103200CF09DFCA94D08222B784E
:1016C0000A2443F002032B70A64B1A610495A54E21
:1016D0001920F368013C83F00803F3600CF01BFC55
:1016E00001200CF031FC19200CF015FC00200CF04E
:1016F0002BFC14F0FF04EAD108239B4F33613B68B5
:10170000180705D5994B1B689847994B01221A7009
:10171000984B994C1B68187B12F028FB974912F0E4
:1017200079FB06F091FD0646208812F01FFB31463A
:1017300012F070FB16F008FB914B1880208812F015
:1017400015FB01468F4812F019FC8F4912F016FC68
:101750008E4B8A4918608E4B8E4C186912F05AFBDA
:101760008D4912F057FB8D4BFF2118601A2220463D
:1017700016F0DDF82046002222703A68884B0121DD
:1017800012F0020F18BF617019701FBF032119708A
:101790000221A170510741BF19784C1C1C70032411
:1017A00048BF445412F00A0F0CD01A780421815417
:1017B000511CC9B205244454D11C02321970D2B252
:1017C00006218154774C21688A0641BF1A78561C3D
:1017D0001E70072648BF86540E0608D51A780926BB
:1017E0008654961C01321E70D2B20A2686546E4A66
:1017F00092F805E0BEF1080F02D0BEF10E0F04D141
:101800001A78561C1E700B2686541A78CD0302F1E6
:1018100001064FF00C0C48BF614D00F802C0F6B253
:1018200048BF02321E7041BF2A705A4A4FF00E0C58
:1018300002F806C04E0741BF1A78561C1E701026CB
:1018400048BF86541A78122602F1010C5FFA8CFC0C
:1018500011F4806F865483F800C0534E0AD096F876
:101860000C523DB14E4D02322A704A4A4FF01308D5
:1018700002F80C801A788D0502F1010C4FF0140863
:1018800048BF474D00F802805FFA8CFC48BF023227
:1018900083F800C041BF2A703E4A4FF0150802F895
:1018A0000C80BEF1180F14D11A784FF0160C00F806
:1018B00002C002F1010C5FFA8CFC4FF0170800F82F
:1018C0000C8002F1030C0232D2B283F800C000F89F
:1018D00002E0090341BF1A78511C1970192348BF4F
:1018E000835400219822314816F021F811F043FA70
:1018F0002F4B304A3049136000224A800A712F4929
:101900000B60A3F5C573B3F898011FFA80FE2C494C
:1019100021F812E00132122AF9D12268120740F1AF
:101920000E8193F89211062900F20381DFE801F09D
:1019300004046F95ACC8C800224A234B01291360E8
:10194000224D2348234A47D14FF0030C4FF0070E96
:10195000117085F800C080F800E00C2243E000BF61
:1019600076300020000C01402011002010070020DC
:10197000280700205C1F00201C00002035FA8E3C48
:10198000801F00200AE81C4100401C464C07002034
:10199000C424002025100020BD378635581F0020A4
:1019A0002410002050260020B026002070250020A2
:1019B0003A280020DC0E0020FC240020742F002098
:1019C0008C260020F406002008300020F0060020BD
:1019D000F8060020802E00200221297003210170CA
:1019E0000021117007221A70834A844B40201A602C
:1019F0000CF0A6F9002800F09C8001234FF0000BAA
:101A000090F9000040218DE808087D4A39E012F085
:101A1000ADF97C4912F0FEF97B4912F0F1F812F0B1
:101A2000E5FB0023794A42F823000133122BF9D158
:101A3000724A774940201160764A13700CF080F9A1
:101A4000002876D001234FF0070A90F900004021CA
:101A50008DE80804704A714B65E0714A674B40207D
:101A60001A606C4B10221A700CF06AF9002860D0D2
:101A700001234FF0000890F900008DE80801694A41
:101A800040214FF4E1334EE0674A5C4B40201A603E
:101A9000604B08221A700CF053F9002849D001233A
:101AA0004FF0000C90F9000040218DE808105F4ACB
:101AB0004FF4E13305F07AFF5D4BC3F8F00134E0F9
:101AC000544A0C23DFF8A0C15A4D5B481370062915
:101AD0004FF000028CF800202A7002700AD0574A9A
:101AE0001B211170564A4FF4E1351370554B0522F6
:101AF0001A7007E0514A21201070514A524D13705C
:101B0000504B1970514A3D4B40201A600CF018F9A7
:101B100078B101234FF0000E90F900008DE80840E5
:101B20002B464B4A402105F041FF003018BF0120F1
:101B300028B9082006F07AFC304B00221A6023688E
:101B4000344A13F4804F1FBF0821117041482B49BC
:101B500018BF086042F20101194051B127493E48BF
:101B60000860980444BF08211170D90744BF0C21B4
:101B7000117011781D06A1F10401517040F1A2808D
:101B80002B48DFF8E8B04FF0000ADFF8E480514658
:101B90001522C0F8F4B1314D00F5FC7088F801A0B1
:101BA000C8F804A0C8F808A015F0C1FEABF1050301
:101BB00050462B6009F049FE294B02201B68C8F8EB
:101BC0000C300CF0BDF8AE4618B9802006F02EFCA3
:101BD00070E090F805C098F80110224B0C2202FB2F
:101BE00001325278624545D00131C9B20429F4D995
:101BF000002288F801203FE05D3401080430002015
:101C000051350108CDCCCC3F0000B044142F00204A
:101C1000A93401080830002059360108A0860100C7
:101C200095340108E9350108813401089D35010822
:101C300078010020F51C0020F41C0020171D002056
:101C4000FF2F0020181D002090D00300B5D20008FF
:101C5000CDD20008D9340108E534010888070020F6
:101C600074260020A49F010800300020982800203E
:101C70006807002088F80110DEF800204FF00C0EF5
:101C8000127890F90000002A98F8012018BF03216B
:101C90000EFB023308BF012100225B780091019204
:101CA000022105F083FECD4B186000288DD0012065
:101CB00009F0CBFDCA4B1868CA4B00F5C5721A6013
:101CC00009F06AFE2368980569D5C74ADFF864837E
:101CD000039B4FF0100AC8F800309369C34843F0E3
:101CE00001039361039B0CA91B888DF832A0ADF80A
:101CF000303002238DF833300DF00EFBD8F8003071
:101D0000BA485B880CA9ADF8303004238DF8323026
:101D10000DF002FBD8F800104FF00F0E0B7A4FF0C9
:101D2000010B03F0030203F0FC0303F1804303F50E
:101D30008033986892000EFA02FE20EA0E00986046
:101D400098680BFA02F202439A604B68A84A002591
:101D5000536115A815938DF858508DF859A08DF83A
:101D60005AB011F003F9D8F800200DA8527A8DF876
:101D700036508DF8342003228DF835208DF837B099
:101D800011F0D6F89B4B9C4A1B683C3B13603B68A8
:101D90004FF0FF3243EA0A033B60984B1A60984BBE
:101DA000984A994F1360994A8033136023684FF023
:101DB0000008D90387F8008040F1C0800EF0CAFA0D
:101DC00040F22A33DFF870C2874D4FF0010A1A46FD
:101DD00060464146CDF814C0039387F800A015F083
:101DE000A6FDA9694FF0100B41F00801A961182167
:101DF0008DF8331003218DF832107C480CA9ADF812
:101E000030B00BF069FDE969814841F00201E961F8
:101E10008049814F0968A5F69475B1FBF0F13888C7
:101E2000013920F45C7000FA0BF020FA0BF03880D6
:101E300089B21D20B8853985A7F814A0398C21F006
:101E4000010101FA0BF121FA0BF13984398CB7F851
:101E500004E0388B21F0020120F0730000FA0BF04F
:101E600001FA0BF120FA0BF021FA0BF11FFA8EFEAA
:101E700040F0600041EA0A01A7F804E03883A7F8BF
:101E800034803984398B21F0080101FA0BF121FAF1
:101E90000BF141F008013983B7F844106FEA414172
:101EA0006FEA514189B2A7F84410D5F8A81F41EA5A
:101EB0000A01C5F8A81F28460BF028FB039B5749C9
:101EC00018938023DDF814C01A934FF48073159192
:101ED0001B9328464FF4005315A91E93CDF8648038
:101EE000CDF87080CDF87480CDF87C80CDF858C0E6
:101EF000CDF85CB00BF0ECFABB890DA89BB243F4B3
:101F00000073BB812B6843F002032B608DF834B063
:101F10008DF835A08DF836808DF837A011F008F8CF
:101F20003F4B1A683F4B43F8292009F10109B9F1E9
:101F3000200FF5D10DF012F90DF010F923685A05B4
:101F400040F19280384F394BD7F838950420C3F8C8
:101F500000900BF0F5FE0421C7F83C050BF0CCFE19
:101F6000334B87F840050820C3F800900BF0E8FEDB
:101F70000821C7F844050BF0BFFEDFF8C08087F8E2
:101F80004805002140462C2215F0D1FC8E2388F80C
:101F900001304FF07C0BE0234FF07D0A88F80330CE
:101FA00088F800B088F82BA0DFF894802C2200215C
:101FB000404615F0BCFC8A2388F801301020A0238D
:101FC00088F8033088F800B088F82BA0C7F84C9543
:101FD0000BF0B6FE1021C7F8500533E0841C00203A
:101FE0005C100020380F002000100240000C01405F
:101FF0000004014074260020600700207C100020AF
:10200000CC280020E8110020F90D0020C81C002079
:1020100000366E010401002000040040340400403A
:10202000349F0108FA0D00207801002014110020CF
:102030006C11002064070020850300203C11002063
:10204000711100200BF058FE87F854052020C7F8C6
:1020500058950BF075FE2021C7F85C050BF04CFE7F
:1020600087F860050FF024FB984F4FF000083B887D
:10207000322023F040031B041B0C3B803B884FF4B1
:10208000805A23F038031B041B0C3B803B880DF166
:1020900054099BB243F040033B809F238DF83430BA
:1020A0008DF835808DF836808DF837800BF033FF52
:1020B0008DF85580DFF88C820DAA0423C8F814A08F
:1020C0003846494603F03EF9C8F810A09DF856205E
:1020D0009DF85530120242EA03429DF857301A43E8
:1020E0007B4B9A427B4B17D008D87B498A420CD055
:1020F00001F51A4102318A4209D01CE077498A422F
:1021000005D001318A4207D015E0202200E080226C
:102110001A804FF4807202E04FF480721A805A8065
:102120009A88198812029A604A43DA606C4A01213F
:1021300082F8611504E000221A805A809A60DA6001
:10214000DB6803B34FEA1348C2464FF0000BC345A8
:1021500012DA0BEB08077F103804494610220DF005
:1021600009FA002359F8232001327CD10133042BD2
:10217000F8D1B846BA46EAE709F0C6FD584B4FEA2F
:102180000A42C3F864252368564A13F4002318BF93
:10219000012313700BF09AFE534B1860534B5B797D
:1021A000052B02BF524B4FF4C8721A80514B4FF4AB
:1021B0007A721A80504BC8221A80504A137843F022
:1021C000080313704E4A137823F00203137040F68D
:1021D0000203226813406BB14A494B4B19604B4BC9
:1021E000032119704A4B012119704A4900230B80C1
:1021F00049490B80930341BF484B04221A71DA7896
:1022000044BF42F00102DA70B36801222360444BFC
:102210001A70049B049A1B7863F07F03137021B03B
:10222000BDE8F08F42F21073A2F8B431A2F8B631D3
:102230003C4B0325C2F8B8313B4BC2F8BC313B4B99
:10224000C2F8C0313A4BC2F8C4313A4BC2F8C83177
:10225000FFF755B90425FFF752B9012C7FF6E1A924
:102260001C46FFF7B4B907F1010B574682E701207E
:102270000DF068FAFEF748BD2F4B00221A7000B22D
:1022800011F074FD2D4911F0C5FD1590B4F95E01F2
:1022900011F06CFD294911F0BDFD1690B4F96001F3
:1022A00011F064FD254911F0B5FD2549179015A8D9
:1022B00005F0D4FFFEF7B6BE0225FFF720B9012CCA
:1022C0007FF6AFA900243070FFF788B900380040CE
:1022D00018BA20000C000020152020001740EF0045
:1022E00078010020D82200200C080020B026002011
:1022F000EE0E00209A30002098300020241100209B
:10230000A33000202C2800200C1100207011002088
:10231000F8000020980E00209A0E0020881C002053
:10232000F80D002009530008B151000801530008BE
:10233000A1510008294B00084C00002035FA8E3CC2
:10234000201D0020000C0140B54B2DE9F04FB3F9E2
:102350000610B44B85B01F6801937A8991420EDB59
:10236000B1F5FA6FFC79BFBF8B1A6343A2F5FA642B
:1023700093FBF4F4ACBFC4F16404643400E064245F
:10238000A94BAA4AB3F898B193F9623112689BB28B
:10239000029215460393002240F2E630A04B4FEA2A
:1023A000420C33F912E0CBEB0E0303F2F316864234
:1023B00003D8002BB8BF5B4201E04FF4FA73022A46
:1023C0002ED0029E96F811611EB1B342CCBF9B1B6A
:1023D0000023642093FBF0F8954E6FF0630A36F803
:1023E00018900AFB083A08F1010836F918600FFA4C
:1023F00089F8C8EB060606FB0AF696FBF0F68D4850
:102400004E4420F80C60BE183679642073438A4E1F
:1024100093FBF6F364339BB2634393FBF0F02CE041
:10242000029890F812611EB1B342CCBF9B1B0023EF
:10243000642093FBF0F0DFF82C926FF0630808FB48
:10244000003A39F91060013039F91000002BA0EB87
:10245000060000FB0AFA9AFBF8FA0398C6EB0A0A90
:102460000AFB00FA7348B8BF5B42A0F804A0B87931
:102470004343714893FBF0F064306B784FF064088D
:10248000434393FBF8F36D4E022AB354EB7A6C4E40
:1024900000FB03F393FBF8F3B3546B7D654E00FB35
:1024A00003F090FBF8F0674B9854674B0ED1DE4574
:1024B00083F802800DDB5C4CB4F89A21914214DB66
:1024C000B1F5FA6FA8BF4FF4FA610FE0DE459C54F6
:1024D00004DA36F80C305B4226F80C300132032A5D
:1024E00005F101057FF458AFE5E71146891A4FF46D
:1024F0007A735943C2F5FA62B1FBF2F1642391FB9E
:10250000F3F2DFF874E16FF063073EF8120007FBA7
:10251000021101323EF9122007B2D21B514391FB46
:10252000F3F30344F380494B424D1B885F063BD5D0
:10253000474A484B10881B88181A00B211F016FC45
:10254000454911F067FC074605F07EFE8046384697
:1025500005F007FE0746B5F9020011F007FC8146B9
:10256000B5F9000011F002FC4146824611F052FC20
:1025700039468346484611F04DFC0146584611F055
:102580003FFB11F00DFE41462880484611F042FC09
:1025900039468046504611F03DFC0146404611F058
:1025A00031FB11F0FDFD68802C4D2B68980740F140
:1025B0009E8045F207212A4B2A4F1A687B69D31A5D
:1025C0008B4240F394807A610BF0EAFA264BDFF8F5
:1025D000AC901A789846032AB9F8003050D10A2BEB
:1025E00058D90023282088F800300BF094FC0BF019
:1025F000D7FA1E4B18880BF0BDFA1D4B1A68D3781A
:1026000090FBF3F0013008281A4BA8BF082018707F
:10261000537980B243433B8313795843788339E03D
:102620008C26002084100020B02600205C100020A2
:102630000E1E0020041100200CFEFFFFF0150020EC
:102640008E0E00200816002054150020E4110020F2
:10265000320F0020FC10002035FA8E3C502600205E
:102660007C300020800E0020701100205C1D0020B6
:102670000C110020F8000020F61D00201011002091
:102680000A2B07D803239B4A88F8003000231370D5
:102690003B837B8398F80030974A012B0CD002D300
:1026A000022B1BD023E03A8BB9F800309A421EDD92
:1026B000012388F800300FE0B9F800107B8B8B42C3
:1026C00002DD022313700FE08C4B1B8B0133994208
:1026D00002DD002313700AE0082006E07B8BB9F8C6
:1026E000002001339A42E3DC07200BF049FC2D68FF
:1026F000290575D5824B814F1A68FB69C3EB020827
:1027000045F2072398456BDDB6F906304FF47A7130
:10271000A3F57A7B7B4BFA61D3F8009098FBF1F834
:1027200099F80A30B4F85201012B774E03D040D308
:10273000022B1FD03FE0754B386A5A7B744B4FF029
:10274000080E33F8122090FBFEF392B2C01A8318E1
:102750003B6293FBFEF3BA8440F6E4429BB25343E0
:10276000B9F80820C2EB13334B43B9F9062093FBA9
:10277000F2F31FE0674BB9F808A01B78C6F800A079
:102780005A0718D510F051FE20B915F0100F18BFD8
:102790004FF0000B0BFB0BF1322391FBF3F3B9F974
:1027A00006205B445A434FF47A7392FBF3F353448D
:1027B00000E0002333603368D7E90A0103FB08F81F
:1027C0004FF47A7398FBF3F810EB080041EBE871D3
:1027D0000023C7E90A01504A11F028FD4F4B186049
:1027E0004F4E3368DB0427D52F0622D54D4B1B787F
:1027F0009D071ED54C4B187804281AD900224B4B44
:102800000521D718951C4FF00A0E122AD154E9B2AF
:1028100087F801E004D0B0EB510F2A46EFD800E072
:1028200014215A18322002F8010CFF225A540F20AA
:1028300000E00A200BF0A4FB3D4D2A68002A51D08D
:102840003C4B3D4F18683968984681424AD83B4B0B
:10285000DFF8F49019785268E1B94FF0010A83F873
:1028600000A0B9F80030D35C23B350460BF06CFBEA
:10287000334B83F800A011F02FF8B9F80030CBB932
:102880002B681B78053B534514D80BF01FFB2D4BD1
:1028900018600FE04FF0000A83F800A0B9F800308C
:1028A000D35C3BB150460BF04FFB254B83F800A0A7
:1028B00011F012F82B68B9F800205B6822499B5C84
:1028C000FE2B02D100230B800CE0FF2B02D10BF07A
:1028D00041FB07E0D8F800000A2505FB030301329D
:1028E0003B600A800B4D2B78580731D5174B0822D7
:1028F0005A616BE0F800002070110020800E00206B
:102900007C3000200C11002018110020441D0020F4
:10291000541D0020A3300020407E05001C11002023
:1029200020100020241100202A1100205020002017
:10293000301E002074260020281E0020241E0020A7
:102940006E300020942400202C1E0020000C01403A
:102950003268D1075CBF43F001032B70984B1B78A2
:102960001F075EBF2B7823F001032B70D60248BFF0
:102970002B78944A44BF23F001032B70924B1B68C1
:1029800013F0040F02D09149098851B99049098880
:1029900009B1980705D48F4B1B88003318BF01235A
:1029A00033B1022313702B7823F001032B7004E062
:1029B0002978C90758BF022313700BF087FA864B9A
:1029C0001B68C01A002801DB10F086FF0EF070FEB5
:1029D000824B1E789846002E00F0AB80804E336804
:1029E000002B00F0E78630680BF040FB002800F079
:1029F000E1867B4B7B4C18680BF035FB092801D036
:102A00003F2850D14FF0000A5746D4F80090764D39
:102A1000B9F1000F05D0754829684A4614F0D4FF73
:102A200010B9AA4607B92F46714B10359D42EFD316
:102A3000C7B1D7F800E0DAF800C023681EF80350E9
:102A40001CF80300A8420DD15A1C684938B92D2B37
:102A500005D8644D2A602025CD54885402E0CD5419
:102A60002260EAE723680BB1574511D061480DF0A9
:102A700059F9574507D857F8100B0DF053F90920AD
:102A80000DF048F9F5E75C480DF04CF94FF00009FE
:102A900023689945A7D2554B13F809000DF03AF970
:102AA00009F10109F4E72368002B40F06886042847
:102AB00040F0A1864D4809F0C7FE00F07BBED9F872
:102AC0000000DFF844A10BF0D1FA40B3DAF80000BF
:102AD0000BF0C9FADBF80030024693F848100029E1
:102AE00035D1242840F09280012283F84820DBF879
:102AF0000030DFF810A193F84820062ADFD193F8C0
:102B0000490002F0A5FD8146002800F0A3803B6843
:102B100098790DF054F83B68002283F84820374B31
:102B200093F83530002B40F018864C36982E00F084
:102B30004186334BF21892F84A100129F5D1314FF2
:102B4000F3583A60304ABB4613609146B7E7012913
:102B500004D14D2814BF00220222C6E7022904D165
:102B60003C2814BF00220322BFE703290CD14028D0
:102B70004FF0000102D983F84810B8E75871197175
:102B8000D97198710422B0E7042906D1997983F8A4
:102B900049004A409A710522A7E70529A7D158792B
:102BA00019798842987906D950409871481C187153
:102BB0000B441A729BE790420CBF0622002294E756
:102BC000241100206E3000202011002098300020B9
:102BD000EE0E00209A30002070300020A43000203B
:102BE000FC1F0020C41C0020CCAA0108941C00205B
:102BF000ACAC010824C6010829C60108800E0020DB
:102C000070250020C4110020C81100202B7858071F
:102C10003FF56DAF232ADAF800300ED1012188F894
:102C20000010AE49AE480B60AE4902920B630DF046
:102C300079F8AD480DF076F8029AAC4B1B681B781A
:102C4000934201BFAA4AAB4B1A60AB4A04BFAB4BDD
:102C5000DA604CE7DAF8002092F849304A2B00F0AD
:102C600038815CD8332B00F09E8421D8292B00F0CA
:102C7000388409D8252B00F00F84272B00F013840B
:102C8000232B40F0B4853CE22D2B00F03B8407D889
:102C90002B2B40F0AC850CF075FF607100F058BD37
:102CA0002F2B00F00885312B00F01A8500F09FBD16
:102CB0003E2B00F004811DD8372B00F0C48404D8CB
:102CC000352B00F0578200F092BD392B00F0F883CD
:102CD0003C2B40F08C85DFF82892D9F800A00CF04E
:102CE00051FF8AF80000D9F8003018780BF0EAFD9F
:102CF00000F02EBD432B00F0838406D8412B40F01A
:102D000076854FF0000900F053BC442B00F01C8581
:102D1000482B40F06C8509F035F800F019BDD02B38
:102D200000F0338368D8CA2B00F0F2801CD84E2BF9
:102D300000F00B8410D84C2B40F059850CF022FF8A
:102D400084F8D0010CF01EFF84F8D1010CF024FFB0
:102D5000A4F8D20100F0FCBCC82B00F08380C92B82
:102D600000F0348300F043BDCD2B00F0198304D86C
:102D7000CC2B00F0278200F03ABDCE2B00F0198357
:102D8000CF2B40F034850CF007FF6FF4AF6283184F
:102D90009BB2C62B98BFA4F898010CF0FDFEA4F8D6
:102DA00044010CF0F9FEA4F846010CF0F5FEA4F87D
:102DB00048010CF0F1FEA4F8D2010CF0E3FE84F817
:102DC000E3010CF0DFFE0CF0DDFE84F8E4010CF012
:102DD000D9FE84F887010CF0D5FE84F894010CF03C
:102DE000D1FE474BD3F800900CF0D6FE00EB8000EC
:102DF0004000A9F8560063E3D62B00F04B820AD8B6
:102E0000D22B19D0C0F00983D32B25D0D42B00F0BE
:102E10004C8200F0ECBCEF2B41D005D8D82B40F011
:102E2000E6844FF00009FFE0F22B00F08682FA2BD7
:102E300000F0C88200F0DBBC2B78590700F18884D1
:102E40000CF0A0FE022884F8A40740F2A4822D4BC7
:102E5000002283F8A4279EE20CF09EFE2A4B1880E5
:102E600000F076BC92F805904FEA5909B9F1120FBB
:102E700003D910F00BF800F06BBC4FF0000ACA4504
:102E800007D20CF089FE214B23F81A000AF1010A3F
:102E9000F5E7144B012283F8342000F059BCDFF829
:102EA0006090D9F800A00CF077FEAAF85A00D9F883
:102EB00000900CF071FEA9F8580000F049BC0CF02D
:102EC00061FE84F8D6010CF05DFE84F8D50100F0B7
:102ED0003FBC0CF061FEA08100F03ABCFC1F00205A
:102EE00059C60108800E002029C601080C260020C2
:102EF000EFBEADDEF04F00200400FA0500ED00E06B
:102F00005C100020B0260020300F00208C2600200E
:102F1000D64B1A689A461278022A6AD1DAF800303B
:102F200009F1080B02930CF02DFE10F01BFFD049A5
:102F300011F024F8029B43F82B00DAF800B00CF0F3
:102F400021FE09F10A030BEB830B10F00BFFC949BB
:102F500011F014F8DAF80030CBF8040002930CF00A
:102F600011FE10F0FFFEC44911F008F809F10E0B34
:102F7000029B09F10109B9F1030F43F82B00CDD1F0
:102F8000B9F1070FDAF800B01AD10CF0FBFD10F020
:102F9000E9FEB74910F0F2FFCBF84400DAF800B0D0
:102FA0000CF0F0FD10F0DEFEB14910F0E7FFCBF8B9
:102FB0004800DAF800B00CF0E5FD8BF84C0012E0A8
:102FC0000CF0E0FDCB448BF80100DAF800B00CF017
:102FD000D9FDCB448BF80B00DAF800B00CF0D2FD31
:102FE000CB448BF8150009F10109B9F10A0FC7D1DB
:102FF000AEE3DAF800B00CF0C5FDCB448BF801006D
:10300000DAF800B00CF0BEFDCB448BF80B00DAF818
:1030100000B00CF0B7FDCB4409F10109B9F10A0F7A
:103020008BF81500E5D193E3DFF840A209F1080B16
:10303000DAF8003002930CF0AFFD10F093FE8E49E9
:1030400010F09CFF029B43F82B00DAF800B00CF064
:10305000A3FD09F10A030BEB830B10F083FE8649F5
:1030600010F08CFFDAF80030CBF8040002930CF07B
:1030700093FD10F077FE804910F080FF09F10E0BF0
:10308000029B09F10109B9F1030F43F82B00CBD1E1
:10309000B9F1070FDAF800B01AD10CF07DFD10F08D
:1030A00061FE754910F06AFFCBF84400DAF800B011
:1030B0000CF072FD10F056FE6F4910F05FFFCBF878
:1030C0004800DAF800B00CF067FD8BF84C0012E015
:1030D0000CF062FDCB448BF80100DAF800B00CF084
:1030E0005BFDCB448BF80B00DAF800B00CF054FD1C
:1030F000CB448BF8150009F10109B9F10A0FC7D1CA
:1031000026E30CF03FFD132883463FF6B2AEDFF80E
:103110005CA1DAF800900CF035FD002357490C2231
:1031200002FB0312117A814220D1137809EB8B093B
:1031300089F879300CF026FD89F87A000CF022FD30
:1031400089F87B000CF01EFD4D4A4E4B89F87C003F
:103150001A60DAF800004C4B0021186079300AF050
:103160007BFE4A4B80F001001870F1E201331B2B0B
:10317000D4D17EE60CF006FD0B2882463FF679AEF0
:103180003A4BD3F800900CF0FDFC03283FF671AEEB
:10319000062303FB0A9989F8CE000CF0F3FC89F8AA
:1031A000C9000CF0EFFC89F8CA000CF0EBFC89F8C0
:1031B000CB000CF0E7FC89F8CC000CF0E3FC89F8BC
:1031C000CD00C5E25379092B7FF653AE019BD3F8AE
:1031D00000900CF0D7FC019B89F80000D3F8009018
:1031E0000CF0D0FC89F801000CF0CCFC019B6428A9
:1031F0001B68A8BF642018710CF0C4FC019B6428F4
:103200001B68A8BF642058710CF0BCFC019BFF2810
:103210001B68A8BFFF2098710CF0B4FC019B6428C8
:10322000D3F8009028BF642089F807000CF0AAFCAE
:10323000019B89F80200D3F800900CF0A3FC019BDD
:1032400089F80300D3F800900CF0A6FC3B68A9F8BD
:103250000A005B790A2B40F27B820D4BD3F8009079
:103260000CF090FC89F8080072E200BF5C100020AE
:10327000000020410000C84200007A44F8A3010881
:10328000F4270020280F00202C0F00200800002029
:10329000841000200CF080FCCB4B23F8190009F1BE
:1032A0000109B9F1080FF5D152E253790F2B7FF4E0
:1032B000E0AD0CF067FC072881463FF6DAADDFF899
:1032C00034A3DAF800B00CF067FC0E2303FB09F915
:1032D000CB44ABF81901DAF800B00CF05DFCCB443C
:1032E000ABF81B01DAF800B00CF056FCCB44ABF89D
:1032F0001D01DAF800B00CF045FCCB448BF81F013F
:10330000DAF800B00CF03EFCCB448BF82001DAF880
:1033100000B00CF037FCCB448BF82101DAF800B098
:103320000CF030FCCB448BF82201DAF800A00CF052
:103330003DFCD144C9F823010AE20CF023FC0F281C
:1033400081463FF696AD0CF01DFCC9EBC909A144BE
:1033500089F8D4000CF016FC89F8D5000CF012FCAA
:1033600089F8D6000CF00EFC89F8D7000CF00AFCA6
:1033700089F8D8000CF006FC89F8D9000CF002FCA2
:1033800089F8DA000BF036F8E2E12B785B0700F100
:10339000DF810EF0D3FA05F07BF805F01BF9D7E1D9
:1033A0002B78580700F1D481884B4FF4C8721A80EB
:1033B000CEE12B78590700F1CB81854A137843F091
:1033C000040328E02B785A07E5D510E20CF0DAFB6D
:1033D0007F4B1A7810B142F0020201E022F00202A3
:1033E0001A700CF0CFFB7B4BDFF80C9218700CF0CE
:1033F000DDFBC9F800000CF0D9FBC9F804000CF0A3
:10340000CBFB754B18800CF0C7FB744B744A1880CB
:10341000137843F0020313709AE10CF0B3FB0290AF
:103420000CF0C4FB83460CF0C1FB82460CF0BEFBE3
:1034300081460CF0B1FB0CF0AFFB0CF0A3FB029B40
:10344000A3B9684B1020C3F800B0C3F804A004F07F
:10345000CCFF5F4A137843F001031370B9F1000FFA
:1034600000F07681604BC3F8009071E1102B40F0C2
:103470006F815E4BC3F800B0C3F804A0B9F1000F30
:1034800002D0594BC3F800905848594B0222011DF5
:103490001A7008F03BFA5BE1A0600CF087FBA368B0
:1034A0001843A06054E10CF077FBA4F85C010CF029
:1034B00073FBA4F85E010CF06FFBA4F8600147E118
:1034C0000CF060FB84F87C010CF05CFB84F880015C
:1034D0000CF058FB84F87F010CF054FB84F8810158
:1034E00036E10CF059FBA4F882010CF055FBA4F86E
:1034F00084010CF047FB84F886010CF04DFBA4F826
:10350000880125E10CF03EFB84F892010CF044FBAD
:10351000A4F89C010CF040FBA4F898010CF03CFBD3
:10352000A4F89A010CF02EFBDAF8003084F893012D
:103530005B79082B40F20C810CF02EFBA4F89E0165
:103540000CF02AFBA4F8A00102E192F805900323F5
:10355000B9FBF3F9B9F10E0F3FF68BACDFF89CA085
:103560004FF0040BCB4580F0F3800CF00BFB8AF896
:10357000A2010CF011FB40F2ED23984205DD40F66C
:10358000CA039842A8BF184601E040F2EE20A0F21C
:10359000EE20192390FBF3F00BF1010B8AF8A30145
:1035A0000AF1020ADEE70CF0EDFA84F89401CFE0AC
:1035B0000CF0E8FA04EB090309F10109B9F1080F6D
:1035C00083F88A01F4D1C3E0E21F0020EE0E002050
:1035D000241100202A11002028110020261100208B
:1035E0008A1000208C1000209C10002094100020D5
:1035F000340F00205C1000202C110020B026002089
:103600000CF0C0FAC4F8089060710CF0CFFAA3680F
:103610001843A0600CF0B6FA84F892010CF0BCFAE2
:10362000A4F85C010CF0B8FAA4F85E010CF0B4FA4E
:10363000A4F860010CF0B0FAA4F882010CF0ACFA26
:10364000A4F8840184E053794FF0070AB3FBFAF23F
:10365000C2EBC2029A1A12F0FF0F7FF40AACB3FB5E
:10366000FAFA0AF1FF3A5FFA8AFABAF1FF0F6FD05D
:103670000CF088FA5FFA80FB4FFA8BF00AF028FB17
:10368000814600283FF4F5AB80F800B00CF084FAD6
:10369000A9F802000CF076FA89F804000CF072FA2E
:1036A00089F805000CF06EFA89F807000CF06AFA48
:1036B00089F80600D5E7DFF8509209F1400A0CF0CE
:1036C0006BFAA9F89C020CF05DFA89F89E020CF0E6
:1036D00059FA09F1040989F89B02D145EFD137E085
:1036E0000CF050FA1F2881463FF6C3AB3B685B796C
:1036F000082B7FF4BEAB0CF04FFA09F1860904EBFE
:10370000890900F03F00A9F806000CF045FAB9F865
:103710000630800100F4FE501843A9F806000CF0B2
:1037200031FA000189F804000CF02CFA99F8043001
:1037300000F00F00184389F804000CF023FA89F810
:1037400005000CF007FE03E05D4B012283F83520F5
:1037500000200CF063FAFFF7DAB95A4B98590AF0D7
:103760007CFC18B932200AF0D6FBF6E70AF000FE1E
:1037700004F064FE544A554BDA60FFF7D6B90C28C2
:103780003BD00A2842D1524D52480CF0CBFA284681
:10379000232114F002F908B1401B20602368002B9C
:1037A00057D14B4800213022236014F0C0F898F81C
:1037B00000302BBB484B1B689B060FD5474B40493D
:1037C0001B688A6B9A1A002A08DB454A1278042A79
:1037D00082BF03F5123303F5F8738B63414B9B688B
:1037E000002B69D0404805B0BDE8F04F18470FF0F6
:1037F0004DFBFFF78CB90C2804D13C480CF092FA31
:103800003B480DE07F2812D1FFF7EDB80D28BAD064
:103810007F2809D12E4A013B002136482360D1542C
:103820000CF080FAFFF7DFB82F2B3FF6DCA8A0F1F1
:103830002002D2B25E2A3FF6D6A813B920283FF460
:10384000D2A85A1C2260224AD0540CF063FAFFF727
:10385000CAB85A1EA95C202901D113469FE71C4A09
:1038600000212360D154244B244DD3F800A0D5F877
:1038700000B0DFF85C90584614F09DF807465946B2
:103880003A46484614F0A0F81D4A28B919F80730FE
:1038900053445B785B0703D010359542E7D306E0CD
:1038A000954204D2781CEB684844984702E01548DA
:1038B0000CF038FA002374E705B0BDE8F08F00BFC4
:1038C000800E0020702500200400FA0500ED00E0C5
:1038D000941C002031D40108201100207C300020ED
:1038E0002A110020C4240020BC0E00202EC601088E
:1038F00029C6010855C601080C010020CCAA010800
:10390000ACAC010839C60108B02600202DE9F04F03
:10391000A04EA14D3368A14C03F59C432033236096
:103920002B889F4A01332B8042F20103116889B032
:103930000B4092461BB19B4A1378013313700FF072
:10394000FFFEDAF80030DF0405D5974B1B68D80777
:1039500001D40EF0DBFC954B37681A68907AB8B149
:103960009349137B013831F810001BB1C0F53B605F
:10397000083080B200B2A0F57A70B0F57A7FA8BFA7
:103980004FF47A7020EAE07010F0F0F9894930E0E5
:10399000DAF80030190435D56368804EFB1A002B25
:1039A00030DB07F59C4320337360834BD27A59791F
:1039B000824B33F81130317A9BB293FBF2F3013131
:1039C00001F00F0232723244537203467C4A825C29
:1039D0000130134410289BB2F8D11BB293FBF0F0D6
:1039E00000B26428A8BF642020EAE07010F0BEF99D
:1039F000744910F0C3FA744910F00CFA10F0F6FB99
:103A0000724B1880DAF80030694E13F4807F00F0B2
:103A100081806F4B9F4204D92B7913B95E4B0122F1
:103A20001A71B5F900E06B4ABEF1140F1778CCBFDC
:103A30004FF0000E4FF0010E574BC7F38007BEF159
:103A4000000F06D04FF0000883F8068083F8058049
:103A500001E04FF00308E369A8790193D4F820C08E
:103A6000B5F9009069796B883288032848D8DFE877
:103A700000F0020E1B36BEF1000F02D03280002291
:103A80002BE0002F40F062863280AF713AE09CF864
:103A9000000000EB8000814502DC328001221CE046
:103AA00001206FB300F0DABE47B1019A4FF002086F
:103AB000D2897280B280BCF80200F0809CF800B01D
:103AC0009CF80100584400EB8000814500F34186DA
:103AD000002F00F03E8632800222AA7112E032806E
:103AE0000322AA7169716B8077B13A4A137843F067
:103AF00002031370284B00225A710EF007FC03E0FA
:103B00003280A87169716B80B8F1000F02D0404615
:103B10000AF036FA304FB7F852010FF086FC0197E1
:103B2000834668B90EF0A8FF2C4B0022C3F800B002
:103B3000C3F804B0C3F808B0294B1A605A609A6001
:103B4000244F3B785B0763D5DAF80030D8065FD5A1
:103B5000244B1B78D9065BD4234B1B7893B1019B74
:103B600093F8D631BBF1000F42D173B11F4B1A68E5
:103B7000636A9B1A002B08DA0EF0C8FB074B83F828
:103B800028B045E0BBF1000F3AD110200AF0F8F957
:103B900001233BE07C300020FC240020C00E0020EC
:103BA000502600200B30002020100020742F002011
:103BB0008C26002000007A44441D0020541D002063
:103BC000C90E00200000C84200C07F4480100020C1
:103BD000404B4C00A3300020B0260020741500207C
:103BE0002816002024110020080000207426002040
:103BF00033B1AD4A4FF47A71126801FB032363625B
:103C000094F8283023B10AF0A5F9002384F828306D
:103C1000019B93F8D4310293019B93F8D511B3F82B
:103C20009AE1B3F89CC10023184636F913208008A6
:103C30007245C4BF60F07F00C0B201336245B8BFB7
:103C400040F04000042BF0D194F82930974A834289
:103C500005D192F82A30F92B04D8013300E0002373
:103C600082F82A30924B84F829001A78DFF85C82B7
:103C70009946DAB9D8F80030DA0708D5BBF1000F59
:103C800014D13B78DB0711D50EF098F90EE03B78A4
:103C900058070BD5874B1B7843B16B7933B911B1FA
:103CA0000EF034FB02E0BBF1000FF9D094F82A309B
:103CB0007E4A142BDFF818B240F08F80029B00334D
:103CC00018BF0123029399F8003063B392F82930AA
:103CD0005F2B11D13B7803F0040303F0FF0113B114
:103CE0000EF014FB08E00B20049103920AF048F94F
:103CF000039A049982F82A10029BA3B194F8293000
:103D00007D2B10D13B7803F0040303F0FF0213B1C5
:103D10000EF0FCFA07E00B2003920AF031F9634B36
:103D2000039A83F82A203B7803F0040303F0FF0191
:103D3000002B52D194F829305C4A572B16D15E4B98
:103D40004FF47A721A80DAF80030190601D507F0BC
:103D500073FE5A4B1B685A0742BF594A0A21118009
:103D600013F0080339D1574A138036E0DAF800001F
:103D7000400717D55A2B15D192F82B302BB10123C0
:103D800082F82B1082F82C3027E092F82D3083F047
:103D9000010382F82D300BB10C2000E00D200AF059
:103DA000EFF81AE05D2B00F0D7845B2B00F0D6848F
:103DB0005E2B02D1032000F0D2BC562B01D104F0BF
:103DC000D5FD99F80030002B00F0DE8494F82930FE
:103DD0006F2B40F0D4840EF0F1F8DAF800305B0776
:103DE00036D594F82D30314A93B13B7858070FD52A
:103DF000019BB6F90610B3F89A31994208DDD8F85C
:103E0000003013F0010302BF3221118682F82D30F9
:103E1000D8F80030D9030CD594F83220234B22B9BE
:103E200093F82B200AB932221A86012384F8323003
:103E30000EE094F82B301D4A53B13B7803F0040395
:103E400003F0FF0123B9012382F82B1082F82C30F4
:103E5000DBF800700023C8F8003007F17B0607F19B
:103E6000CB093278737816F8010C9A420DD231469C
:103E700009F0CEFF48B116F8022C012303FA02F232
:103E8000D8F800301343C8F8003004364E45E8D166
:103E90000D4B1B78F3B10D4E084F336813F0020F32
:103EA00040F03A8332E300BF74260020C00E0020A9
:103EB000080000200A3000209A3000202011002045
:103EC00098300020FC100020A4300020201000209A
:103ED0005C10002007F1CA0607F5897732787378FD
:103EE00016F8010C9A4222D2314609F091FFF0B146
:103EF00096F804E00C21B37801FB0E41B44A013B73
:103F000003EB430313448A6B96F803809A42B1484B
:103F10000DD08B63002390F86420CB63012303FA58
:103F20000EF322EA030381F8348080F86430063609
:103F3000BE42D3D1A84BDFF8BC921F68A74B4FF00D
:103F4000000B1B680293A64B1B780393D9F8003033
:103F5000002B00F0C48293F80080B8F1000F00F04D
:103F6000BE82D9F8042002998A1A002A0CDB01F5D6
:103F7000FA72C9F8042094F86410012202FA0BF2D4
:103F800021EA020284F86420039A002A00F0A78242
:103F900019F8042C59780432D2B2002940F060821A
:103FA000904931F91210904AB2F8982102F1C800F4
:103FB000814201DD9E7814E0C83A914202DA997894
:103FC0004E420EE094F86420012303FA0BF322EA38
:103FD000030384F86430029B03F5FA73C9F80430D4
:103FE0007DE294F8643043FA0BF3DA0700F177824C
:103FF000002ECCBF0220012009F0E4FF08F1FF32BF
:10400000744B132A00F26382DFE812F014002100DF
:104010002E003D0056005D00C1003A019E01CB011B
:10402000FA0161023D004C005D00C1003A019300BD
:104030000C017001397838460E44FA2EA8BFFA26D2
:1040400026EAE6763E7009F0C9FE012019E079788B
:1040500038460E44642EA8BF642626EAE6767E70B3
:1040600009F0BCFE02200CE0F97838460E44642EBC
:10407000A8BF642626EAE676FE70996E09F066FE11
:1040800003203146B9E179790D2031446429A8BF74
:10409000642121EAE171797109F004FFB8F10D0F93
:1040A00000F0158239790E2031446429A8BF6421BB
:1040B00021EAE1713971A0E1B9790520314481F338
:1040C0000801B97199E1DB6E1A78022A22D13046D3
:1040D00004930FF04BFE45490FF050FF049B596AC3
:1040E00005930FF08FFD0021049010F031F8059B2F
:1040F00048B9049A3E49104610F048F8049A059BC6
:1041000010B13B4A00E000225A620F20114609F02C
:10411000B4FE0AE099780F203144C829A8BFC8210D
:1041200021EAE171997009F0BDFEB8F10F0F00F0BE
:10413000CE81284BD3F86C8098F80030022B1AD12E
:1041400030460FF013FE29490FF018FFD8F8201061
:104150000FF058FD002106460FF0FAFF30B9304647
:10416000234910F013F810B1214E00E00026C8F8E2
:104170002060122064E198F8011012203144C8290F
:10418000A8BFC82121EAE17188F8011035E1DB6E92
:104190001A78022A37D1304604930FF0E7FD14490C
:1041A0000FF0ECFE049B196B05930FF02BFD002123
:1041B00004900FF0CDFF059BF0B9049A0C4910460E
:1041C0000FF0E4FF049A059BB8B1094A15E000BF5F
:1041D0008CA30108C00E002084100020742600204B
:1041E0000A3000208C260020B0260020000020414C
:1041F0000000C842F80E002000221A631020114669
:1042000009F03BFE0AE0197B10203144C829A8BF01
:10421000C82121EAE171197309F044FEB8F1100FC9
:1042200000F05581B24BD3F86C8098F80030022B27
:104230001AD130460FF09AFDAE490FF09FFED8F824
:104240002C100FF0DFFC002106460FF081FF30B983
:104250003046A8490FF09AFF10B1A64E00E00026A4
:10426000C8F82C601320EBE098F80B1013203144B1
:10427000C829A8BFC82121EAE17188F80B10BCE069
:10428000DB6E1A78022A22D1304604930FF06EFDBD
:1042900099490FF073FE049BD96B05930FF0B2FCA4
:1042A000002104900FF054FF059B48B9049A9149EE
:1042B00010460FF06BFF049A059B10B18D4A00E089
:1042C0000022DA631120114609F0D7FD0AE0997D3A
:1042D00011203144C829A8BFC82121EAE17199758C
:1042E00009F0E0FDB8F1110F00F0F180804BD3F838
:1042F0006C8098F80030022B1AD130460FF036FD52
:104300007D490FF03BFED8F838100FF07BFC002100
:1043100006460FF01DFF30B9304676490FF036FFE4
:1043200010B1744E00E00026C8F83860142087E011
:1043300098F8151014203144C829A8BFC82121EAD3
:10434000E17188F8151058E0D3F86C8098F80030C7
:10435000022B1AD130460FF009FD68490FF00EFE0E
:10436000D8F828100FF04EFC002106460FF0F0FEA2
:1043700030B930465F490FF009FF10B15D4E00E0E3
:104380000026C8F8286009205AE098F80310092090
:104390003144C829A8BFC82121EAE17188F8031077
:1043A0002BE0D3F86C8098F80030022B1AD13046FD
:1043B0000FF0DCFC4F490FF0E1FDD8F834100FF09E
:1043C00021FC002106460FF0C3FE30B930464949B2
:1043D0000FF0DCFE10B1474E00E00026C8F8346054
:1043E0000A202DE098F80D100A203144C829A8BFF2
:1043F000C82121EAE17188F80D1009F053FD66E04B
:10440000D3F86C8098F80030022B1DD130460FF0A5
:10441000ADFC39490FF0B2FDD8F840100FF0F2FBB7
:10442000002106460FF094FE30B9304631490FF0B6
:10443000ADFE10B12F4E00E00026C8F840600B2002
:10444000314609F01AFD42E098F817100B2031446C
:10445000C829A8BFC82121EAE17188F81710CCE764
:10446000012934D19878264B33F91230B3F5617FA6
:1044700005DB40F633029342A8BF134601E04FF438
:104480006173B8F10C0F22D14FF4966292FBF0F0F9
:10449000A3F5617393FBF0F31A4ADEB21378B342CB
:1044A00015D0042E34BF334602231370019A08FB43
:1044B0000323154A03F2A67313600DF0F9F9404681
:1044C000314609F0EFFC701CC0B209F07BFD94F896
:1044D0006420012303FA0BF3134384F864300BF1D7
:1044E000010BBBF1040F09F10C097FF42FADD2E4ED
:1044F000C00E00200000C84200007A4400002041A5
:104500008C260020E01F002084100020DAF8003004
:10451000DB050FD56B796BB13B6898070AD5AC4BBF
:104520001B8813F001050AD10EF0A6FA012003F052
:104530006DFF04E0012003F058FF012300E0002399
:10454000326851070DD563B1012003F04EFFA04B37
:104550001B889A0708D40EF08FFA022003F056FF4A
:1045600002E0022003F041FF3B6813F00A0F26D05F
:104570003368DB060BD5964B1B885D070AD40420F5
:1045800003F044FF934B1B88A4F8703002E0042032
:1045900003F02BFF3368980607D58D4B1B8859060F
:1045A00006D4402003F032FF02E0402003F01DFF5C
:1045B00033685A0642BF874B1B88A4F872303B68A9
:1045C0009B0608D433681F0540F18E804FF480703D
:1045D00003F01CFF8CE0804B7D4F1B7813F0020F23
:1045E0004DD07E4B1B78042B49D9336813F40078E7
:1045F0000ED03B88DD0636D4102003F007FF2020C4
:1046000003F0F3FE7648011D07F080F9022326E04F
:104610003D8805F01005ADB22DB1102003F0E5FE88
:10462000012584F874803368580511D5A36F6D494E
:104630005A89B1F90030002BB8BF5B42934207DAC8
:10464000B1F90230002BB8BF5B429342C0F20C813B
:104650003B88990608D5202003F0C7FE002384F884
:104660007430012500E0002594F87C30B3B90E20A9
:1046700009F086FC5C4B012283F87C200EE03B882D
:1046800003F03003002B9DD0102003F0AEFE20205D
:1046900003F0ABFE002384F8743001E0002D91D0CC
:1046A00000200546514B002423F81540504B1A1D9D
:1046B00003F10A0122F815400022425001444C60E7
:1046C0008A6023F8154003F132015A334250C25038
:1046D000014403444C608A605C609A601430002D91
:1046E0007FF470AF0125DDE74FF4807003F07DFEAD
:1046F000404B5A791C46082A01D00E2A02D140208C
:1047000003F073FEDAF800305A0540F1C28094F8E5
:104710000C3223B9384B1B7813F0040F02E03368D6
:1047200013F4002F0BD0354B00221A703C200EF0F2
:10473000B1FB002800F0AD800BF004FAF6E70CF0B6
:10474000B7FF09B0BDE8F04F0EF015BB0120FFF731
:104750008CB90320FFF789B9012000E002205FFA3D
:1047600080F9019A09F1FF3382F8A43703F090FE33
:1047700003F030FF484609F025FCFFF72EBB029AF4
:1047800012B17E2B3FF427AB94F82930972B05D13B
:10479000154B4FF4C872DA85FFF71FBBA72B06D164
:1047A0000D4A137843F004031370FFF716BB002281
:1047B000BB2B079201D1022303E0B72B04D14FF6A4
:1047C000FE73ADF81E3021E0BE2B19D102231BE091
:1047D000E4110020FC100020241100202A110020E8
:1047E0008C10002004110020C00E00209C300020FE
:1047F0003E0F0020B0260020A33000200826002015
:10480000BD2B1AD14FF6FE73ADF81C30DBF800203B
:10481000BDF81C10B2F858300B44A2F85830BDF85F
:104820001E10B2F85A300B44A2F85A3004F09EF829
:10483000002384F82A30FFF7D0BA792B04D1164A26
:10484000D37823F0010306E07A2B7FF4C6AA124A3C
:10485000D37843F00103D370FFF7BFBA01330146A9
:104860009BB20220FFF701B93B889B063FF5FCAEE7
:10487000202003F0CBFD094B09481A685B68011D35
:104880004360026007F042F8064B012583F874503C
:10489000EAE609B0BDE8F08F881C00202C1100204A
:1048A00094100020C00E00209148F0B50368914A92
:1048B0009C8AA4B2E1B211F0010F2ED0198821F424
:1048C00000610904090C1980198889B241F48061DA
:1048D000198000211170517899B1917811B9D1786E
:1048E000FF290ED1012191701179022901BF198888
:1048F00089B241F400611980517941F001011982B6
:10490000E1E0517901F0FE011982D378FF2B00F02C
:10491000DA80784BFF211970D5E08E073AD5BFF3C6
:104920005F8F1479E4B2012C13D1517889B1917859
:1049300079B1198821F480610904090C1980BFF349
:104940005F8F198B1988947189B241F400711980B5
:104950001BE0198BBFF35F8F14796649022C0AD1D3
:104960004C7844B1897831B1198821F48061090407
:10497000090C1980A1E014795E49032C05D14C780B
:104980001CB18978002940F09880998889B241F457
:10499000806197E04D0756D501219171517800292A
:1049A00037D09178002934D011791C8802291178E8
:1049B0001DD924F480642404240C1C801E8A95686C
:1049C000CCB2F6B249B26E54198889B241F4007182
:1049D00019800168A31C13700B8A0134DBB264B226
:1049E0002B558B889BB243F480638B8026E0A4B266
:1049F00044F400741C801D8A9668CCB2EDB249B2B2
:104A000075541B8A611C49B2DBB2033473541470B1
:104A100014E09178374C09B9217B41B1198889B2EA
:104A200041F40071198013780133137006E019887E
:104A300089B241F4807119800123A37001680B8849
:104A4000DB05FCD43FE001F0400101F0FF05E1B1DE
:104A500014781F8A9668E5B2691C64B2FFB23755B4
:104A6000C9B21679117049B2CC1CA64201BF9C880C
:104A700024F480642404240C08BF9C8013798B42A6
:104A800021D11C4B02351D701DE027061BD5117866
:104A90004CB2661C0AD0156901312C5DC9B21C826A
:104AA0001479117049B28C420DD106E0D17815709D
:104AB0001982517809B9117929B9998821F480614D
:104AC0000904090C9980137992F9004001339C4242
:104AD00008490CD100238B708B7933B101688B8826
:104AE00023F440731B041B0C8B8000231375F0BD53
:104AF000D81F0020C00F0020074B984201D1074A61
:104B000003E0074B984204D1064A138801339BB255
:104B100013804FF0FF30704700300140F202002058
:104B200000380040E00600206B4B6C4A2DE9F04F46
:104B30005E8994694FEA062AB4EB0A0A9C884FF012
:104B400000054FEA04481C894FF0000BA4FB0A67DC
:104B500065EB0B0B04FB0B77F40944EA476418EB95
:104B600004065C884FF000094FEAE7154FEAC438A5
:104B7000DC8849EB050787B0CDE90467A4FB0A6729
:104B800004FB0B77340A44EA076418EB04064FEA87
:104B900027259C894FF0000949EB0507CDE90067FF
:104BA000AAFB046704FB0B77F40D44EA472414F5D1
:104BB000FA664FEAE75545F10007B6F5FA6F77F167
:104BC0000003CDE90267964666DADDE90489A4FBB5
:104BD000046704FB05F34FF0050C07EB4307A6FB46
:104BE0000C230CFB07335F104FEA3206B8EB0608C4
:104BF0004FEA920646EA837669EB07099F10DDE9E2
:104C00000023921B63EB0703CDE90023DDE9026774
:104C1000334A4FF0FF33964277EB0303CDE9048923
:104C200027DA40F6AC520023A4185D4104FB05F3DB
:104C3000A4FB04456FF0060205EB4305664202FB48
:104C40000566A4FB0223334418EB020649EB030775
:104C5000CDE904670B26A4FB062306FB0533DDE93B
:104C600000455B104FEA3202A41A65EB0305CDE95B
:104C70000045DDE902450AFB0BF3AAFB0AAB0BEB8F
:104C8000430B4FEADA7242EA4B02A41A4FEAEB7383
:104C900065EB0305CDE90245DEF81C40009B019D54
:104CA000A4FB032304FB05334FEA525848EAC32808
:104CB0004FEA6359DDE90423B8EB020269EB030311
:104CC0009946D30B43EA494300B1036009B1029B03
:104CD0000B6007B0BDE8F08FF6020020C00F002087
:104CE00024FAFFFF2DE9F04FDFF8589285B0074610
:104CF000D9F820000E460FF039F88E4C80462088F7
:104D00000FF030F84FF05C51054640460FF082F846
:104D10004FF06451824628460FF07CF80146504619
:104D20000EF06EFF4FF06251824640460FF072F86F
:104D30004FF06A51804628460FF06CF80146404615
:104D40000EF05EFF0546B4F902000FF00FF80146C1
:104D500028460FF05FF85146054650460FF05AF8C6
:104D60008046B4F904000FF001F8014640460FF008
:104D700051F8014628460EF045FF80460FF010FA24
:104D80006D490546A06140460FF0F8F8D9F8243087
:104D90008046284601930EF0E9FF4FF07C510FF05A
:104DA00039F866490EF02CFF0546E389B4F90A008C
:104DB00002930EF0DBFF29460FF02CF829460FF086
:104DC00029F84FF058510FF025F88146B4F9080042
:104DD000B4F810B0B4F80CA00EF0C8FF29460FF0DC
:104DE00019F8014648460EF00DFF4FF058510FF0EC
:104DF00011F84FF060510FF00DF84FF07E510EF0AA
:104E000001FF8146E0880EF0ADFF014648460FF0F5
:104E100001F8002181460FF091F900287BD1294645
:104E200028460EF0F7FF03900FFA8BF00EF09EFF6E
:104E3000039B014618460EF0EDFF4FF060510EF057
:104E4000E9FF8346BDF908000EF090FF01462846B1
:104E50000EF0E0FF01460EF0D5FE014658460EF07A
:104E6000D1FE4FF07A510EF0D5FF834601980EF037
:104E70007DFF01464FF093400EF0C2FE05460FFA4B
:104E80008AF00EF073FF4FF08F410EF0C3FF014622
:104E900058460EF0B7FE4FF066510EF0BBFF0146CC
:104EA00028460EF0ADFE26490EF0B4FF49460FF03D
:104EB00065F80546B4F916000EF058FF29460EF0C5
:104EC000A9FF29460EF0A6FF4FF040510EF0A2FFB9
:104ED0008146B4F914000EF049FF014628460EF051
:104EE00099FF4FF060510EF095FF014648460EF0D5
:104EF00089FE8146B4F912000EF038FF014648469B
:104F00000EF080FE4FF076510EF084FF01462846E9
:104F10000EF078FE00E0002017B10FF041F9386084
:104F20002EB140460FF03CF964235843306005B081
:104F3000BDE8F08F480300200000A04500007A473C
:104F40000050C345C00F0020704770472DE9F04165
:104F5000324C334D62892B8DB4F904809A1A23891F
:104F6000B4F902E05A43B4F91230D613B4F914205C
:104F7000DB02324493FBF2F232440A26E2615643EA
:104F8000A2F57A6202FB02F3B4F90EC002FB0EFE38
:104F900002FB08F2B4F90C801B130CFB03FC03FBAF
:104FA00008F31B1403EB62320232E388921002F51D
:104FB000004253434CF25032B4F920704FEAEE2EC7
:104FC000B4F900400EEBEC2C0CEB8404BC40ED6A11
:104FD0000234A5EBA4043A4162434FEAD3384EBFF2
:104FE000B2FBF8F35400B4FBF8F340F6DE3448BFEC
:104FF0005B001A12524362430A4C08365C43241485
:1050000004EB224202F6CF62361103EB221300B109
:10501000036001B10E60BDE8F08100BF080300200D
:10502000C00F002043E3FFFF024B4FF480521A8071
:10503000704700BF1C000020704710B5224C236849
:10504000998A89B211F4706F1EBF204A012082F83C
:10505000300011F4E06F2BD01A8B9A88890522F466
:1050600080624FEA02424FEA12429A8020D41A88A4
:1050700092051DD41A88D0050FD51A88D105FCD405
:105080001A8892B242F400721A801A889205FCD4EF
:105090000F4B18780AF056FB0AE01A8892B242F4D5
:1050A00000721A809A8822F440721204120C9A80BC
:1050B0002268938A23F470631B041B0C9382034BB6
:1050C00000221A7510BD00BFD81F0020C00F00209D
:1050D000DC1F0020054A08B5138801339BB21380FA
:1050E000034B18780AF02EFB002008BD1E1000208C
:1050F000DC1F002010B51E4C4000C0B2A36023612D
:105100001C4B6071E17001200021217360702271DD
:105110002075186884F8301040B383889B0515D437
:105120000388D9050DD447F230530288920502D581
:10513000013BFAD112E08BB103889BB243F4807338
:10514000038083889BB243F44073838047F23053DB
:10515000227D12B1013BFBD100E013B9BDE8104044
:10516000B8E7034B93F8300080F0010010BD00BF9A
:10517000C00F0020D81F002007B5002101AB03227B
:105180007720FFF7B7FF9DF805309DF804001B025C
:1051900043EA00439DF80600184303B05DF804FBA2
:1051A00008B5FFF7E9FF014BD86108BDC00F00202B
:1051B00008B5FFF7E1FF014B986108BDC00F002063
:1051C00007B5F7216B4606227620FFF793FF9DF87F
:1051D00000309DF801101B0343EA01139DF80210F3
:1051E000094A43EA111353629DF803309DF80410F5
:1051F0001B0343EA01139DF8051043EA11131362E0
:1052000003B05DF804FB00BFC00F002007B5F62116
:1052100001AB03227720FFF76DFF9DF805309DF865
:1052200004201B0243EA02439DF806201343054A6B
:10523000B2F92020C2F10802D340034AD36203B07E
:105240005DF804FB08030020C00F002007B5F6211D
:1052500001AB02227720FFF74DFF9DF804209DF857
:10526000053043EA0223024A138503B05DF804FBCC
:10527000C00F002013B5204B400002ACC0B25871E3
:1052800004F8012DD970012200211A7359701A7186
:105290001A751A4A1C6110689C6083F8301040B37C
:1052A0008288920515D40288D4050DD447F2305275
:1052B0000188890502D5013AFAD112E08AB1028843
:1052C00092B242F480720280828892B242F44072BA
:1052D000828047F23052197D11B1013AFBD100E0D2
:1052E00012B9FFF7F7FE04E0034B93F8300080F0AB
:1052F000010002B010BD00BFC00F0020D81F002069
:10530000772048210122B5E7772058210122B1E713
:105310007620F4213122ADE7044B772093F820204A
:10532000F4219201343202F0FC02A3E708030020CA
:105330007720F4212E229DE7FFF7B6BA7DE6FFF72E
:10534000B3BA7AE670B584894FF47A74FBB112B1BE
:105350001578013207E0FF2505E04FF6FF76013CA6
:10536000A4B2B4420DD00689B607F6D5ADB2858198
:105370000589ED070DD44FF6FF75013CA4B2AC4290
:10538000F6D1FFF7B9FB003018BF012070BD012036
:1053900070BD8589ADB209B10D700131013BD5E712
:1053A00008B540F2E9330289920704D4013B9BB26D
:1053B000002BF8D10AE040F2E93389B281810289F9
:1053C000D20706D4013B9BB2002BF8D1FFF794FB28
:1053D00000E08089C0B208BD2DE9F041174688463B
:1053E000084C094E102540F0800165613046FFF7FA
:1053F000D7FF3046414600223B46FFF7A3FF256119
:10540000BDE8F081000801400030014013B50122E1
:1054100004460DF107013A20FFF7DEFF9DF8073043
:1054200003B10123237002B010BD184A13B51388CD
:10543000044623F040031B041B0C138013883B20FD
:1054400023F038031B041B0C1380138869469BB29E
:1054500043F0400313800622FFF7BEFF9DF80020B3
:105460009DF8013043EA022323809DF802209DF835
:10547000033043EA022363809DF804209DF8053041
:1054800043EA0223A38002B010BD00BF00300140F8
:10549000174A13B51388044623F040031B041B0C62
:1054A00013801388432023F038031B041B0C138044
:1054B000138869469BB243F0400313800622FFF72E
:1054C0008BFF9DF800209DF8013043EA02232380E2
:1054D0009DF802209DF8033043EA022363809DF883
:1054E00004209DF8053043EA0223A38002B010BDDA
:1054F00000300140F8B503460F46074C074E102513
:10550000194665613046FFF74BFF30463946FFF7D5
:1055100047FF2561F8BD00BF000801400030014091
:10552000284A08B51388802123F040031B041B0C74
:10553000138013886B2023F038031B041B0C43F0EB
:105540003003138013889BB243F040031380FFF7AE
:10555000D1FF962008F0DFFC03216820FFF7CAFF87
:10556000962008F0D8FC03216B20FFF7C3FF012031
:1055700008F0C6FC10216A20FFF7BCFF012008F0EC
:10558000BFFC00216C20FFF7B5FF012008F0B8FC3C
:1055900000211920FFF7AEFF012008F0B1FC102117
:1055A0001C20FFF7A7FF012008F0AAFC1B201821F0
:1055B000FFF7A0FF012008F0A3FC034B01221A70A3
:1055C00008BD00BF00300140F00200201F4A13B5A3
:1055D00013886B2023F040031B041B0C13801388DB
:1055E000802123F038031B041B0C43F0300313808D
:1055F000138806249BB243F040031380FFF77AFF21
:10560000962008F088FC75200DF107010122FFF7B4
:10561000E3FE9DF80730682B04D0013C14F0FF0432
:10562000EED10EE00C200DF107010122FFF7D4FEB0
:105630009DF80730142B04D3182B04D9543B062BA8
:1056400001D9002000E0012002B010BD003001406F
:105650002DE9F0474B28A0B0044600F0458600F243
:10566000B480302800F0D08651D8222800F09184F0
:1056700023D8032800F0608114D8012800F050815D
:10568000022840F02C8704200AF0C8FA43200AF0D0
:1056900096FA4C200AF093FA46200AF090FA4C2031
:1056A00000F057BE042800F05181052840F017870C
:1056B0001A200AF0B3FA002459E1282800F0E28504
:1056C00015D8242800F0C985262840F00887B44C56
:1056D00006200AF0A3FAB4F85C010AF0A2FAB4F8C2
:1056E0005E010AF09EFAB4F8600100F0B3BD2C2808
:1056F00000F0DB852E2800F057862A2840F0EF8640
:1057000001200AF08BFAA64B587900F022BE3D2802
:1057100000F0EF821ED8362800F02C860BD83228F5
:1057200000F01186342840F0DA8648200AF076FA34
:10573000002500F050BC3A2800F0AF823B2800F072
:105740002184382840F0CB8604200AF067FA944C74
:1057500000F089BD452800F0AF8627D8402800F02A
:10576000FB85422840F0BB868D4C10200AF056FA8B
:1057700060790AF024FAA0680AF05CFA94F89201C1
:105780000AF01DFAB4F85C010AF04BFAB4F85E01B5
:105790000AF047FAB4F860010AF043FAB4F882015B
:1057A0000AF03FFAB4F8840100F054BD472800F035
:1057B0006186C0F04E86492840F0918602200AF0AA
:1057C0002DFA774B988900F045BD702800F0E482EF
:1057D00058D8692800F041822AD8652800F0FA805C
:1057E00015D84D2800F08F85642840F07886072072
:1057F0000AF014FAE7200AF0E2F9694B58790AF046
:10580000DEF900200AF0DBF9042000F064BE67280E
:1058100000F0A68100F2148212200AF0FFF9614B19
:1058200000241B88B3F5806F8CBF082501257AE121
:105830006C2800F0258217D86A2800F091846B2824
:1058400040F04D8605200AF0E9F9574B18880AF018
:10585000E8F9564B18880AF0E4F9554B93F86E00B6
:1058600000F0010000F075BD6E28514D00F01C8263
:1058700000F26A8206200AF0D1F9E86D0AF0DAF93E
:105880004C4B08E2782800F0788119D8742800F091
:10589000C3830BD8722800F02384732840F01F863E
:1058A00008200AF0BBF9012400F053BC762800F070
:1058B000778400F2F5832F200AF0B0F93E4C59E3CB
:1058C000A42800F0938414D87B2800F0F982A02843
:1058D00040F005860C200AF0A1F9384B18680AF050
:1058E000A9F9374B18680AF0A5F9364B186800F08B
:1058F000F2BDF12800F07D81FE2800F09E84F028A2
:1059000040F0ED852A4C04200AF088F9236CB3F8A6
:105910005A000AF086F9236CB3F8580000F09ABCDC
:1059200003200AF07BF900200AF049F920460AF02A
:1059300046F90C2000F00DBD0AF070F901200AF0C4
:105940003EF90A200AF03BF900F04EBC06200AF0AE
:1059500065F943200AF033F943200AF030F9332087
:105960000AF02DF944200AF02AF900F072BC164B17
:10597000185D01340AF023F90B2CF8D10024134BE5
:10598000185D01340AF01BF9082CF8D10024104BE3
:10599000185D01340AF013F9072CF8D100F09DBD11
:1059A000B02600201C0000209E110020A011002025
:1059B0001C100020F4100020C7A30108E8F7FF1F07
:1059C000ECF7FF1FF0F7FF1F7CC3010888C3010835
:1059D0005DC30108CC4C0B200AF020F920880AF0A6
:1059E00020F9608880B20AF01CF9C84B1B68C3F329
:1059F000C000C3F38002800040EA4200C3F34002CB
:105A00001043C3F3401240EAC20003F010031843EE
:105A10000AF007F9BE4B1A88636812F0010F14BF31
:105A20004FF0020C4FF0000C12F0020F02F00808C9
:105A300014BF4FF0040E4FF0000E03F4475912F05C
:105A4000040F14BF1027002749EA080912F0400F7D
:105A500003F4804814BF2026002649EA080912F002
:105A6000100F03F4004814BF4FF40075002549EAF5
:105A7000080912F0200F03F4803814BF4FF480603F
:105A8000002049EA080912F4807F03F4003814BFAB
:105A90004FF40061002149EA080912F4007F03F481
:105AA00080289C4A49EA080903F4002849EA0809C1
:105AB000127803F4801849EA080903F0007349EAF0
:105AC0000303C2F3800243EA020343EA0C0343EAFE
:105AD0000E0E4EEA070746EA070645EA060540EAC3
:105AE000050041EA00014FF00000034614BF4FF4E7
:105AF00000184FF0000841EA0808217A8B420BD2C7
:105B0000854A9C5C012202FA04F414EA080F1CBFC7
:105B10009A4010430133F1E70AF08CF87F4B93F879
:105B2000A40700F016BC7E4B33F91400013490FB3F
:105B3000F5F080B20AF075F8032CF4D1724CA08C09
:105B40000AF06FF8E08C0AF06CF8208D0AF069F822
:105B5000608D0AF066F8A08D0AF063F8E08D79E3B5
:105B600010200AF05BF800246E4B185D01340AF037
:105B700026F8102CF8D100F0B0BC70200AF04EF8D6
:105B800000260E247443604D01362B6C2344B3F879
:105B900019010AF046F82B6C2344B3F81B010AF0F4
:105BA00040F82B6C2344B3F81D010AF03AF82B6C33
:105BB000234493F81F010AF002F82B6C234493F856
:105BC000200109F0FCFF2B6C234493F8210109F01C
:105BD000F6FF2B6C234493F8220109F0F0FF2B6CA5
:105BE0001C44D4F823010AF025F8082EC9D100F08E
:105BF00074BC70200AF012F8484C04F1700594F857
:105C0000D40009F0DCFF94F8D50009F0D8FF94F82F
:105C1000D60009F0D4FF94F8D70009F0D0FF94F82B
:105C2000D80009F0CCFF94F8D90009F0C8FF073478
:105C300094F8D30009F0C3FFAC42E0D100F04DBCB2
:105C4000102009F0EBFF0024374B185D013409F0F8
:105C5000B6FF102CF8D100F040BC344D0024287859
:105C6000400000F0FE0009F0D9FF2B789C4280F044
:105C700034842F4B33F8140009F0D3FF0134F4E7D8
:105C80002C4C062009F0CAFF208809F0CAFF608862
:105C900009F0C7FF284B1888DCE2042009F0BEFF9A
:105CA000194B186E00F017BC072009F0B7FF234B03
:105CB0001888FF28A8BFFF20C0B209F080FF204B42
:105CC000186880F3100080B209F0ABFFB5F86400EB
:105CD00009F0A7FF114B93F887211A4B186822B1DE
:105CE0000A23584380F3100001E000F30F0080B254
:105CF000B0E20A4C022009F091FF94F8D60109F0B5
:105D00005EFF94F8D50124E31C1000202011002030
:105D1000E4110020A330002025100020B026002030
:105D2000EE1000204C1000206010002008300020F1
:105D30008C26002046260020FC1000201011002098
:105D40001C110020181100200B2009F067FFAB6E1A
:105D50000026187809F033FFAB6E587809F02FFF52
:105D6000AB6EBE4C33441879013609F028FF032E80
:105D7000F6D1A36ED87909F022FFA36E987809F0C6
:105D80001EFFA36ED87809F01AFFA36E588909F098
:105D900048FFA36E187ADCE2B04C1E2009F03EFFEB
:105DA000236C00251B78022B77D1236C05F10802A8
:105DB00053F82200AA490EF02DF811F0C5FFFA2879
:105DC000A8BFFA2020EAE070C0B209F0F8FE236C08
:105DD000A44903EB8503D86A0EF01CF811F0B4FF58
:105DE000FA28A8BFFA2020EAE070C0B209F0E7FE66
:105DF000236C05F10E0253F822009B490EF00AF8BD
:105E000011F0A2FF6428A8BF642020EAE070C0B2AD
:105E1000013509F0D4FE032DC7D1072D236C2AD1FB
:105E2000586C8F490DF0F6FF11F08EFFFA28A8BFCD
:105E3000FA2020EAE070C0B209F0C1FE236C884964
:105E4000986C0DF0E7FF11F07FFFFA28A8BFFA2049
:105E500020EAE070C0B209F0B2FE236C93F84C0067
:105E60000DF080FF11F070FFFA28A8BFFA2020EA99
:105E7000E070C0B20BE02B44587809F0A0FE236C10
:105E80002B44D87A09F09BFE236C2B44587D0135B6
:105E900009F095FE0A2DC0D11FE3236C2B445878DE
:105EA00009F08DFE236C2B44D87A09F088FE236C10
:105EB0002B44587D013509F082FE0A2DEDD10CE30B
:105EC0003C2009F0ABFE0024644D04F108022B6C69
:105ED000654953F822000DF09DFF11F035FF80B2A7
:105EE00009F09FFE2B6C604903EB8403D86A0DF028
:105EF00091FF11F029FF80B209F093FE2B6C04F1A1
:105F00000E0253F8220058490DF084FF11F01CFFD7
:105F1000013480B209F085FE032CD5D1072C2B6CFF
:105F200016D1586C50490DF075FF11F00DFF80B27D
:105F300009F077FE2B6C4C49986C0DF06BFF11F05B
:105F400003FF80B209F06DFE2B6C93F84C000BE060
:105F50002344587809F065FE2B6C2344D87A09F065
:105F600060FE2B6C2344587D013409F05AFE0A2C44
:105F7000D4D1B2E214F8010F002800F0AE8209F08B
:105F80001EFEF7E7012009F049FE344B1B6C187820
:105F9000DFE1502009F042FE0025304B0C211C6C43
:105FA000324B04EB850494F87920013501FB023370
:105FB00093F8380009F003FE94F87A0009F0FFFD29
:105FC00094F87B0009F0FBFD94F87C0009F0F7FDE4
:105FD000142DE2D181E2214B1C6C062303FB054406
:105FE00094F8CE0009F0EBFD94F8C90009F0E7FD44
:105FF00094F8CA0009F0E3FD94F8CB0009F0DFFD46
:1060000094F8CC0009F0DBFD013594F8CD0009F0DF
:10601000D6FD0C2DDFD160E24FF0000801260027ED
:106020000E4B1A7A974232DA0933FA5C00240C23B9
:1060300063430E4D05F13001595C914207D12B4469
:10604000586B11F0B8FC82462EB9B14610E001340D
:106050001B2CECD119E0804417E000BF1C1000207D
:10606000000020410000C84200007A44C8A3010893
:10607000D1450ADA0C2303FB04535B6B13F80900C8
:1060800009F09DFD09F10109F2E70137C8E7002E8B
:1060900000F023825FFA88F009F0C0FD0026BEE719
:1060A000CC4D0024287A09F0B9FD2B7A9C4280F06F
:1060B0001482C94B0021E65C0C2202FB01F3C748A5
:1060C00000F13007DA5DB24205D1034493F838009D
:1060D00009F075FD02E001311B29EDD10134E4E73F
:1060E000BF4C162009F09AFDB4F8980109F099FD0B
:1060F000B4F8440109F095FDB4F8460109F091FDAA
:10610000B4F8480109F08DFDB4F8D20109F089FD19
:1061100094F8E30109F053FD002009F050FD94F8D4
:10612000E40109F04CFD94F8870109F048FD94F86A
:10613000940109F044FD002009F041FDA54B0A201F
:106140001B6CB3F9563093FBF0F080B209F069FD97
:1061500089E0E0B2013409F032FD092CF9D1BCE14B
:10616000102009F05BFD9F4B9F4C187800F0020057
:1061700009F025FD9D4B187809F021FD206809F0F4
:1061800059FD606809F056FD994B188809F049FDE2
:10619000984B188809F045FD8E4BB3F86C0059E018
:1061A00009F0F0FC0746122009F038FD894C17B9B8
:1061B000266F656F05E0102F19BF00252E46A66FCC
:1061C000E56F384609F0FBFC304609F033FD284600
:1061D00009F030FDD4F8800009F02CFD002009F012
:1061E00020FD002009F01DFD0020B2E0794D0024C3
:1061F00095F884002E4680000130C0B209F00EFDF3
:1062000095F8840009F0DBFC96F884309C4280F01D
:106210006481794D285D09F0D2FC05F11003185D09
:1062200009F0CDFC05F12003185D303509F0C7FCFD
:10623000285D09F0C4FC0134E6E7082009F0EEFC13
:10624000002009F0EEFC002009F0EBFC002009F032
:10625000E8FC002009F0E5FC3FE1042009F0DEFC49
:106260005F4B986837E194F87C0109F0A8FC94F83A
:10627000800109F0A4FC94F87F0109F0A0FC94F8D7
:10628000810166E0564C072009F0C8FCB4F8820191
:1062900009F0C7FCB4F8840109F0C3FC94F8860146
:1062A00009F08DFCB4F88801D4E74D4C0C2009F0BE
:1062B000B5FC94F8920109F082FCB4F89C0109F055
:1062C000B0FCB4F8980109F0ACFCB4F89A0109F0FC
:1062D000A8FC94F8930109F072FCB4F89E0109F04F
:1062E000A0FCB4F8A001B5E73D4C042009F096FCF1
:1062F00094F8D00109F063FC94F8D10109F05FFC37
:10630000B4F8D201A6E73D4C3D4D20780426043870
:1063100000EB4000C0B209F081FC237802359E42B8
:1063200080F0DB8015F8020C09F049FC15F8010C2F
:10633000013600EB800000EB800000F2EE2080B21E
:1063400009F06FFCE9E7012009F068FC244B93F8A1
:10635000940109F034FCC0E0082009F05FFC00243F
:106360001F4B234493F88A01013409F028FC082CC0
:10637000F6D1B2E0174B1A4C93F8C50004F1200592
:10638000C0EBC000C0B209F049FC94F8EA01002358
:106390001C4AD25C904200F0A4800C33302BF7D121
:1063A0000834AC42F1D198E0402009F037FC0C4CA5
:1063B00004F14005B4F89C0209F033FC94F89E0205
:1063C00009F0FDFB043494F89B0209F0F8FBAC42A1
:1063D000F0D182E01C10002025100020C8A3010885
:1063E000B0260020241100202C1100202A110020AA
:1063F0002811002026110020A110002008300020C4
:106400005228002010260020E02009F007FC424C12
:1064100004F18005B4F81E02043400F03F0009F0D6
:1064200000FCB4F81A02C0F3861009F0FAFB94F8E5
:106430001802000909F0C3FB94F8180200F00F00DD
:1064400009F0BDFB94F8190209F0B9FBAC42E1D1A7
:1064500043E0324C0D2009F0E1FB09F053F809F05C
:10646000AEFB208809F0E6FBE06809F0E3FB05F0ED
:106470008BFB30E009F09AFB0546842009F0CEFB47
:10648000284609F0D7FB254BDC6805F18003A342C1
:106490008CBF641B802405F037FC284622466946E1
:1064A00009F068F805460024AC4216DA1DF804002D
:1064B00009F085FB0134F7E7132009F0AFFB002456
:1064C000174B185D013409F07AFB0B2CF8D1002032
:1064D00009F0B0FB002009F0ADFB012018E000201E
:1064E00016E009F06CFBB4F8EC0109F09AFB94F8A3
:1064F000EE0109F064FB94F8EF0109F060FB94F8F9
:10650000F10109F05CFB94F8F00109F058FB47E752
:1065100020B0BDE8F08700BFB02600200C000020AE
:106520007CC301082DE9F347C54C06462378C54FC7
:10653000002B00F0D9813A686368D31A7C2B40F2B3
:10654000D381237A6260013323724FF0000808F18F
:106550002400BB4DC0B20BF05FF805F10A0333F91C
:1065600018000DF003FCB84B814618880DF0FEFBB7
:10657000014648460DF002FDB4490DF04BFC0DF00C
:106580000FFE08F1010800B20BF034F8B8F1030F68
:10659000DDD130200BF040F8B5F910000BF02AF8EF
:1065A0000BF032F82B7A9A072CD141F288336A68C3
:1065B0009A4218D910200BF02FF868694FF0640840
:1065C00090FBF8F000B20BF015F821200BF024F846
:1065D000686990FBF8F308FB13000028B8BF40423D
:1065E00000B20BF007F814200BF016F8B4F91800FD
:1065F0000BF000F81C200BF00FF800200AF0FAFF57
:106600000BF002F8237ADFF838825B0740F049810B
:1066100002200BF001F8D8F81C006423323090FB04
:10662000F3F000B20AF0E6FFB8F926504FF0050A81
:1066300095FBFAF503200AF0EFFF854BADB21B780E
:10664000DFF8209213F0040F0BD030460CF0EDFE73
:1066500028B9D9F8003013F0100F18BF002528B260
:1066600005E0D8F828309889B0FBFAF000B20AF0BB
:10667000C1FFD9F800309E0765D5DFF8EC91A28DF7
:1066800099F800304FF0640808FB02325B00B2FB5F
:10669000F3F3E68D06203601B6B246EA0326B6B21B
:1066A000C3F303231E430AF0B7FF30B20AF0A2FF80
:1066B000E38D99F8001001339BB293FBF1F201FBDB
:1066C0001233E385236B5E4D9B7B012B05D1392073
:1066D0000AF0A2FFB5F92C0019E0AD8D6E235D43E1
:1066E000152695FBF6F53A20AEB20AF095FFB6FBFB
:1066F000F8F528B208FB15650AF07CFF3B200AF08C
:106700008BFFA8B2451D0A2095FBF0F000B20AF0FD
:1067100071FF28200AF080FF636B0A2093FBF0F0E2
:1067200000B20AF067FF04200AF076FFA36A9B8993
:1067300013B107F0F9F903E0414B986B80F31000B7
:1067400000B20AF057FFE36B3D4E9D0640F19F807B
:1067500096F8403098071DD511200AF05DFFB6F875
:1067600042004FF4F36568433A4B90FBF3F000B2FC
:106770000AF040FF19200AF04FFFB6F842004543E7
:10678000642095FBF0F595FBF0F300FB135000B28D
:106790000AF030FF94F84030B4F8445013F0020F80
:1067A00008BF002501200AF037FF28B20AF022FFB7
:1067B00009200AF031FF00200AF01CFF264B94F854
:1067C00046501A88B2F5967F0AD91D4B1B7A03F002
:1067D0000F03072B04D842F20F75954228BF1546C8
:1067E00005200AF019FF236B5B7B0BB928B216E07A
:1067F000A5F120000DF0BAFA18490DF0BFFB0021F9
:1068000005460DF0A5FC10B94FF07C5101E04FF0AA
:106810003F4128460DF0F6F90DF0C2FC00B20AF037
:10682000E9FE94F84020064B910703D493F84720E3
:10683000012A1BD1012384F8473009482DE000BF0D
:10684000E4100020742600201C00002000007A4480
:10685000A3300020A0860100FA0000206666E63F13
:106860002C11002050260020F80000201D6BAF499D
:1068700068680DF0CFFA0DF093FCAC490090A86861
:106880000DF0C8FA0DF08CFC0190684605E0A84AAE
:1068900092E803008DE8030068460AF0CDFE0AF096
:1068A000B3FE237A282B1FD1A24B00221A723B6819
:1068B0004FF47A70B3FBF0F83C2617200AF0ACFED8
:1068C000B8FBF6F5B5FBF6F006FB1050000200B27F
:1068D0000AF090FE18200AF09FFE06FB158000B219
:1068E0000AF088FE0AF090FE94F85030914D002B8B
:1068F00000F0408107F0EAFA6B6D8F4AC31A9342A9
:10690000064640F2C280002385F85A3085F85C3094
:10691000AB8DDAB21B0A85F8762085F8773085F8DA
:106920006C2085F86D30D5F884203B689A1AD5F82C
:106930008830D97B4FF47A734B439A420ED37F4B06
:106940001B68C5F8843095F88C30013B012B9FBF44
:10695000102385F85A30022385F85C30626B0A20D8
:10696000A36B92FBF0F293FBF0F384F87420121205
:1069700084F8752084F8783094F840201B1284F84D
:10698000793094F8463092076A4984F8A73003D4E6
:106990002D2381F8A83077E0D4F848906848DFF8D4
:1069A000ACC199FBF0FA0CFB0A924FF0060E042BD7
:1069B0000EFB02F28CBF3323322381F8A830614BE7
:1069C000E76C92FBF3F197FBF0F003FB11226425D7
:1069D00092FBF5F20CFB007C0EFB0CFE84F8992078
:1069E000121284F89A209EFBF3F203FB12E393FB4E
:1069F000F5F30AEB8A0A4FFA81F80AEB8A0A08EBE8
:106A00008A0189B284F8971000EB8000090A84F8A3
:106A1000981000EB800051B201EB800292B284F832
:106A20009C20120A84F89D2084F89E30B4F84220FD
:106A30001B1284F89F302423534393FBF5F5B4F8DD
:106A4000BA300A2284F8A0301B0A84F8A130B4F8C6
:106A500044304FEAD979B3FBF2F303F5FA739BB2F2
:106A600084F8A2301B0A84F8A330B4F8BC30FF0FBE
:106A700084F89450C5F3072584F8969084F89B70A9
:106A800084F8955084F8A930666594F8BE80294D45
:106A9000B8F1000F0DD1D5F8C40007F0E7FA0128CE
:106AA00007D90228284F00F038820AF095FD01230B
:106AB000BB70D4F8C8001F4D00285BD095F8BE709D
:106AC0003FB140F6B732D5F8D030F31A93420BD825
:106AD00050E00123D5F8C400022185F8BE3007F04C
:106AE000B9FA85F8D47043E095F8CC305BB9D5F8A5
:106AF000C4000121C5F8C83085F8BE3007F0AAFAF5
:106B00000AF06AFD34E0013BDBB285F8CC3095F841
:106B1000D41095F8D520DBB94B1C013285F8D43060
:106B200085F8D520D5F8C40020E000BF8096184B2A
:106B300048A50108E41000203F0D03007426002042
:106B40008096980040420F001C000020806967FF7B
:106B5000034613F8017B01327818394685F8D400D2
:106B6000D5F8C400C5F8C83085F8D52007F081FAFB
:106B7000C4F8D06094F8D6309C4DF3B1D5F8D83035
:106B8000DBB1D5F8DC30C3B1C5F8E0301B68984AFA
:106B9000C5F8E430D5F8E8301344187AFEF758FD0C
:106BA000D5F8E030987909F00AF8D5F8E8300133E3
:106BB000092B88BF0023C5F8E8308E4D94F8EC20EF
:106BC0002E688A4B002A00F0E281D3F8F020002AD8
:106BD00000F0DD8193F8F430013B012B00F2D78106
:106BE000D4F8F000814F07F041FAE0B1D7F8F00097
:106BF00007F039FA97F8F53080467E2BD5F80090EB
:106C00000ED102231B2887F8F43009D1D7F8F00001
:106C100007F02CFA20B90123C7F8F89087F8FC3068
:106C200084F8F580DCE7D7F8F8202B689B1A41F64A
:106C3000583293421DD9032387F8F430A7E16E4AF6
:106C400032F8130010B903464FF403600133B0F576
:106C5000C06FDBB275D01DD9B0F5006F7AD031D9D5
:106C6000B0F5036F3ED184F8FD30E36B5F4F9906BA
:106C70003FD494F8FC1094F8FD30002900F04A81CC
:106C80002A68921B012ADAD984F8FD30002384F89F
:106C9000FC307CE1B0F5007F42D007D8B0F5807FB2
:106CA00047D0B0F5887F00F08380E6E7B0F5806FCD
:106CB00000F0A680B0F5826F00F0EB80B0F5047FA5
:106CC000DBD123E0B0F5E26F00F08280B0F5E46F35
:106CD00000F08380B0F5E06FCFD184F8FD30B4F9D7
:106CE0000A107EE0B0F5046F6BD0B0F5026FC4D12E
:106CF000FAE097F840309A07BBD5B7F84210242342
:106D00004B436421123393FBF1F1FDE084F8FD3035
:106D10003A4B364F1B689B07ABD5BB8D0A21F2E07F
:106D200084F8FD30354B314F1B681905A1D5796BBF
:106D3000EAE084F8FD30E36B2C4F5A0799D5796966
:106D4000E2E084F8FD302D4B284F1B681B0590D5E1
:106D5000B96BD9E0E16B254A8F0684F8FD3088D500
:106D600092F84010880784D5D90710D5D36C192222
:106D700083EAE371A1EBE37101EB5101B1FBF2F1A5
:106D8000002BACBF41F0004141F040410DE0936C5D
:106D9000192283EAE371A1EBE37101EB5101B1FB2D
:106DA000F2F1002BB8BF41F080414FF400608AE05F
:106DB00084F8FD30E36B0D4F5B077FF55AAF3969FF
:106DC000A2E084F8FD30B4F91830642159437AE028
:106DD00084F8FD30B4F90C1003E0B4F90E1084F817
:106DE000FD302C2391FBF3F16DE000BFE410002097
:106DF00048A50108742600206CC701085026002011
:106E000084F8FD3094F8FE30624A0133DBB2032B84
:106E100088BF012382F8FE3042F2107394F8FE100E
:106E200059435D4B1B78D80748BF01319A0748BFCB
:106E300002315F07B4F8003148BF0431D80748BFBA
:106E40000A319A0748BF14311F0648BF2831D805B8
:106E500048BF28315A0748BF64311F0748BFC831AF
:106E6000980548BF01F5C8719A0648BF01F57A71C7
:106E7000DF0648BF01F5FA61580648BF01F57A619F
:106E80004FF480600AF074FB424B002283F8FC2030
:106E9000EFE6E16BDFF8FC8011F0200784F8FD30AD
:106EA00017D098F8402012F0020F14BF4FF47A71F7
:106EB000002112F0010F14BF4FF4FA6300230B44BA
:106EC00094F8461019440AF053FB002384F8FC3070
:106ED000CFE6324B1B6819067FF5CBAE39460AF078
:106EE00047FB88F8FC70C4E684F8FD30E36B294F5B
:106EF0009A067FF5BEAE97F840309B077FF5B9AE96
:106F0000B7F84430642159430AF032FB002387F874
:106F1000FC30AEE684F8FD3039E0BB7823B1C5F82B
:106F2000C06087F80280C4E5D5F8C030F31AB3F525
:106F30007A6FFFF4BEAD0123D5F8C400BB7007F033
:106F400092F80746D5F8C40007F08DF87F067FF465
:106F5000B0AD8A2802D08E280CD0AAE5EB6B98063B
:106F60007FF5A7AD95F8BE30002B7FF4A2AD05F1FB
:106F70008D0306E095F8BE30002B7FF49AAD05F145
:106F80005803C5F8C8302D2385F8CC3091E502B000
:106F9000BDE8F087E4100020A33000205026002038
:106FA000F8B504460E46174600252046202110F06D
:106FB000F4FC0446D0B10134204610F051FDB0F588
:106FC000617F05DB40F634039842A8BF184601E014
:106FD0004FF46170A0F56170192390FBF3F00DB9C7
:106FE000307000E070703B7801333B700DB90125C3
:106FF000DBE72046F8BD7FB504780646E4B9364B9A
:107000001921186800EB840090F87B5090F87920E3
:107010004D4305F5617590F87A30009590F87C0045
:10702000414301F5617101912C482146013401F081
:1070300069F8142CE3D14CE010F012FD132805463A
:1070400041DC254B701C1C68202100238DF80F307B
:1070500010F0A3FC1E35064670B10136304610F024
:10706000FFFC19289FBF04EB850358709DF80F3073
:10707000013398BF8DF80F303046202110F08DFC81
:10708000064670B10136304610F0EAFC0D289FBF6D
:1070900004EB850398709DF80F30013398BF8DF88D
:1070A0000F3004EB85043046E11C0DF10F02FFF7B1
:1070B00077FF9DF80F30042B0BD0601C00210422B9
:1070C00010F035FC05E0064806490022132301F0C4
:1070D00019F804B070BD00BF5C1000205CC8010846
:1070E00071C8010890C80108014808F01BBE00BF24
:1070F00096C801082DE9F04304788FB00546002CAE
:1071000059D17B4B0021142209A807AED3F8008087
:1071100010F00DFC07223046002110F008FC00237F
:107120001A46A70005A8059308EB07058380714957
:10713000B5F802E031F813C01CEA0E0F0AD00E3188
:107140000DF1380C595C02F1010E624402F81C1C6E
:107150005FFA8EF20133072BE9D100210B46664A14
:10716000B5F802E011F802C01CEA0E0F0AD0063290
:107170000DF1380C8A5C03F1010E634403F8242CF2
:107180005FFA8EF301310629E9D118F807308DE84E
:1071900041006A785949029209A81A0903F00F03BD
:1071A00000F09BFF2146564809AA013400F0AAFFCF
:1071B000202CA6D199E010F053FC1F28044600F3C0
:1071C000868028462021E4B210F0E7FB1F2C02D96C
:1071D000FFF78AFF89E0464B451C1B68002103EB43
:1071E00084042046042210F0A2FB0027454B09AE80
:1071F000304600210A2217F803905FFA87F810F052
:1072000096FB002315F8012B32B10A2B04D04A4516
:1072100002D0F2540133F5E74A455FD108F1FF335C
:10722000032B09D8DFE803F01005023F0DF123011D
:1072300034E00DF123011EE0304610F011FC2378FC
:10724000C0B243EA001006E0304610F009FC237893
:1072500000F00F001843207031E00133062B0AD0F4
:10726000244800F11B069E5D9642F6D103445A7DE8
:1072700063881343638011F8012F02B30023EFE703
:107280000133072B0AD01B4800F10E069E5D964283
:10729000F6D130F8132063881343638011F8012F6F
:1072A0006AB10023EFE7304610F0DAFB0F2804DC68
:1072B000304610F0D5FB607001E0002363700137A9
:1072C000052F93D1012409F045F874B980E70E49E0
:1072D00000221F230D4800F015FF06E02046002184
:1072E000042210F024FB0024EDE70FB0BDE8F0838A
:1072F000E81100205CA5010871A50108A4C80108D7
:10730000B3C801087DA5010890C8010871C801082B
:107310002DE9F041047807467CB9344D2146B5F893
:10732000BE21B5F8C0313248013400F0EBFE042C28
:1073300005F10405F2D1BDE8F0812E4910F000FB03
:10734000B0B92A4B4FF47A714FF4FA62A3F8BE1128
:10735000A3F8C021A3F8C211A3F8C421A3F8C61151
:10736000A3F8C821A3F8CA11A3F8CC21BDE8F08185
:10737000384610F075FB032805462ED838462021E4
:1073800010F00BFB044630B10134204610F068FBCE
:107390000127064600E007462046202110F0FDFAAE
:1073A00010B9BDE8F0419FE6013010F059FB012F04
:1073B000F7D140F2DC53A6F2EE229A42F1D8A0F2C5
:1073C000EE229A42EDD88642EBDA084B6E3503EB9B
:1073D0008503DE801881BDE8F08107480749002257
:1073E0000323BDE8F04100F08DBE00BFB0260020B1
:1073F000BFC80108D2C8010871C801087FD50108BB
:107400002DE9FF4104780546002C34D16E4808F080
:1074100089FC6E4D686900210CF090FE002840F058
:10742000CF8021466A4800F06DFE6869694600F029
:10743000EFFC0146674800F065FEA869694600F068
:10744000E7FC0146634800F05DFEE869694600F02C
:10745000DFFC01465F4800F055FE286A694600F0EF
:10746000D7FC013401465C4800F04CFE0C2C05F1C1
:107470001005CFD1A4E05949052210F0A5FA38B97A
:10748000524B002203441030C0285A61F8D197E0D3
:1074900028465349042210F097FA04462846002C47
:1074A0003FD1202110F079FA002800F08980451C96
:1074B000284610F080FA07464A4B53F824601EB95C
:1074C000494808F02FFC7BE028463146FAB210F01C
:1074D0007BFA01340028EFD13C4B0021C218103058
:1074E000C02851619E46F7D1404B03EBC402D2F84D
:1074F00004C09846BCF1000F04D131463C4800F06E
:1075000001FE53E0002718F834309F42F5DA3B01C2
:107510000EEB0305143563440FCB013785E80F00EC
:10752000F1E710F09DFA0B28064643DC284620219F
:1075300010F033FA054648B10135284600F0D2FB79
:10754000224B012403EB0613586100E00446284651
:10755000202110F022FA054640B10135284600F0FE
:10756000C1FB1A4B013403EB061398612846202116
:1075700010F013FA054640B10135284600F0B2FB81
:10758000124B013403EB0613D8612846202110F07A
:1075900004FA10B9FFF7A8FD12E0013000F0A2FBD9
:1075A0000A4B032C03EB06163062F3D11148FFF7A8
:1075B00027FF05E01048114901220C2300F0A2FD2D
:1075C00004B0BDE8F08100BFD8C80108B026002093
:1075D000F3C80108F9C80108D5D20108D2C80108CA
:1075E000FDC80108ACAC010802C901088CC701083C
:1075F00011C9010858C6010871C8010890C80108DE
:10760000F0B5047887B0064614BB514B19201968B1
:10761000062303FB041191F8CA5091F8CE2045438C
:1076200005F5617591F8C930009591F8CB50C831D6
:10763000684300F5617001900879029049794548E6
:1076400003912146013400F05DFD0C2CDDD17DE07D
:1076500010F006FA0B28044672DC3D4B701C1D68C6
:10766000202100238DF8173010F097F9064680B1DD
:107670000136304610F0F4F903289FBF062303FBC0
:10768000045383F8CE009DF817309CBF01338DF86A
:1076900017303046202110F080F9074680B10137BD
:1076A000384610F0DDF90D289FBF062303FB045375
:1076B00083F8C9009DF817309CBF01338DF817304F
:1076C00006266643A9193846CA310DF11702FFF79D
:1076D00067FC202110F061F9074670B10137384688
:1076E00010F0BEF914289FBF9DF8173076190133AA
:1076F00086F8CC0098BF8DF817303846202110F05E
:107700004CF978B1013010F0ABF90D289FBF06237A
:1077100003FB045383F8CD009DF817309CBF013361
:107720008DF817309DF81730062B0FD0062202FB7C
:1077300004500021C93010F0FAF8FFF7D5FC05E03D
:107740000548064900220B2300F0DCFC07B0F0BD21
:107750005C1000201DC9010871C8010890C801080B
:10776000F0B5027887B08AB94A4C04F1200694F843
:10777000EA210023484950B2595681426DD00C335A
:10778000302BF7D10834B442F1D180E000220492CA
:107790000592451C10F064F9C4B260B206F098FA84
:1077A000074618B18DF81040012400E00446284631
:1077B000202110F0F2F8054638B10135284610F0C6
:1077C0004FF90134ADF81200E4B20026284620211A
:1077D00010F0E3F8B0B3451C284610F041F9002240
:1077E0002E495FFA82FE51F82230834204D00132E2
:1077F000082AF5D1002300E0734651F82320824285
:1078000020D1022E0FD0032E12D05A1E012ED2B23A
:1078100004D0042A13D88DF814300EE0042A0ED8B0
:107820008DF8153009E0052B09D88DF8173004E0E4
:107830009A1E052A03D88DF816300134E4B20136B9
:10784000042EC3D1052C03D807B0BDE8F0404BE4AB
:1078500004AB03CB3860796019E094F8EF010F4B6B
:1078600094F8EE5153F82000B4F8EC21009094F80D
:10787000F10153F82000019094F8F00153F8200032
:1078800053F825300290064800F03CFC7AE707B038
:10789000F0BD00BFB026002010260020A0C10108C6
:1078A0003DC90108F7B5047806464CB9204601A940
:1078B0000BF0AAFD0134FFF7F5FF0E2CF6D14EE0D8
:1078C00010F0CEF8C5B20D2D45D8701C202110F057
:1078D00064F8034650B15B780130682B07D0732BF6
:1078E00001D1012704E0FFF7FFFB38E000E00027AB
:1078F000202110F052F81B4C05F1D006C0B1013028
:1079000010F0AEF840F2ED2380B2984205DD40F66B
:10791000CA039842A8BF184601E040F2EE20A0F248
:10792000EE20192290FBF2F004EB46039F70D87012
:1079300004EB4604A378E278012B4FF0190303FB14
:1079400002F329460CBF7322682203F2EE23064895
:1079500000F0D8FB03E005480E2100F0D3FB03B094
:10796000F0BD00BFB02600205CC901086EC9010847
:1079700010B50446204606F070FB18B90A2006F040
:10798000CAFAF7E710BD002207490C2303FB0213D4
:107990005968814204D10022C2621A725A6070474B
:1079A0000132042AF0D17047102600202DE9F04F53
:1079B000064687B088469DF8407011461A469DF8E5
:1079C000443000250C206843594C00EB040E00574E
:1079D000A146B04205D19EF808A0BAF1000F04D02C
:1079E000A2E00135042DEDD19EE0022E00F08C8046
:1079F00005DC002E40F0988000934E4886E0142E5F
:107A00000AD01E2E40F09080504601F041FA3946CF
:107A1000044606F01FFB7DE0474F484CBB6903223C
:107A200043F00403BB614FF4805B204605A98DF849
:107A300016200392ADF814B08DF8176005F04CFFD6
:107A4000C4F814B0C82006F066FAC4F810B0BB69D8
:107A5000039A43F00403BB614FF4C053204605A9C9
:107A6000ADF814301C23364C8DF816208DF81730E5
:107A700005F032FF334A4FF4802353614FF0010B7E
:107A8000636304F13400082384F8393084F83AB091
:107A90000BF06CFA2C4B2D4AC3F800A0FB6905A82B
:107AA00043F40003FB612A4BDA6002238DF81530A2
:107AB0008DF814608DF816A08DF817B00BF038FA19
:107AC0002A238DF814309DF817308DF815B08DF8F5
:107AD00016A01BB105A80BF02BFA04E01D4B4FF4C8
:107AE0008062C3F884201C4B1C4A1D49136002228B
:107AF0001A721C4B1C4A13601C4A1B681160984781
:107B00001B4B63601B4C06E01B4800933B4604F094
:107B1000B1FB044644B10C2303FB059526712046B6
:107B200085F808806C6000E0002007B0BDE8F08FA9
:107B300010260020003801400010024000080140DB
:107B4000E811002000040140D80042420005FA0577
:107B500000ED00E000E100E0102500200C250020F1
:107B600020000020C8000020BC1F0020B81F0020FB
:107B700084A50108EC11002000480040F0B5012464
:107B8000B0FBF4F58D4201D34C43F9E70026D4B1A4
:107B9000B0FBF4F504FB1500B4FBF1F41EB9002DA5
:107BA00001DC002CF3D1092D03F1010EEFB204DD4D
:107BB000002A14BF3725572500E030253D441D70AD
:107BC00001367346E3E71C70F0BDF0B50124B0FB4D
:107BD000F4F58D4201D34C43F9E70026D4B1B0FB54
:107BE000F4F504FB1500B4FBF1F41EB9002D01DC23
:107BF000002CF3D1092D03F1010EEFB204DD002AB0
:107C000014BF3725572500E030253D441D7001364F
:107C10007346E3E71C70F0BD03685A1C02601970DC
:107C200070472DE9F843089E002B07468846144606
:107C3000334614BF4FF030094FF0200913F8012BE1
:107C40000AB9254603E0002CFBDD013CF6E7002DD8
:107C500004DD38464946C047013DF8E7354624EA89
:107C6000E474A01B284415F8011B11B13846C04725
:107C7000F7E7BDE8F883024B186806F0FAB900BFD1
:107C8000B00E0020F8B507460C464868002115469E
:107C90001E460CF053FA58B128460CF067F810490C
:107CA0000CF0B8F801464FF07E500CF067F96060B8
:107CB000616830460BF0A6FF014630460CF05EF9D5
:107CC00025680646294638460BF09AFF014630469D
:107CD0000CF0A0F8014628460BF094FF2060F8BD98
:107CE000DB0FC9402DE9F04102780346202A00F15C
:107CF0000100F9D0092AF7D02D2A02D10346414DBF
:107D000004E02B2A08BF03464FF07E551C46002690
:107D1000234614F8012BA2F13007F9B209290DD836
:107D2000394930460CF076F8064638460CF01EF815
:107D3000014630460BF066FF0646E9E72E2A17D1CA
:107D4000314F234614F8010B3038C2B2092A0FD83C
:107D50000CF00CF839460CF011F9014630460BF0E6
:107D600051FF2949064638460CF054F80746E8E723
:107D70001A7802F0DF02452A39D15A782D2A02D129
:107D80000233012704E02B2A14BF013302330027FA
:107D9000013B002413F8012F303AD1B2092903D84E
:107DA0000A2101FB0424F5E7B4F59A7F28BF4FF4BC
:107DB0009A74A0464FF07E53B8F1070F07D91846C2
:107DC00012490CF027F8A8F108080346F4E704F07C
:107DD000070434B118460C490CF01CF8013C03466A
:107DE000F7E719462FB130460CF0C8F804E04FF021
:107DF0007E5130460CF00EF8014628460CF00AF889
:107E0000BDE8F081000080BF0000204120BCBE4CD6
:107E100030B5054687B00C4603A800210C220FF0B0
:107E200086FD284600210CF0B1F920B128462849EA
:107E30000BF0E8FE03E0284625490BF0E1FE25495A
:107E40000BF0E8FF0CF0ACF9054680EAE0706946FB
:107E5000A0EBE5700BF0D8FA002DACBF20232D234A
:107E600068468DF80C300FF0A6FD012807D13023AD
:107E70008DF80D308DF80E308DF80F300CE00228A3
:107E800005D130238DF80D308DF80E3004E0032835
:107E900004BF30238DF80D30694603A80FF06EFD46
:107EA00003A80FF088FD0338C5B22A4603A920466F
:107EB0000FF0ACFD00236355204607490FF05EFD2F
:107EC00003AB204659190FF059FD204607B030BDCD
:107ED0006F12033A00007A4485C9010870B506465E
:107EE000B6FBF2F40846154614B12046FFF7F6FF3C
:107EF00005FB1464024B1B5D00F8013B70BD00BF25
:107F000087C901082DE9F04F81468A4616461C466E
:107F100089B000253178002900F0DB80252902D0C6
:107F20000136484674E072784FF00008302A0CBFE2
:107F3000B278B71CA2F1300312BF4FF0000BF71C50
:107F40004FF0010B092B19D8A2F13003D9B209293E
:107F500005D80A2202FB083817F8012BF4E7A2F132
:107F60006103052B02D8A2F1570305E0A2F14103FA
:107F7000052B03D8A2F137030A2BEADD6C2A30D196
:107F80003A787E1C642A00F083800BD8252A3DD0E5
:107F900003D8002A00F09D80BCE7582A0CD0632A41
:107FA00019D0B7E7732A22D002D86E2A37D0B1E7AA
:107FB000752A5CD0782AADD1271D2068A2F158041B
:107FC00062424FF01001624155E02CD9582A32D05C
:107FD000632A2AD13E4648462178271DD0470135DD
:107FE0000FE0642A63D00ED9732A14D13E46236869
:107FF00048460093514642460023FFF712FE271DD4
:1080000005443C4686E7252ADFD13E4648462521E1
:10801000D04701357EE70AD86E2A06D13E4623684E
:1080200004341D6076E7002A53D03E4672E7752A75
:1080300026D0782AF9D1A2F1580304F1040C5A424F
:108040002068CDF80CC04FF010015A4105ABFFF786
:1080500095FDDDF80CC03E46644605AB00934846EE
:10806000514642465B46FFF7DCFD054452E7206877
:10807000271D0A21002205ABFFF7A7FD3C46ECE7D0
:1080800004F1040CCDF80CC020680A210022DDE7C1
:108090002068271D002808DA2D238DF8143040426F
:1080A0000DF115030A210022E6E705ABFAE7206887
:1080B00004F1040C00280ADA2D238DF81430404214
:1080C0000DF11503CDF80CC00A210022BFE705AB66
:1080D000F8E7284609B0BDE8F08F0EB40FB505AB40
:1080E00053F8042B0190064901A80393FFF70AFFF8
:1080F000019B00221A7004B05DF804EB03B07047D6
:10810000197C00080FB413B50B4904AB08680B4980
:1081100053F8042B09680193FFF7F4FE0446084B5B
:10812000186805F09AFF0028F9D0204602B0BDE893
:10813000104004B0704700BF7C010020780100208F
:10814000B00E002080EAE073A3EBE0738B4206DB05
:10815000002801DD401A704702D008447047002013
:10816000704770B504460CF01BF82030402857D8F3
:1081700020462C490CF00AF828B120462A490BF079
:108180003FFD0446F4E7204628490BF0E1FF28B103
:10819000204625490BF036FD0446F4E720462449E5
:1081A0000BF0F4FF30B1224920460BF029FD0146C7
:1081B0001F480AE020461F490BF0CAFF40B11C4986
:1081C00020460BF01FFD01461A480BF019FD04462E
:1081D000214620460BF01EFE0546204629460BF0A0
:1081E00019FE1549064628460BF014FE13490BF0FC
:1081F00007FD014628460BF00DFE11490BF002FD6C
:10820000014628460BF006FE0E490BF0F9FC01462C
:1082100030460BF0FFFD014620460BF0F3FC70BD2D
:10822000002070BDDB0F4940DB0FC940DB0F49C0A8
:10823000DB0FC93FDB0FC9BF9A7C2E36FAAF4F392F
:108240003587083CA4AA2A3E08B503490BF0DAFC9E
:10825000BDE8084085E700BFDB0FC93F2DE9F04FBF
:10826000056885B0814628460C46FFF7EDFF80463D
:108270002846FFF776FFD9F8045006462846FFF750
:10828000E3FF07462846FFF76CFFD9F8089005463C
:108290004846FFF7D9FF82464846FFF762FF41464E
:1082A000814650460BF0B6FD4146834648460BF0EA
:1082B000B1FD5146019030460BF0ACFD49460290AD
:1082C00030460BF0A7FD3946039050460BF0A2FD57
:1082D0004946206007F100400BF09CFD2946606094
:1082E000A56002980BF096FD014601980BF08AFC00
:1082F0002946E06003980BF08DFD014658460BF0CF
:108300007FFC3946206106F100400BF083FD2946D1
:10831000606158460BF07EFD014603980BF070FC3F
:108320002946A06101980BF075FD014602980BF0FB
:1083300069FC4146E06138460BF06CFD206205B0F7
:10834000BDE8F08F2DE9F04107688AB0466885687E
:108350000446084601A9FFF781FF019938460BF052
:1083600059FD0499804630460BF054FD01464046C5
:108370000BF048FC0799804628460BF04BFD014660
:1083800040460BF03FFC0299206038460BF042FD5E
:108390000599804630460BF03DFD014640460BF006
:1083A00031FC0899804628460BF034FD01464046D2
:1083B0000BF028FC0399606038460BF02BFD069902
:1083C000074630460BF026FD014638460BF01AFCF6
:1083D0000999064628460BF01DFD014630460BF074
:1083E00011FCA0600AB0BDE8F081074B10B51A88F7
:1083F0001C4622EA00009042188002D0012005F0BD
:10840000E1FD208810BD00BFE4110020064B10B52F
:108410001A881C4610439042188002D0012005F0B3
:10842000D1FD208810BD00BFE4110020024A9368EE
:1084300023EA000090607047B026002008B5104B7A
:108440001A780023D9B2914207D20E49002051F880
:108450002310013309680880F4E7322005F05BFD42
:10846000094B1B685A0309D5084B9B685B0305D46D
:10847000BDE8084040F2DC5005F04DBD08BD00BF2E
:10848000002000200420002050260020B0260020DC
:108490004B4A69232DE9F34113704FF4FA6353807B
:1084A000BE231371EF2382F8CD37002319461646F9
:1084B00082F8CE37F25C0133B3F5FA6F81EA02013C
:1084C000F8D13F4B3F4A83F8CE173F4B04275A6001
:1084D00002F188325A600020013F17F0FF075ED09A
:1084E000394B3422394CDA6004F17848A8F5FC386D
:1084F000C8F3090353B100234FF4005056F8088025
:10850000019305F0C5F80428E6D11CE04FF43020B3
:1085100005F0BEF80428DFD12B4D4FF430202B6935
:1085200043F002032B616C612B6943F040032B6124
:1085300005F0AEF841F6FD732A69042803EA020348
:108540002B61D8D0C8E7204D4FF400502B6943F081
:1085500001032B611FFA88F3238005F099F80428A2
:1085600013D1A31C0193019B4FEA1848A3F8008084
:108570004FF4005005F08CF841F6FE732A69042888
:1085800003EA02032B6106D0A6E741F6FE732A69CF
:1085900013402B61A0E70E4B04349C42A4D10A4A3D
:1085A0000428136943F08003136102D109F0A4F990
:1085B00010B90A2005F01EFD02B0BDE8F08100BF31
:1085C000B0260020230167450020024000F8010882
:1085D000D0FF01082DE9F04109F08EF910B90A2009
:1085E00005F008FDBB4CBC494FF4FA6220460FF081
:1085F00093F994F8A4374FF4CC71022B84BF002375
:1086000084F8A43794F8A427B44D01FB02F3E018D2
:1086100000F537702344286093F8300301FB0242D1
:10862000022803F54A7384BF0020187292F8303391
:10863000AB4A13700C2202FB0343AA4A03F2A6734F
:10864000136046F20902A3681A401AB9A14A43F41A
:1086500000539360A368DF0703D54FF40050FFF782
:10866000E5FEA3685E0409D50820FFF7DFFE4FF49E
:108670000050FFF7DBFE0120FFF7D8FEA3681807C4
:1086800006D54FF40050FFF7D1FE0120FFF7CEFED4
:10869000A368990413D54FF40040FFF7C7FE8D4B34
:1086A00093F88631012B03D14FF40060FFF7BEFE33
:1086B0004FF48030FFF7BAFE4020FFF7B7FEA36803
:1086C0005A0603D54FF48030FFF7B0FE022005F0C4
:1086D000FFFA854E40B1438833B133689B0303D51D
:1086E0004FF40030FFF7A2FE94F8D421794B2AB161
:1086F00093F8D82112B1002283F8D821336803F40B
:108700001073B3F5107F03D14FF40070FFF78EFEA6
:108710004FF0000C6746754E754B1E6004EB0C0362
:10872000B3F8ECE14FEA5E0101F077314FEA9E03C6
:1087300003F03333C1EB0E00C11A4FEADE0303F03E
:108740001133CB1A03EB231303F00F32FF2392FBF9
:10875000F3F31EF00108C3EB032318BF0137A2EBAC
:10876000030318BFFFB2012B0ADD022B40F0AE80DD
:10877000B8F1000F00F0AA801EF0BC0F00F0A68038
:108780000CF1080CBCF1200FC8D1013F012F00F201
:108790009D8009F08DF83022002156480FF0C7F86F
:1087A000554F564BD5F800801F60554B002108F1FE
:1087B0007900C3F8008005F04FFB524B80F00100B8
:1087C0001870514B07F126021A60504B07F1C8028E
:1087D0001A6098F8000006F075F828684C4B00F510
:1087E000C5721A6003F0D8F84A4B07F18C021A6080
:1087F000494B00221A809A71484B2D6807F12C02D0
:108800001A60474B05F219121A60464B05F289129D
:108810001A60454B07F108021A60444BDFF84881A3
:108820001F60434B07F194021A6007F19E03C8F8DA
:108830000030404BB4F866011E600BF093FAC8F8A4
:108840000800B4F868010BF08DFA95F85C3008F177
:10885000040288F8043095F87830C8F80C0088F8DD
:10886000053094F8D731286E88F81030324BC8F8AC
:1088700014501A60314B05F164021A6030490BF054
:10888000C9FA01464FF07C500BF078FBB5F8164161
:108890002C4B186020460BF069FA01462A480BF071
:1088A0006DFB2A490BF0B6FA294A2A4B15602A4A71
:1088B000186005F168031360284A05F21115156068
:1088C000274A1760274A1360BDE8F0810AF094FA3E
:1088D0005FE700BFB026002000F801085C10002010
:1088E000E01F002084100020502600203A2800209D
:1088F000742F0020F40E0020F4270020280F002001
:108900002C0F00200800002090070020B006002057
:10891000380F0020E00E0020FC240020E407002097
:10892000CC1C0020B4090020D41E0020D81E00203A
:10893000C80800208C0900205C1F00209C1F00201C
:10894000DB0F4940981F0020000061444C3D0F445C
:108950005C070020C408002050070020B408002055
:10896000BC080020380700202412002008B5FFF7BB
:108970008FFDFFF72FFEBDE80840012005F022BB68
:10898000426A806A131A58425841704741717047D1
:1089900043799B070AD5436A8269D154436A0169C6
:1089A0000133B3FBF1F201FB1233436270474379A9
:1089B00013F001031FBFC36803F1FF32C369006AEC
:1089C0001DBF181A1040C0B218467047437910B541
:1089D00013F0010304460DD0FFF7E9FF58B1236AF5
:1089E0006269E168D05C0133B3FBF1F201FB123341
:1089F000236210BD184610BD90F83B3210B57BB90C
:108A000090F83A3290F83942A34209D2B0F84012B5
:108A100001229A400A430133A0F84022DBB2F3E777
:108A200010BD8379DB0748BFB1FA81F1D0F834314A
:108A300048BF49095A681B8909B1136170475361DE
:108A4000704710F80A3C0133DBB20A2B84BF10F8E0
:108A5000131C054A00F80A3C82BF002322F811309B
:108A600000F80A3C704700BF5C2F0020354A70B503
:108A7000136C90681944344B1B78D94040F68C2312
:108A8000081A98429160D060516013463BD9127821
:108A900093F9451010468A420BD1111F082908D8B6
:108AA00093F84610182901D8013103E083F84420D7
:108AB00002E0002183F8461093F944402149A24284
:108AC00019D191F84740B4B10C310024944206DA30
:108AD00051F8046F1D4D25F814600134F6E70C2899
:108AE00005D01A49002421F810400130F7E7184852
:108AF00001780131017083F84520002201211A70AC
:108B000083F8471070BD92F84710C9B140F2DA51AE
:108B1000A0F2EF248C4208D811780B2905D80B1D40
:108B20000131117042F8230070BD002283F8472004
:108B3000084B03F13002002143F8041F9342FAD19D
:108B400070BD00BFA00100209F0100205C2F00200D
:108B5000F9060020AC010020024A136C01331944CD
:108B600011647047A0010020024B53F820301B68AD
:108B70001980704704200020074BA1F57A7153F843
:108B800020301A681B8959434FF47A7391FBF3F133
:108B900089B21180704700BF042000201FB5012357
:108BA000ADF80830ADF80410002301A9ADF80A3083
:108BB000ADF80C30ADF8062004F07BFD05B05DF893
:108BC00004FB38B5A0F513746379A579DB0745D5A7
:108BD00094F8383205F00105F3B1226B1068838DEB
:108BE000C3F34E03838494F83C3223B1B4F8423289
:108BF0000133A4F84232917A6A00FFF7CFFF0123D4
:108C000084F83B32002384F8393284F83A3284F80D
:108C10003832A4F8403238BD94F83B322046012B5C
:108C200004BF94F8393284F83A32FFF7E5FE94F83D
:108C30003B22236B3AB9012284F83B221868997AC7
:108C400005FA02F207E0002284F83B2295421868F8
:108C5000997A08BF0222BDE838409FE738BD10B5B9
:108C6000A0F5127494F83C22BAB9A36A616A9942D9
:108C700028D0591CA069A162C35C2069DBB25B00EB
:108C800043F400738142A4F83E324FF00A0384F8A3
:108C90003D3228BFA262012312E094F93D327BB13C
:108CA000B4F83E1220464B08A4F83E3201F0010110
:108CB000FFF7B7FE94F83D32013B84F83D3201E006
:108CC00084F83C3294F83832002B4ED194F8393283
:108CD0000133DBB2092B84F8393203D12046BDE8D9
:108CE000104089E60A2B40D194F83B322BB9B4F8F6
:108CF000403243F00103A4F840326379D9071CD510
:108D0000B4F84002820501D4C30705D4B4F8443254
:108D10000133A4F8443210E0E36AC0F347000BB11A
:108D200098470AE0E3696269D054E369E168013376
:108D3000B3FBF1F201FB1233E361012284F8382224
:108D400094F83B220023012A84F839320DD1A2790C
:108D500084F83B32236B12F0010F1868997A0CBF2C
:108D600002220022BDE8104018E710BDF0B5046DE6
:108D70008279A389467923F4005312F0020F4FEA57
:108D800003434FEA13430CBF00214FF4005112F08C
:108D9000040FA38114BF4FF4806E4FF0000E16F045
:108DA000010F8768054614BF04200020B307238AFB
:108DB00048BF40F008029BB223F4405343EA01034A
:108DC0002382A18948BF90B289B221F4B05121F029
:108DD0000C014EEA010140EA0102A281A38A87B098
:108DE00023F440731B041B0CA38201A804F006FCAF
:108DF000039B049E254A944218BF1E46A38919224C
:108E000072431BB2002BB4BF7E00BE00B2FBF6F66D
:108E10006427B6FBF7F00001010907FB1163A28983
:108E200012B2002AB7BFD9001A013231B1FBF7F2F2
:108E3000A7BF3232B2FBF7F302F007021043A8BF1C
:108E400003F00F03AA79A8BF184380B212F0010FF4
:108E500020812B6D06D00D498B4202BF0420A1F565
:108E60003051086112F0080F9A8A0BBF22F00802F5
:108E700092B2120442F0080208BF120C9A829A8938
:108E800092B242F400529A8107B0F0BD003801401E
:108E90002DE9F04F4E4C4FF4147585B08046914645
:108EA0001E4605FB0045274620B94A4B2B63103B65
:108EB000C5F834314FF4147303FB08F3464AFC1829
:108EC000FA5003226271224603F59C733B44E1622F
:108ED000A36100214FF48070D4F8343134324FF064
:108EE000010B62612162E161A162616284F83C125E
:108EF00084F83912A4F84212A4F84412C4F8089075
:108F0000A671E060206184F838B284F8468258681F
:108F10001B890222ADF80C3003A910238DF80E3006
:108F20008DF80F20019206F0F7F9236B019A597B17
:108F300058681B898DF80E1003A9ADF80C308DF818
:108F40000F2006F0E9F928465946FFF76AFD32205E
:108F500004F0E1FF214BD4F834A11B681A46B2FBA0
:108F6000F9F1B1F5803F03D3012AF8D95208F6E7A9
:108F70001B4A5046B3FBF2F289B2D2B203F0AEF80C
:108F80004FF4147000FB08F0164B07EB000800F5D7
:108F900012703C180022C8F848325046214603F0AF
:108FA000E5F8D8F8307016F0010F0CBF022200224D
:108FB0003868B97AFFF7F2FD0B4B3846C8F84C32E7
:108FC000211D002203F0D2F8284605B0BDE8F08F3D
:108FD0003C12002084C201085CAA010804010020A0
:108FE00040420F005F8C0008C38B000803460A460E
:108FF00090F84602D96A9B794AE71FB50123ADF87C
:1090000008300023ADF80C30ADF80A30084BADF84D
:1090100004101B7801A9012B08BF0323ADF806201B
:1090200008BFADF80C3004F044FB05B05DF804FB5C
:109030009C01002038B510F80E2C044650F8043C72
:1090400052B9012200F80E2C20F80C1C997A1868ED
:109050000222BDE83840D0E730F80C2C20F80A1C7A
:10906000891A89B220F8081C074A10F80F0C00254D
:1090700022F8101004F80E5C1868997A2A46FFF757
:10908000BCFF04F8065C38BD5C2F0020044B53F88D
:1090900020301BB107289CBF1B681980704700BF98
:1090A000C80200202DE9F7438E460546DFF8A0925E
:1090B000114699F850420068164698467246631C5D
:1090C00089F8503202F0B6FF2B8901A9ADF80430BF
:1090D00018238DF80630686802238DF8073006F0F3
:1090E0001BF9AB7A09F51577240127442A6849460C
:1090F0000C2B00F2F680DFE813F00D00F400F40012
:10910000F4005100F400F400F4008A00F400F400CC
:10911000F400C200138CDFF83CC223F001031B04EF
:109120001B0C1384138CB2F804E0108B624520F002
:1091300073004FEA00404FEA10409BB21FFA8EFEC8
:1091400040F0700014D00CF5006C624510D00CF5A6
:10915000406C62450CD00CF5806C624508D00CF573
:10916000806C624504D023F0020343F0030307E060
:1091700023F00E032EF4407E43F003034EF4807E72
:10918000A2F804E01083A2F834801384138B23F038
:1091900008031B041B0C43F0080336E0138CDFF8B4
:1091A000B4C123F010031B041B0C1384138CB2F8FE
:1091B00004E0108B624520F4E6404FEA00404FEA9D
:1091C00010409BB21FFA8EFE40F4E04008D00CF530
:1091D000006C624504D023F0200343F0300307E025
:1091E00023F0E0032EF4406E43F030034EF4806E23
:1091F000A2F804E01083A2F838801384138B23F4C0
:1092000000631B041B0C43F40063138369E0138C9D
:10921000DFF840C123F480731B041B0C1384138CF0
:10922000B2F804E0908B624520F073004FEA0040F2
:109230004FEA10409BB21FFA8EFE40F0700008D03B
:109240000CF5006C624504D023F4007343F44073C2
:1092500007E023F460632EF4405E43F440734EF461
:10926000805EA2F804E09083A2F83C801384938B84
:1092700023F008031B041B0C43F0080330E0138C9D
:10928000DFF8D0C023F480531B041B0C1384108C14
:10929000B2F804E0938B20F4005023F4E6431B045F
:1092A00000041B0C000C62451FFA8EFE43F4E043E1
:1092B00040F4405003D00CF5006C624503D12EF40D
:1092C000804E4EF4804EA2F804E09383A2F84080D2
:1092D0001084938B23F400631B041B0C43F4006382
:1092E00093832B7B43B1B2F844306FEA43436FEA78
:1092F00053439BB2A2F8443013889BB243F001035E
:109300001380AB7A0C2B19D8DFE803F00718181874
:109310000B1818180F18181813000B1902F1340045
:109320000AE00B1902F1380006E00B1902F13C00CB
:1093300002E00B1902F14000C3F8540238460C4415
:10934000A4F85C62C4F8582203B0BDE8F08300BF03
:109350003C120020002C0140084A13689B020BD5E8
:10936000074B002119704FF6FE7306490868034049
:109370000B604FF400135360704700BF00000240C1
:10938000A23000206C000240344B354A1B68126842
:1093900010B51A60334A1168596051689268996033
:1093A000DA60314A116819615168926859619A61AD
:1093B0002E4A1168D9615168926819625A622C4A22
:1093C00011881985518859859188D2889985DA85BF
:1093D000284A118819865188598692889A86264A81
:1093E0001188D986518892881987194621F83A2F11
:1093F000224A10780022824206DA214C34F81240C8
:10940000013221F8024FF6E71E4A1288A3F86420C1
:109410001D4A1288A3F866201C4A1188A3F86C1014
:1094200051889288A3F86E10A3F87020184A3B2147
:1094300012689A66174A126892FBF1F2B2F5967FAB
:10944000C8BF4FF0FF325A67134A1288A3F878203A
:10945000124A5289A3F85E2010BD00BFFC220020F2
:109460007C300020C4150020D0150020DC15002021
:109470000411002040100020EE10002000200020E9
:10948000601000205C1D0020A40E0020461000206B
:10949000F810002000000020801000204C10002058
:1094A00070B5472008F042FD174B1B681B0307D51A
:1094B000164B174A5B6810681B68C01A08F068FDF5
:1094C000144E154C154D307808F062FD236828685D
:1094D000C01A08F06CFD63686868C01A08F067FD80
:1094E0000F4B188808F054FD0E4B188808F050FDFB
:1094F0000D4B188808F04CFD337823742B68A3605B
:109500006B68E36070BD00BF80240020FC22002057
:109510007C3000202A110020E82200202C1100209D
:109520002811002026110020881000200A4A1388E4
:1095300001331380094A136801331360084A138802
:1095400001339BB2202B01BF00231380054A1388EF
:1095500008BF013313807047A02400208824002016
:109560008C2400208E24002038B53A4B05461B7809
:109570000C46083B012B6BD8452008F0D7FC284649
:1095800008F0D4FC0C2D23D004D80A2D0AD014D80E
:1095900035B138BD0E2D4BD02ED3FF2D50D038BD58
:1095A000206849E0207808F0C1FC62796378002ADD
:1095B00014BF80200020184300E0207808F0B6FC9B
:1095C000A07808F0B3FCE07808F0B0FC20793BE02C
:1095D000B4F9000008F0D2FCA07808F0A7FCE0780D
:1095E00008F0A4FCB4F9040008F0C8FCB4F90600C3
:1095F000BDE8384008F0C2BC637820788BB180F0B9
:10960000800008F093FCA468E0B208F08FFCC4F37B
:10961000072008F08BFCC4F3074008F087FC200EFD
:1096200012E008F083FC6068BDE8384008F0BFBC79
:10963000206808F0ADFC6068BDE8384008F0A8BCC0
:10964000054808F0F7FB0020BDE8384008F06EBC84
:1096500038BD00BFD8220020ACC901082DE9F04F69
:10966000BF4B8BB018880193002840F0A380BD4EFB
:1096700007F0A0FEFFF788FE34684920254608F071
:1096800055FCB94B04F11C08186808F081FC55F82A
:10969000040B08F07DFC284609F060FB04F1100083
:1096A00009F05CFB1027B14D01232A68BB4013422F
:1096B00003D0D8F8000008F07AFC0137132F08F126
:1096C0000408F0D1AA4F04F1280009F037FBB7F8DD
:1096D0004431B4F92E00B846C01A08F059FC2B6882
:1096E00013F4805F08D0A34BB4F864001B88181AE9
:1096F000C0F30D0008F04CFC2B68990403D5B4F8B6
:10970000660008F045FC2B685A0503D504F16C008F
:1097100009F014FB2B681B0502D5A06E08F047FC6E
:109720002B685F0402D5606F08F041FC2B681804B9
:1097300003D5B4F8780008F02BFC274604F130007C
:1097400009F0FCFA04F1360009F0F8FAB8F84431EF
:1097500037F93C0F4FF00108C01A08F019FC864B8E
:109760001B78984509DA37F9020FB4F93C3008F153
:109770000108C01A08F01BFCF1E72B68990505D514
:10978000B4F95E00A0F2DC5008F011FC32687B48AE
:109790007260B260121A9110794A4A43531C032234
:1097A00093FBF2F202EB42029A1A7C2303FB0203C0
:1097B000336068E2734B744A1B6811688B4206D0B1
:1097C0000AA941F8203D00201360FFF7CDFE684A4A
:1097D000019B92F8CA171B8892F8CB070B44013BF8
:1097E000B3FBF0F200FB12338B4280F017825D4F27
:1097F000012007F0DFFDFFF7C7FD50203E687D68C0
:1098000008F094FBBA683B6810681B687A680344E8
:109810001068A3EB400008F0CAFB6A68736802A8EE
:109820009B1A0293AA68B3689B1A0393EA68F368C9
:109830009B1A049309F092FA2A6933699B1A0293DE
:109840006A6973699B1A0393B369AA699B1A0493A3
:109850000023194602AA52F8212002F120003F28D5
:1098600042D802F108000F2806D80232032A04D990
:10987000002B08BF012300E0022301310329E9D1B5
:10988000012B02980ED0022B21D0039B00F0030085
:1098900003F003039B0043EA0010049B03F003035F
:1098A00018430CE000F00F0040F0400008F03EFBD1
:1098B0000498039B00F00F0040EA0310C0B208F0C8
:1098C00035FB06F11C0B05F11C0810246FE000F0BD
:1098D0003F0040F0800008F029FB9DF80C0008F0E4
:1098E00025FB9DF81000EAE702224FF0000802ABCA
:1098F00053F822304FEA880803F18001FF2910D97C
:1099000003F50041B1F5803F02D248F0010808E0BC
:1099100003F50003B3F1807F34BF48F0020848F03C
:10992000030812F1FF32E2D268F03F00C0B208F043
:10993000FDFA02AC0DF1140A08F00303022B2078A3
:1099400007D0032B22D0012B29D108F0EFFA607841
:1099500025E008F0EBFA607808F0E8FAA0781EE05D
:109960008C240020FC220020882400208024002059
:10997000B02600207C2400200020002008230020A6
:10998000DF7BEFBD942400209024002008F0CEFA65
:10999000607808F0CBFAA07808F0C8FAE0780434D0
:1099A00008F0C4FA54454FEAA808C5D189E7B84978
:1099B00001220B68A2401A428A4606D0DBF800005A
:1099C000D8F80030C01A08F0F2FA0134132C0BF169
:1099D000040B08F10408EAD106F1260005F126017E
:1099E000002331F9024F30F9022F121B02AC44F868
:1099F00023200133042BF4D103214FF000094FEA57
:109A000089035FFA83F902AB53F821206AB102F1AE
:109A100008000F2802D849F0010906E08032FF2A29
:109A200094BF49F0020949F0030911F1FF31E6D270
:109A30004846002408F07AFAA0460DF1080B09F018
:109A40000302022A16D0032A1DD0012A38D1B8F108
:109A5000000F05D1DBF8004090462401E4B22FE06E
:109A6000DBF800004FF0000800F00F00204308F082
:109A70005DFA25E0B8F1000F0CD0DBF80000C0F370
:109A80000310204316E0B8F1000F08D19BF8010045
:109A900008F04CFA9BF8000008F048FA10E0DBF8F8
:109AA0000000C0F30330204308F040FADBF8000068
:109AB000C0F3071008F03AFADBF800402401E4B2E2
:109AC0000BF1040B06AB9B454FEA9909B7D1B8F1EE
:109AD000010F02D1204608F029FADAF8003013F419
:109AE00080541FBFB6F86420B5F864100124521AE0
:109AF00018BF02929A040AD50AAA02EB8401B5F8AB
:109B00006600B6F866200134121A41F8202C580578
:109B100013D502AA02EB840C06F16A0E05F16A0065
:109B200000223EF9021F30F9028FC8EB01014CF808
:109B300022100132032AF4D10334190508D50AAAE8
:109B400002EB8400A96EB26E0134521A40F8202C48
:109B50005A0408D50AAA02EB8400696F726F0134B7
:109B6000521A40F8202C18040BD50AAB03EB8402E0
:109B7000B5F87810B6F8783001345B1A42F8203C1A
:109B800000E0FCB1012C03D1029808F010FA19E0B2
:109B9000631E002002AA52F823204000C0B20AB17E
:109BA00040F00100013BF5D508F0C0F94FF0000886
:109BB00002AB53F8280008B108F0F9F908F10108E0
:109BC000A045F5DB3020032107F034FC36200321CB
:109BD00007F030FC2F4B3C20197807F02BFCDAF80B
:109BE0000030990506D5B6F95E00B5F95E30C01AA9
:109BF00008F0DDF93A6828487B687A60121A9110FB
:109C0000264ABB604A43531C032293FBF2F202EB49
:109C100042029A1A7C2303FB02033B60204B1B6821
:109C20001A0630D51F4C204D22682B689A420BD162
:109C300062686B689A4207D1019B1B88102B11D177
:109C40001A4B1B885B060DD1482008F06FF920687D
:109C500008F0ADF9606808F0AAF923682B60636822
:109C60006B600EE0124A104B11782A7C914208D1A9
:109C7000104A99681068884203D15268DB689A429A
:109C800001D0FFF70DFC08F0C3F80BB0BDE8F08F72
:109C9000802400200020002008230020DF7BEFBD6F
:109CA000502600208C100020E82200208E24002066
:109CB0002A1100202C1100202DE9F84F0C9EC2EB38
:109CC000030B394C0B9B002914BF4FF0060A4FF0D1
:109CD000040AF61A636805460133904613D12368D7
:109CE00053455ED2314A032B98BF294652F82320B0
:109CF0002F4808F009F963680022013363602D4B97
:109D000005461A7013E0002511E02B4A127895429F
:109D100040DA0B9BE3B109FB06F2995C01228A4011
:109D2000264909680A4213D1636801336360D4F895
:109D300004900A9B1C4F9945E7DB2BD10A2008F0C1
:109D4000F5F83B6801333B604FF0FF337B6021E067
:109D5000184A117821B12C2008F0E8F8013501E00B
:109D60000121117009FB0BF3226808EB030752B9BC
:109D700058F8030008F05EF897F9041005444B1CEE
:109D8000D2D00F4802E03A440E48117908F0BCF8EE
:109D90000544C9E7206850452CBF00200120BDE8DC
:109DA000F88F0020BDE8F88F9824002074AA0108DD
:109DB000B7C90108501500200801002080240020A8
:109DC000C6C901084CDF01082DE9F04F89B00593A1
:109DD000A04B80461B880492980737D540F2E632A4
:109DE000129B9D48DC89B0F900301B1B03F2F31570
:109DF000954203D8002BB8BF5B4201E04FF4FA73E1
:109E0000B0F9022040F2E630121B02F2F314844251
:109E100003D8002AB8BF524201E04FF4FA729342CD
:109E2000B8BF13460522C3F5FA7393FBF2F30A2277
:109E3000643B534398F81C20D2105343642293FB95
:109E4000F2F3134423EAE373DBB200E06423C14678
:109E50000193CB1C03930024039B022C13F8016F86
:109E60007E4F03934FEA440A05D1B7F904301B36FD
:109E70005E4376114AE07A4B37F9142033F91430F7
:109E800003EB4202049B5B429A4203DB049B934236
:109E9000A8BF1346734A32F90A50059A5B1B32F980
:109EA000145003EB050B08F065FA88B16E4A58466A
:109EB000155D09F05BFF6D490AF060F80146284620
:109EC00009F084F8694909F0A5FF0AF069F98346A9
:109ED000604A1288D10714D437F90A501B366E43F2
:109EE00093074FEA261611D598F812509DF90420D1
:109EF00005FB0BF35343642293FBF2F306EB2316AB
:109F000004E098F8085005FB0BF52E11584B04257A
:109F100033F90A30574F93FBF5F5751B99F801603B
:109F2000E35D6E435E430293642396FBF3F698F879
:109F300051B0F611BBF1000F1BD0022C30460CD1F2
:109F400009F014FF5FEA5B0304D05B45A8BF5B46E2
:109F50001A4600E00122484905E009F007FF5A4689
:109F6000391D01EBC401FB69FDF78CFE0AF018F9FD
:109F70000646424B99F80B7019883E4B01FB05F2DF
:109F800003F1200E5EF82400D21207FB02073C4AC0
:109F9000B7F5001FA8BF4FF40017974203F12C003C
:109FA000B8BF174650F8242040F824504FF6FF70F1
:109FB0000909B0FBF1F1AA1A4A4303F1380103F190
:109FC00044054EF8247051F824E055F8240045F873
:109FD00024E098F85050921170444FEA840C7F139B
:109FE000104441F824208DB1CDF818C0079309F032
:109FF000BDFE079B2A4603F1500101EBC401DB695A
:10A00000FDF740FE0AF0CCF8DDF818C099F81530DD
:10A01000F2195843029B013443431846642390FBD2
:10A02000F3F0184B0012024423F80A2003F108024F
:10A030004CF80260032C03F1140203F120034CF8E6
:10A0400002704CF8030009F101097FF405AF09B073
:10A05000BDE8F08FE41100208C26002004110020C0
:10A060009C300020462600208CAA010800002041D8
:10A070004010002054150020681500201C100020FE
:10A080000000E0FFBC1500202DE9F04F8BB00793D6
:10A09000CA4B0592B3F90220002682EAE279A9EBC5
:10A0A000E279B3F90020804682EAE273A3EBE2731F
:10A0B0009945B8BF9946B4463446B9F5FA7F06913A
:10A0C000A8BF4FF4FA79029001960396BC4D2B88F5
:10A0D000990755D0B94B610033F91420B94B33F9C6
:10A0E000143003EB4202059B5B429A4203DB059B63
:10A0F0009342A8BF1346B44A8F5E079ADB1B32F91E
:10A1000014001F1808F036F990B1B04B384613F818
:10A1100004A009F02BFEAE4909F030FF014650467D
:10A1200008F054FFAA4909F075FE0AF039F807460D
:10A1300098F8083064227B4393FBF2F398F81C20D4
:10A140006FF0040101FB02FC634505DB02EB8202B8
:10A150009342A8BF13469C4642F210729D4B53F89F
:10A16000240038449042A8BF10469B4A9042B8BF92
:10A17000104643F8240098F8123058430313039311
:10A180002D8805F00303012B38D08C4B934933F90C
:10A190001430A6000193029B51F8247093F801E05B
:10A1A0008F4B33F9140080EAE073A3EBE073B3F54F
:10A1B000206F16DC019A50235A4392FBFEF30422CF
:10A1C00090FBF2F0181A0744B7F57A5F854BA8BFE9
:10A1D0004FF47A579F42ACBF41F8247041F82430C5
:10A1E00002E0002341F824308B597D2693FBF6F6DC
:10A1F000029BDB7A7343402693FBF6F6AA0712D53F
:10A20000019B09FB06F509FB03F70398C9F5FA72F0
:10A2100002FB0C7702FB00524FF4FA7197FBF1F34B
:10A2200092FBF1F505E0EB0755BF35466346019B10
:10A23000039D6B4A042732F91420DFF8ACB192FB7E
:10A24000F7F70BF19C02A25C4FEA440A57436FF008
:10A250004F0297FBF2F798F851201F449AB1384605
:10A26000CDF810C0089209F081FD0BF1040101EB5B
:10A27000C401089ADBF81C30FDF704FD09F090FFDB
:10A280000746DDF810C0564B4FEA840B3AF803003E
:10A29000554B02B203F1A0013AF901E02AF801009E
:10A2A000CEEB02024FF0040E92FBFEF203F1A4018A
:10A2B00003F1AC0E04925EF8240051F824201044FF
:10A2C000049A104451F824204EF82420049A41F8AE
:10A2D000242098F8502092B1CDF810C0099308922C
:10A2E00009F044FD099B089A03F1500101EBC401F8
:10A2F000DB69FDF7C7FC09F053FFDDF810C03A4BEE
:10A3000003F1B402125D03F168015043202290FB77
:10A31000F2F07A19121A2AF8012003F170024BF8B0
:10A32000027003F17C024BF80250404203F18802B4
:10A330004BF80200029A013202920CB90124C5E6E0
:10A340001E4A0420B2F90410069A9C6A92790F32D0
:10A3500052004A4322495511B1F9041085EAE572C9
:10A3600091FBF0F0A2EBE572322AA5EB000098F821
:10A370000D100BDC01FB00411C4A8A42A8BF0A46B3
:10A380001B498A42ACBF9A62996201E000229A623C
:10A3900098F8031001FB00F216499211097803297D
:10A3A0002BD9B8F84E10B1F5FA7F26D24842824236
:10A3B00022DB8A42A8BF0A461FE000BF041100202A
:10A3C000E41100209C300020462600208CAA0108C1
:10A3D00000002041E8150020F0D8FFFF7415002090
:10A3E0004010002080C1FFFF54150020FEFFFF0F2A
:10A3F000020000F0002000200246996A6FF0FF0082
:10A4000041F34F31B1F5807FA8BF4FF48071814295
:10A41000B8BF01469A6750180022A3F86C00C3F831
:10A420008410C3F890200BB0BDE8F08F2DE9F04FF9
:10A4300087B00393B94B81461D88029105F0020550
:10A44000ADB2019295B1B64BB3F90250B3F90030F9
:10A45000002DB8BF6D42002BB8BF5B429D42B8BF14
:10A460001D46B5F5007FA8BF4FF40075CB4600260A
:10A47000AB4BAC4933F91620AB4B4FEA460A33F9E4
:10A480001630520083EAE374A4EBE374B4F5206F52
:10A490004FEA860851F8260011DC042493FBF4F3FC
:10A4A000D31A0344B3F57A5FA048A8BF4FF47A5398
:10A4B0008342ACBF41F8263041F8260002E0002379
:10A4C00041F8263051F808709BF80B30FF119BF8CB
:10A4D00001405F43914B54431B88BF119B074FEAD8
:10A4E000A41456D0924B3AF903301A44019B5B42B4
:10A4F0009A4203DB019B9342A8BF13468D4A3AF967
:10A5000002209B1A039A32F916201A44049207F08B
:10A5100031FF049A98B1884B10469B5D049309F073
:10A5200025FC864909F02AFD049B0146184608F0DF
:10A530004DFD824909F06EFC09F032FE024642F2FE
:10A5400010707F4958F8013013448342A8BF034676
:10A550007C488342B8BF034648F8013099F8081098
:10A5600099F81C004A4300EB8000D21141428A4214
:10A5700003DB8242A8BF0246114699F81220641AF2
:10A5800053431B13FF1A6F436C4303EB672701EB25
:10A590006424654B04223AF9033093FBF2F16A4BD1
:10A5A00003F19C02925D4A43A4EBA21499F8512056
:10A5B0007AB120460593049209F0D8FB059B049AD2
:10A5C000191D01EBC601DB69FDF75CFB09F0E8FD35
:10A5D0000446554B3AF803005B4B02B203F1B80155
:10A5E0003AF901E02AF80100CEEB02024FF0040E26
:10A5F00092FBFEF203F1BC0103F1C40E58F801C056
:10A6000058F80E0048F801206044104499F8502092
:10A6100048F80EC072B10593049209F0A7FB059BA0
:10A62000049A03F1500101EBC601DB69FDF72AFB37
:10A6300009F0B6FD444B0BF1010B03F1B402925D3E
:10A6400003F168015043E2194011121A2AF801205F
:10A6500003F1700248F8024003F17C0248F80270EE
:10A66000404203F1880248F802000EB90126FFE6D5
:10A670002B4A0420B2F90410029A9C6A92790F3294
:10A6800052004A4328495211B1F90410002A91FBA3
:10A69000F0F0A2EB0000B8BF5242322A99F80D1038
:10A6A0000BDC01FB0041294A8A42A8BF0A4628491F
:10A6B0008A42ACBF9A62996201E000229A6299F8DC
:10A6C000031001FB00F223499211097803290CD9E8
:10A6D000B9F84E10B1F5FA7F07D24842824203DB47
:10A6E0008A42A8BF0A4600E00246996A6FF0FF005E
:10A6F00041F34F31B1F5807FA8BF4FF480718142A3
:10A70000B8BF01469A6750180022A3F86C00C3F83E
:10A710008410C3F8902007B0BDE8F08FE41100204A
:10A7200004110020741500204010002080C1FFFF9C
:10A730009C300020462600208CAA01080000204101
:10A74000E8150020F0D8FFFF54150020FEFFFF0F92
:10A75000020000F0002000202DE9F04F054690F89F
:10A7600050008DB008910592099318B13228A8BF06
:10A77000322000E0012009F0F9FA0146AA4809F068
:10A78000FDFBAA4B04461888002808BF012009F0E9
:10A79000EDFAA749069009F03DFB0190019920468A
:10A7A00009F030FA0146019809F0E8FBA14B079047
:10A7B0001B889A0724D5A049B1F90030B1F90200ED
:10A7C00083EAE37280EAE071A2EBE372A1EBE0714D
:10A7D00091420C46B8BF1446B4F5E17F12DA9142BB
:10A7E00003DD0028D8BF404203E0002BCCBF184651
:10A7F000584209F0BBFA914909F0C0FB064603E054
:10A80000002601E04FF07E564FF00009CA4603953E
:10A810000024630004938A4B33F9140009F0A6FA6C
:10A82000884909F0F7FA09F0BBFC09F09FFA86495C
:10A8300009F0F0FA804B029033F9140009F096FA0F
:10A840007C4B07461B889B077ED0014609F0DAF94E
:10A850007E4B804633F9140009F088FA01464046E1
:10A8600009F0D0F909F09CFC059B5B42984203DBA0
:10A87000059B8342A8BF0346754A0499885E099ADE
:10A880001B1A32F91400184409F070FA804607F0D8
:10A8900071FD70B16F4B40466F4914F8039009F099
:10A8A0006DFB0146484608F091FB6B4909F0B2FA8E
:10A8B0008046287F09F056FA684909F0ABFA8246CB
:10A8C000287A09F04FFA0146404609F0A3FA644994
:10A8D00009F0A0FA09F064FC81460AF1004009F091
:10A8E0005FFC814505DB504609F05AFC4845A8BF8E
:10A8F000484609F03BFADFF88C91019982464046C0
:10A9000009F088FA59F8241009F07CF955494FEA02
:10A91000840B804609F01CFC38B94046524909F0C6
:10A9200035FC20B1DFF8408101E0DFF8388149F8DB
:10A930000B80A87C09F016FA0146404609F06AFA35
:10A940004A4909F067FA81463A4BB3F800B01BF068
:10A95000010F40F099803A4B049ADFF82081D35ED2
:10A96000002BB8BF5B42B3F5206F4FEA84030A9314
:10A9700003DD002348F824302AE03D49384609F039
:10A9800049FA039B0B90587809F0ECF90B9A0146B1
:10A99000104609F0F3FA029909F032F9019909F029
:10A9A00039FA58F8241009F02DF93249804609F097
:10A9B000CFFB38B94046304909F0E8FB20B1DFF859
:10A9C000B88001E0DFF8AC802C4A0A9B42F8038093
:10A9D000039BD87A09F0C6F9284B53F8241009F0E4
:10A9E00019FA274909F016FA1BF0020F80464DD0DC
:10A9F0003846514609F004F90146304609F00AFA92
:10AA00000146504609F0FEF849460746404609F01F
:10AA1000F7F80146304609F0FDF90146484609F0CD
:10AA2000F1F8804632E000BF83F9223E1C1000207E
:10AA3000BD378635E4110020041100200000E143F9
:10AA4000401000200000A03ECDCC4C409C300020A7
:10AA5000462600208CAA0108000020410000A040EA
:10AA60006F12033C0000F0C10000F0410AD7A33D83
:10AA70000000A043000040C300004043281600200F
:10AA80000AD7233C20160020C8465746DFF83CB2C0
:10AA90000BF19C03185D09F069F90146029809F071
:10AAA000B9F9894909F0B6F90146384609F0A8F81C
:10AAB00095F85120034642B10BF10401DBF81C303C
:10AAC00001EBC401FDF7DEF80346804F029807F161
:10AAD000E00B5BF824100A9309F092F8019909F051
:10AAE0004DFA029B07F1E8024BF8243052F824B0EB
:10AAF0000292594609F084F80146079809F08AF94C
:10AB00000146584609F07EF8029A834642F824002E
:10AB100007F1B402105D09F029F90146584609F021
:10AB200079F96B4909F076F983460A9B4146184644
:10AB300009F068F8594609F063F80DF005F9049B2F
:10AB400007F16802D0520A9B07F170021846029280
:10AB500009F026FB029A07F17C0342F824004046E4
:10AB6000029309F01DFB029B07F1880843F82400BB
:10AB70000BF1004009F014FB039B48F8240001335B
:10AB800003930CB9012444E6089A524B9479B3F923
:10AB90000430640028345C434F4B6411B3F9040063
:10ABA00009F0E4F84FF07A5109F034F90DF0CCF8DF
:10ABB000201A09F0DBF8002CB8BF6442322C06469C
:10ABC00002DD0023BB6224E0069809F0E9FA20F0D8
:10ABD000030009F0CBF88046687B09F0C3F8014612
:10ABE000304609F017F93D490446404609F0C6F9D8
:10ABF0000146204609F00EF909F0D2FABB6A184462
:10AC0000374B9842A8BF1846364B9842ACBFB86243
:10AC1000BB62BB6A6FF0FF005B13B3F5807FA8BF18
:10AC20004FF480739842B8BF184609F09FF88046E9
:10AC3000304609F0B5FAEB785843801109F096F8E0
:10AC4000294B04461B78032B11D9B5F84E60B6F595
:10AC5000FA7F0CD209F0A4FA7342984203DBB042A7
:10AC60000346A8BF3346184609F080F8044695F815
:10AC7000512062B1530803D09A42A8BF1A4600E09F
:10AC8000012220461949FB69FCF7FCFF04464146B6
:10AC9000204608F0B7FF09F083FA00B209F066F821
:10ACA0000DF052F8A7F86C00204609F079FAB86761
:10ACB000404609F075FA0023C7F88400C7F89030C1
:10ACC0000DB0BDE8F08F00BFA69B443B541500209B
:10ACD000F7CC9238041100204010002000803B4542
:10ACE000FEFFFF0F020000F000200020681500208A
:10ACF0002DE9F74F03F0EAF8A64C80462668656810
:10AD0000A768861BF643451BC71BED43FF43F60FA1
:10AD1000ED0FFF0F2EB93FB9002D00F08782B94625
:10AD20002CE04FF0000929E0B14627E003EB8A0B45
:10AD3000BBF802301A050ED413F4805F1DBF964A8B
:10AD40009BF801101268954A954B14BF52F82120C8
:10AD5000126843F82A20BBF80230D80516D49905AA
:10AD60000AD5904B1B7813F0040F0CBF8E4A8F4A04
:10AD70008B4B126843F82A2009F10109207B5FFA06
:10AD800089FA8B4982450B68D0D326E0894A504620
:10AD9000594605F06FFA884B1B885A0603D5504672
:10ADA0005946864A16E0580703D550465946844A04
:10ADB00010E0190703D550465946824A0AE09A071F
:10ADC00003D550465946804A04E0DB07D4D55046A7
:10ADD00059467E4A05F04EFACEE7DFF808E20093C6
:10ADE000BEF906307822A3F57A7353434FF47A7292
:10ADF00093FBF2F3F34603F22B13019300225FFA65
:10AE000082FE864517D2009B03EB820EBEF802E05D
:10AE10001EF4806F0DD040F2671ADFF88491019B19
:10AE200039F822E09E449EFBFAFC0AFB1CEE29F84E
:10AE300022E00132E3E74DB308F5C333A03363608A
:10AE4000637B544A13BB9373614B1B6813F0020F6F
:10AE50000AD0DFF894E19EF800E0BEF1000F03D0C5
:10AE60004FF0010E82F80EE0DA0506D5594B5B79FA
:10AE70001BB1A37B43F00203A3734A4B1B7813F06F
:10AE8000050F02BFA37B43F00403A37394F80EE005
:10AE9000BEF1000F03D13F4B5B7B002B4FD094F8EA
:10AEA0000DC01CF0010FACF10C031DD1BCF1030F60
:10AEB00007D8DFF8E8901EF0040F3B4A08BF4A4667
:10AEC00000E0364AACF1040CBCF1070F05D8DFF8FE
:10AED0001CC11EF0010F18BF6246DBB2032B0ED857
:10AEE0001EF0020F3C4B06E0DBB2032B06D82F4BC3
:10AEF0002A4A1EF0020F18BF1A4600E0274A4FF0F8
:10AF0000000C5FFA8CF383420DD20B6803EB8C03C9
:10AF10005B881B0642BFD2F80090214B43F82C906F
:10AF20000CF1010CEDE785B1BEF1000F08D0637B99
:10AF3000184A0133DBB2142B06D1002304E025B1FB
:10AF4000637B002BF3D100E05373002E52D0234AD1
:10AF50003223B2F90250B2F90020002DB8BF6D4281
:10AF6000002AB8BF524295FBF3F592FBF3F2EDB223
:10AF7000D3B2AB4238BF2B46194A13B192FBF3F35D
:10AF800000E0134643442360E37B024A83BB012372
:10AF90002FE000BF44160020C81C002024C3010875
:10AFA000FA0D0020A33000208CC101087CC10108EB
:10AFB000E81100208EAA0108E411002094AA0108DB
:10AFC0009AAA0108A0AA0108A6AA0108ACAA010829
:10AFD00050260020FC24002094C101080411002008
:10AFE000400D03008C260020701100209CC1010838
:10AFF0000023D3738F4D904B2D78E27BADB9002F9A
:10B0000000F00F818D4B267B1A788D4B02F00402E5
:10B0100093F800C08B4BD2B2D3F800E00B6800214C
:10B02000894D03EB86060F46B5E01AB9874A1A61C7
:10B03000002508E0864AFAE70A68AB00D618768849
:10B04000760604D40135EBB28342F5D3D7E7814EBF
:10B05000B6F90060192E25DD12F803E094F814C04B
:10B060000EF00F09E14526690CDCDFF8CCC19CF835
:10B0700015C0BCEB1E1FDEBFD6F800C0DFF8D8E15C
:10B0800043F80EC012F803E094F816C00EF00F0952
:10B09000E14533DBDFF8A0C19CF815C0BCEB1E1FF7
:10B0A0002CDC26E0193629DA12F803E094F814C0F3
:10B0B0000EF00F09E14526690CDCDFF87CC19CF835
:10B0C00017C0BCEB1E1FA2BFD6F800C0DFF888E196
:10B0D00043F80EC012F803E094F816C00EF00F0902
:10B0E000E1450BDBDFF850C19CF817C0BCEB1E1F1D
:10B0F00004DBD6F800E0584E43F806E0554EB6F9AA
:10B100000260192E1BDD12F803C094F814E00CF055
:10B110000F09F14526690CDCDFF81C9199F81590B0
:10B12000B9EB1C1FDEBFD6F80090DFF82CC143F846
:10B130000C90D25C02F00F0CF4451EDD82E719364C
:10B1400080DA12F803C094F816E00CF00F09F1450C
:10B1500026690CDBDFF8E09099F81590B9EB1C1F1D
:10B16000DEBFD6F80090DFF8F0C043F80C90D25C58
:10B1700002F00F0CF445FFF665AF94F817E0BEEB54
:10B18000121FA2BF3668344A9E505BE758880005FC
:10B1900004D404330435B342F8D122E04AB101EBC0
:10B1A0000C0A06209AFBF0F900FB19A001280DDC1F
:10B1B00001E057B9012793F801900EEB89003EF8A2
:10B1C00029A090F80290C07803E01746002081463D
:10B1D0008246013125F802AC85F800906870C9B24A
:10B1E000D7E7174A1378013B13F0FF0308BF062384
:10B1F0001370124B1B785B0741BFBBF906304FF44D
:10B200007A72A3F57A7303EBC30348BF93FBF2F39F
:10B21000124A46BF0133DBB2012392FBF3F34344EE
:10B22000A36003B0BDE8F04F03F098BF03B0BDE8E2
:10B23000F08F00BF0A30002044160020A330002009
:10B2400044000020C81C0020FC0D002098C101080B
:10B2500024C3010804110020FA0D0020400D030052
:10B2600010B508F083FD0021044608F08FFF08B1F7
:10B27000204601E004F10040054908F07FFE054941
:10B2800008F0C8FDFCF7E0FF034B186010BD00BFDD
:10B290008096184B35FA8E3C6C000020F8B59C4B1C
:10B2A00004461B68187818B1012800F06A819AE2F8
:10B2B000242C984D0CD006D80A2C00F0D9800D2CE7
:10B2C00000F0D68048E12A2C06D02C2C04D043E193
:10B2D00028706870A87050E18F4B69782F78002033
:10B2E0008C4A58542FBB1978D770472921D15978E7
:10B2F00050291ED19978472907D1D978472904D1F7
:10B300001979412901D10121D1709978824A5229B4
:10B3100003D1D1784D2900F0688299787E4A472977
:10B3200007D1D178532904D11279562A04BF0322B8
:10B33000EA70EA78774E022A39D0032A4CD0012AE3
:10B3400040F08580BA1E072A00F28180DFE802F013
:10B3500004080F131A257F2A07F0AAFF686076E019
:10B360001B78532B73D16B685B426B606FE007F007
:10B370009FFFA8606BE01B78572B68D1AB685B42DE
:10B38000AB6064E01B78302B644B1A788CBF42F0C2
:10B39000020222F002021A7059E0002007F0E8FFD2
:10B3A000287354E0002007F0E3FFE8814FE0072F07
:10B3B00006D0082F4BD1012007F0DAFF708246E05B
:10B3C000012007F0D5FF41F2184358434FF47A7338
:10B3D000B0FBF3F030823AE0022F07D0032F0AD1FE
:10B3E000002007F0C5FF4E4B187030E0002007F03A
:10B3F000BFFF30752BE02AD93A1F9210337D0132FE
:10B40000D2B2013B02EB8303DBB2102B1FD8F91E33
:10B41000C2F1010201EB8202D2B2012A0BD0042A4E
:10B4200011D100205E1E07F0A3FF3E4B002298556D
:10B430003D4B9A5507E03D4A5E1E0020935507F0AC
:10B4400097FF3B4B98553B4A136801331360314BD0
:10B450002A2C18BF9A7807F101074FF000000CBFA3
:10B46000012254402F7068700CBF5A759C7084E0A4
:10B47000687D002848D0304B13F8012D2F495A70B1
:10B480008B42F9D1244A234C13785278402B85BF44
:10B49000373B1B011B01DBB298BF03F0F003402ACE
:10B4A0008CBF373A303AD2B21344AA78DBB29A4210
:10B4B00027D121230B702249E0780B68012803F182
:10B4C00001031E4A0B600AD002281CD1722313709C
:10B4D000228A1C4B1A80628A1B4B1A8013E0672356
:10B4E00013700E4B1B789F070ED5184B62681A60BD
:10B4F000A2685A60227B164B1A70E289154B1A809B
:10B5000002E03F230B70002000236B7535E000BF85
:10B51000880700205C1600207C26002024110020D3
:10B52000A0100020D1100020C1100020A110002088
:10B53000B11000205421002084030020700300205B
:10B540006021002026110020881000202C110020EE
:10B550002A110020281100206B78687D0E2B9FBFD8
:10B56000A54A591C5170A54A98BFD454A24A18B98B
:10B5700093785C40947000E00020003018BF0120F8
:10B58000F8BD9D4B0022997D082900F22C81DFE84F
:10B5900001F0050B0F15202B475D6700B52C40F01F
:10B5A0002281DA75012239E0622C08BF022235E0DF
:10B5B00003229A751C765C769C7614E104229A75B7
:10B5C0005A7E997E2244D2B25A760A449A76DC7622
:10B5D00009E105229A755A7E997E2244D2B25A76A2
:10B5E0000A449A769C83FEE006229A755A7E997EDA
:10B5F0002244D2B25A760A449A769A8B02EB0424F9
:10B60000A4B2B4F5AC7F82BF7B4A0121D175002280
:10B610009C83DA83002C40F0E68007229A75E2E0F2
:10B620005A7E997E2244D2B25A760A449A76DA8BAE
:10B63000B2F5AC7F3EBF7049891881F820400132D5
:10B64000998B92B29142DA83E7D9CCE008229A75BD
:10B650005B7EA34200F0C780674B0122DA750DE0E4
:10B66000674D9A7515F8012D6A70664A9542F9D1B1
:10B67000997E614AA14206D03F232B70624A5368EB
:10B6800001335360AFE06148016801310160D07D52
:10B6900010B13E232B70A6E021212970D17E06290E
:10B6A00041D004D8022907D0032923D0F8BD12299C
:10B6B00059D0302967D0F8BD5021546A29705449B7
:10B6C0004C60946A0C60116B4FF47A7491FBF4F146
:10B6D000504C218092F878114F4A19B1117841F0FD
:10B6E000020102E0117821F002011170012283F8B9
:10B6F000792169E05321297092F82510CE0705D5EC
:10B7000092F82420D51E6A426A4100E0024602F007
:10B71000010183F87811002A56D13F490A7822F0B6
:10B7200002020A7050E04F21297092F82B10CC07CA
:10B7300005D592F82A20D11E4A424A4100E002462D
:10B7400002F0010183F8781122B933490A7822F016
:10B7500002020A7093F84F10304A1170B3F84C107F
:10B760002F4A118030E05621546B29702D490C80EE
:10B7700042F21074916B91FBF4F12B4C218001216A
:10B7800082F87A1120E04921297092F82410274A82
:10B79000102988BF10211170254914780022A24277
:10B7A0000ED20E7A234D56554E7A234D5655CE7AEB
:10B7B000224D565511F80C6F214D56550132EEE7CA
:10B7C00020490A6801320A6093F879310A4A002B4D
:10B7D0003AD092F87A31BBB3002182F8791182F81D
:10B7E0007A111846F8BD0020F8BD1279432A7FF47B
:10B7F00094AD0222EA7090E55C1600207C260020C1
:10B8000084030020700300206807002060210020CE
:10B810002C11002028110020241100202A110020C2
:10B82000FA0000202611002088100020A01000201F
:10B830007C160020A1100020B1100020C1100020B3
:10B84000D110002054210020F8BD0449044B0968A0
:10B85000002218705A6199611A7770477426002087
:10B8600068070020F8B5101A0D461F4608F07EFA4A
:10B870000446781B08F07AFA174B079E196808F0FF
:10B88000C9FA21460546204608F0C4FA294607466B
:10B89000284608F0BFFA0146384608F0B3F90CF024
:10B8A000B7FC0E4908F0B6FA08F0A0FC069B294642
:10B8B000186004F100400CF01FFB094908F0AAFAD7
:10B8C000084908F09FF908F06BFC0028BCBF00F5A0
:10B8D0000C40A0303060F8BD6C0000202C7D8E3F05
:10B8E000A00CB34500A00C4644F25063984203DD1F
:10B8F000A0F50C40A0387047034B9842BCBF00F540
:10B900000C40A030704700BFB0B9FFFFF7B5036827
:10B91000174C184D23600B68174E63600068FFF7E3
:10B920009FFC95E80300154B0196009394E80C00EA
:10B93000FFF798FF3668124B60681E606B68114F06
:10B94000C01A08F013FA104B196808F063FA08F0EF
:10B9500027FC2A68236878609B1A3B600B4B1E60AB
:10B960000B4B1B68DA880B4B1A8003B0F0BD00BF8D
:10B97000D42000202C110020E0200020DC2000201A
:10B980001C210020E42000206C0000201421002055
:10B99000380F00201021002070B50446407908F0CF
:10B9A000E1F91E4908F0EAFA1D4D1E4E2860E07BC1
:10B9B00008F0D8F9194908F0E1FAEE606860A0795A
:10B9C00008F0D0F9184908F0D9FA184D2860207C01
:10B9D00008F0C8F9114908F0D1FA6860A07E08F0B3
:10B9E000C1F9134908F0CAFAEE60A860E07908F0DE
:10B9F000B9F90D4908F0C2FA0E4D2860607C08F0D4
:10BA0000B1F9064908F0BAFA6860E07E08F0AAF9D0
:10BA1000074908F0B3FAEE60A86070BD0000C842A4
:10BA2000EC2000200000FA4400002041FC2000200F
:10BA300000007A442021002010B50C4C23789B078D
:10BA400013D50B4B1B78042B0FD90A4A0A4B1068ED
:10BA5000526818605A60FFF703FC084B1A88084BBD
:10BA60001A80237843F00103237010BD24110020B5
:10BA70002A1100202C1100208C100020FC10002026
:10BA800030210020164B13B51B681B0325D5154B21
:10BA9000154C1B7815498DF80030154B20681B7824
:10BAA0008DF8013008F0B6F908F0A0FB11498DF8C7
:10BAB0000200606808F0AEF908F098FB8DF803000A
:10BAC000A06808F093FB0C4B8DF804001B780A204B
:10BAD00069468DF80530FDF747FD02B010BD00BF87
:10BAE000502600204026002064260020000020412F
:10BAF0006026002000007A4444260020054A13787E
:10BB000083F001031370044A00231360034A136097
:10BB1000B8E700BF442600205C26002058260020FD
:10BB2000094A137818441346C0B210F0800F18BFAA
:10BB300080381070054A19781378994201BF0023A4
:10BB40001370014A137070475522002054220020C0
:10BB500010B50A4B0A4A1B7842609C18094A0460D7
:10BB600012789A4225BFD31A0B60C3F180030023D9
:10BB70002EBF4B600B604A6010BD00BF55220020F5
:10BB800056220020542200201FB5684602A9FFF764
:10BB9000DFFF044B02981B6803440398184405B068
:10BBA0005DF804FBDC0600202DE9F04F814689B0EA
:10BBB00002930023039104920193049A934207DABB
:10BBC000039A019952F82320013311440191F4E7BB
:10BBD000029B019D002B57D103F094FC002853D108
:10BBE00002987FE00222414E8DF81C201A0C4FF47F
:10BBF00080578DF81D2006201A0A8DF81E208DF81A
:10BC00001F3003F0A7FC776106213948F9F7C8FB1C
:10BC1000384B01223761C8461A707761264634488E
:10BC2000002107AA0423F9F78DFB039F4FF0000AB8
:10BC3000049B9A451DDABC4657F8043B4FEA8A0B31
:10BC4000002B48D0B34235D333462948002159F858
:10BC50000B20CDF814C0F9F775FB59F80B30DDF85F
:10BC600014C0334449F80B30DCF800309E1BCCF88C
:10BC700000601E4B4FF480521A611F4A2D1B13683F
:10BC80001C44029B14605BB355B31B4B1B68DCB2B6
:10BC90002A19B2F5807F194A88BFC4F58074D2682A
:10BCA00098BF2C4693429DD3154A00231370154A22
:10BCB000137015E0D8F800200D480021F9F742FB79
:10BCC00057F8043CD8F80020F61A1344C8F800309E
:10BCD000002347F8043C0AF1010A08F10408A7E729
:10BCE000019B581B09B0BDE8F08F00BF000C01405C
:10BCF00000380040D9060020DC0600200C0000209F
:10BD0000542200205522002030B50B4C0B4D2278D8
:10BD10002B7885B09A420CD0684602A9FFF718FF2D
:10BD20000123684602A90222FFF73EFF00232B7081
:10BD3000237005B030BD00BF5522002054220020E2
:10BD400030B50E4D0E4C2A78237885B09A4211D02A
:10BD5000684602A9FFF7FCFE002302A902226846FA
:10BD6000FFF722FFFFF7DCFE20782B781B1A5842E2
:10BD7000584100E0012005B030BD00BF5522002031
:10BD80005422002070B50F4C0F4E4FF4805545F2F1
:10BD9000082003F0DFFB062165613046F9F700FB60
:10BDA0000A4B0122256130461A70C7216561F9F7F7
:10BDB000F7FA074A002325611370064A1370064AF2
:10BDC000136070BD000C014000380040D90600200F
:10BDD0005422002055220020DC06002001480249A0
:10BDE00000F0E4B800080040AC1E00200148024901
:10BDF00000F0DCB800040040841E00204FF08040BA
:10BE0000014900F0D3B800BF5C1E00200148024980
:10BE100000F0CCB8002C0140341E0020014802493B
:10BE200000F0C4B8002C0140341E0020026D70B533
:10BE300015880446ADB2A90613D5036B8BB9C36A46
:10BE40001BB1908880B298470BE0E1699288406905
:10BE50004E1CD2B2E6614254E169E268914228BFC9
:10BE6000E3612B0613D5636AA26A9A42236D0AD056
:10BE7000511CA069A162825C9A802369994206D311
:10BE80000023A36270BDDA6822F08002DA6070BD20
:10BE9000026B0346C16810B5406942B11A6C8C1A36
:10BEA000013A08BF0A46005D1A64C0B210BD1A6AA2
:10BEB000805C01328A4228BF0022C0B21A6210BDE3
:10BEC000436B13B190F844007047836A406A1B1AB1
:10BED000584258417047036B13B15B68016C01E035
:10BEE000C369016A8B423CBFC2689B18581AC0B232
:10BEF0007047836A8169426B1944D160416A9942F3
:10BF000097BF0169CB1ACB1A536096BF00235360C9
:10BF100083624FF0000380F84430136888BF816269
:10BF200043F0010313607047436A8269D154436A46
:10BF300002690133934228BF00234362436B1BB164
:10BF40001B68DB0705D4D4E7026DD36843F0800398
:10BF5000D360704738B50D4B0D4D99680D4B1A687D
:10BF60001C465288114203D001F0B0FF286007E060
:10BF700001F0ACFF2B68984282BFC01A064B1860D4
:10BF800023685A68054B5A6138BD00BF000C014058
:10BF9000D8170020640700200000002000040140A2
:10BFA0004171FCF7E3BE8160FCF7E0BE2DE9F04192
:10BFB00005460E46078A83899BB21F40002F37D063
:10BFC000B7FA87F24FF00043D340DB4399B21F40EA
:10BFD000A2F11B032982042BF0D8DFE803F0221F13
:10BFE0001C190300746A24B1013C0023A4B27362DB
:10BFF00001E0AC8DA4B2D6F82080B8F1000FDDD0FE
:10C00000D8F80030404621469847D8F80480F4E735
:10C010003068A98E08E07068298F05E0B068A98FA4
:10C0200002E0F068B5F84010036889B29847C5E7A8
:10C03000BDE8F081254B10B55A43254B254C1B68B4
:10C040000139B3FBF2F20388013AA04289B292B2FD
:10C050009BB212D004F50064A0420ED0B0F1804F24
:10C060000BD0A4F59834A04207D004F58064A04218
:10C0700003D004F58064A04202D123F070039BB288
:10C08000154CA04206D004F58064A0421CBF23F4E6
:10C0900040739BB203800F4B8185984202850FD07D
:10C0A00003F5006398420BD003F54063984207D034
:10C0B00003F58063984203D003F58063984201D171
:10C0C000002303860123838210BD00BF40420F007E
:10C0D00004010020002C01400010004073B505460B
:10C0E0000068FFF7A7FF2A680124138800269BB287
:10C0F00043F001031380EB7A01A88DF804308DF82A
:10C1000005408DF806608DF8074006F011FFEB7AC8
:10C110001B2B0BD1192301A88DF804308DF8054095
:10C120008DF806608DF8074006F002FF02B070BD82
:10C130000C4B800A98420CD004D8B0F5801F0CD16B
:10C1400001207047084B984205D04933984206D0E9
:10C1500003E00220704703207047FE207047002054
:10C16000704700BF01001000020010002DE9F843E5
:10C1700004680746204688469146FFF7D9FF032802
:10C180004BD8BA7A9108B8F1000F06D1A589AEB2A2
:10C1900002258D4026EA0505A5810A2303FB00132D
:10C1A0001F4A42F82380043342F82390B8F1000F6D
:10C1B00007D0BD7AA189AD080223AB400B439BB2E7
:10C1C000A3812823434303F120011144EFF3128696
:10C1D000502585F3128803F10C051C3315441344D4
:10C1E00055F8047F17B10F60296804319D42F7D1DB
:10C1F00000230B60F3B283F31188282303FB002094
:10C20000036A23B1A3899BB243F0010304E0A3892D
:10C2100023F001031B041B0CA381BDE8F88300BFBE
:10C22000341E002096E695E694E60148FEE500BF40
:10C23000DC1700200048F9E5301800200B4B4FF4C4
:10C2400000525A604FF6FE730948D0F88C201168EE
:10C250000B401360C26FD0F880309A4201D0583042
:10C2600047E6012380F89C30704700BF0000024081
:10C27000D81700202DE9F0431E469C4B8DB0984204
:10C28000894690469DF850705ED1994B994AC3F803
:10C2900060809A6503F1AC02DA6603F5D6721A671C
:10C2A0004FF480725A669A66934AC3F8A800C3F89E
:10C2B0008C20A2F54842403AC3F8A0208F4B9A69DF
:10C2C00042F480429A615A6942F001025A610223A3
:10C2D0008DF803303A074FF40073ADF8003001D504
:10C2E0001C230FE0B30706D51823854869468DF84F
:10C2F000023003F011F8F5070AD54FF48063ADF86A
:10C30000003048237E4869468DF8023003F004F877
:10C3100001240E23002501A88DF804308DF8054076
:10C320008DF807408DF8065006F002FE252301A87F
:10C330008DF805408DF807408DF804308DF80650D3
:10C34000704C06F0F5FD50E06F4B984240F0C9800C
:10C35000674B684AC3F80C805A6003F52B729A61E8
:10C3600003F56B72DA614FF480721A615A61674AA1
:10C370005865DA641A65614B3C07DA6942F4802239
:10C38000DA619A6942F008029A614FF002038DF86F
:10C3900003304FF48063ADF8003001D51C230FE06B
:10C3A000B00706D518235A4869468DF8023002F0C6
:10C3B000B3FFF1070AD54FF40063ADF8003048230E
:10C3C000534869468DF8023002F0A6FF27238DF806
:10C3D00004300022012301A88DF805308DF80620D5
:10C3E0008DF8073006F0A4FD4A4C0025012384F89F
:10C3F00044302562E561A5626562C4F82C906671DF
:10C40000C4F80880A7712046FCF7B0FCF20731D5CC
:10C41000206B002826D0E36C039501934FF48053E2
:10C420000A9380230693E3680595049320230993D8
:10C4300063690795029308950B9501F067F801A9C8
:10C44000206B01F045F8226B216D136843F0010366
:10C4500013608B8A9BB243F040038B8253689BB27C
:10C46000236407E04FF6DF72236D1A80DA6842F02A
:10C470002002DA60B3072CD5606B28B3A36C0025CB
:10C4800001934FF480530A93802306932369029506
:10C4900004931023039305950795089509950B952B
:10C4A00001F034F8606B01A901F012F8636B1A68AF
:10C4B00042F002021A60226D5D605D60938A9BB259
:10C4C00043F08003938204E0226DD36843F080033D
:10C4D000D360226D204693899BB243F4005393812D
:10C4E00000E000200DB0BDE8F08300BF003801403F
:10C4F000D8170020B4AA01084400024000100240EE
:10C500000008014030180020004800400448004066
:10C51000000C0140DC17002038B500240B4D605999
:10C52000254403F0FFFB696811B10948FBF7EAFDF8
:10C53000A96811B10748FBF7E5FD0748103403F07F
:10C54000F1FBB4F5F07FE9D138BD00BFCCAA0108FA
:10C55000EAC90108F0C9010831D4010870B50546DF
:10C5600028460BF028FA064658B91A4B1A485A7949
:10C570001A4BBDE8704003EB8203D3F8DC11FBF7E4
:10C58000C1BD2846164932460BF01EFA60B915485F
:10C5900003F0C8FB144C54F8041F19B11348FBF7FF
:10C5A000B1FDF8E7124805E00024124B53F82410BF
:10C5B00021B91148BDE8704003F0B4BB28463246AB
:10C5C0000BF002FA01340028EFD1024B0B4D5C71E5
:10C5D000C6E700BFB0260020F6C90108CCAA0108B2
:10C5E00002CA010807CA0108A8AC01081ACA010852
:10C5F00031D40108ACAC010802C9010858C60108D1
:10C60000F0B585B004460BF0D6F9082826D1621E95
:10C61000E01D1F4912F8013F09681944497801F0EB
:10C620000301022908BF203B82421370F1D1254645
:10C6300004F1080715F8016B164831460BF0ADF907
:10C6400020B1284631460BF0A8F910B1FAF74CFD9D
:10C650001CE0BD42EED1204606F0FAFB0E4803F086
:10C6600061FB00230D4A04A91A4492F88A210A4466
:10C670000849595C0133082B02F80C1CF2D1002345
:10C68000074801A98DF80C30FBF73CFD05B0F0BD63
:10C690000C010020B4DF01081ECA0108B0260020EA
:10C6A000D5D20108264B274C1D6880B52068FBF7C2
:10C6B0005FF92846FBF75CF9206841798A0703D4C3
:10C6C00041F0020101F0C6FC1F4B08221A611F4B0A
:10C6D0001A681F4612F4003F1FBF06236371E379F7
:10C6E00023F001031CBF43F00203E371206801F053
:10C6F000BDFC90B1144E08237361124B186801F011
:10C70000B2FC8046FEF7CAFD08B103F07DFE284664
:10C71000414601F0AEFC08233361284601F0A6FC37
:10C7200038B12846266801F09EFC0146304601F0EB
:10C73000A0FC3B689B03D9D504F02FFAD6E700BFD5
:10C74000FC1F0020841C0020000C0140502600200B
:10C750002DE9F04705460BF02EF92F4E0446D6F88A
:10C76000088090B92D4803F0DDFA2D4B53F82410C2
:10C7700049B10123A34013EA080F02D02948FBF76F
:10C78000C1FC0134F1E7284822E028462749224627
:10C790000BF01AF958B9264803F0C4FA254C54F89E
:10C7A000041F0029EFD01F48FBF7ACFCF7E72B78FC
:10C7B0004FF000092D2B03BF013504F1FF344FF07A
:10C7C000010A4FF0000A164B53F8297027B91A488E
:10C7D000BDE8F04703F0A6BA2846394622460BF0DA
:10C7E000F3F8A8B9012000FA09F0BAF1000F03D05C
:10C7F000FBF71CFE114803E040EA0800B060104857
:10C8000003F090FA3946BDE8F0470E48FBF77ABCD2
:10C8100009F10109D7E700BFB026002024CA0108AA
:10C8200014AD01081ACA010831D4010802CA01086E
:10C830002ECA010810AD010802C901083ACA010850
:10C8400043CA0108D4D2010810B5084803F06AFAB7
:10C85000074B00241C741C64064B1C7001F0AEFDD9
:10C8600003F0D6FC044B1C6010BD00BF4BCA01088E
:10C87000841C0020A4300020FC1F002070B5064658
:10C8800000240B4BE518AA8816420AD0E158094843
:10C89000FBF738FC2846002103F0D5F9064803F0E1
:10C8A00041FA40F6944314349C42EAD170BD00BF73
:10C8B000B8B3010877CA010831D4010808B508489F
:10C8C000FBF720FCFFF75EFA02F01CFE18B96420AB
:10C8D00001F021FBF8E70348BDE80840FBF712BC74
:10C8E00081CA01088ECA01082DE9FF410A4806885D
:10C8F00085684488B0F80480C768FFF745F9CDF82B
:10C9000000800290019731462A4623460348FBF7F0
:10C91000F9FB04B0BDE8F0810C00002096CA0108C4
:10C92000F0B504788BB005460CB1002436E04A4BD4
:10C9300019680E2303FB0411B1F91D51B1F9192136
:10C94000B1F91B31009591F8205101F58C700195DA
:10C9500091F8215101F59071029590F9070003902B
:10C9600091F902103D48049121460134FBF7CAFBBE
:10C97000082CDCD16DE02D2B14D1072C1BDC2846B4
:10C980000BF06EF80AAB661C03EB440424F8100CA1
:10C9900015F8013F303B092BFAD934462B78002B90
:10C9A000E9D104E0A3F13002092A09D8E5E7082C0F
:10C9B000BDF8182009D00BB0BDE8F040FAF794BBE1
:10C9C000202BF8D101352646E7E7072AF3D840F2B5
:10C9D000DC55BDF81A00204BA0F2EE2189B2A94225
:10C9E0001B68E8D8BDF81C10A1F2EE24A4B2AC423A
:10C9F000E1D8BDF81E7004B23EB2A642DBDB0DB238
:10CA0000AE42D8DCA542D6DBBDF92440642CD2D19D
:10CA1000BDF8266034B2112CCDDCBDF82050B42D09
:10CA2000C9D8BDF82240B42CC5D812B24FF00E0EB2
:10CA30000EFB0233A3F81B116421A3F81901A3F81C
:10CA40001D7183F8205183F8214183F81F1183F869
:10CA500022610BB0F0BD00BF5C100020F3CA0108DA
:10CA6000F0B504468FB020460AF0A5FFC5B21DBB45
:10CA7000AB4803F057F9AB4C94F8D61009B9AA4863
:10CA800053E049B294F8D42094F8D530009194F84A
:10CA9000D710A648019194F9D8100734029194F95F
:10CAA000D210039194F8D310049129460135FBF775
:10CAB00029FB102DE0D1E2E720469D4905220AF02E
:10CAC00083FF0546B8B929469A4870220AF02FFF1D
:10CAD0002846994B19680E2303FB001301300022EE
:10CAE000082883F8232183F8242183F8252183F85B
:10CAF0002621F0D112E12046904904220AF064FF79
:10CB000005462046002D4AD120210AF046FF002884
:10CB100000F00481461C30460AF04DFF2C460746C3
:10CB2000874B53F824502DB986480FB0BDE8F0402C
:10CB3000FBF7E8BA30462946FAB20AF045FF01345D
:10CB40000028EDD1774A164602F17001002382F8E1
:10CB5000DA3082F8D63082F8D53082F8D430073215
:10CB60008A42F3D1784901EBC40191F8A0229342A3
:10CB700010DAD1F8A472C3EBC302B0183A441768B4
:10CB800000F1D401C0F8D470908801338880927984
:10CB90008A71E7E729466D48FBF7B4FA8FE06C49E4
:10CBA00007220AF011FF05462046002D49D1202119
:10CBB0000AF0F3FE06460AF0FEFEC4B26CBB6548FE
:10CBC000FBF7A0FA214664480134FBF79BFA0E2CD0
:10CBD000F8D15548FBF796FA002460482146FBF748
:10CBE00091FA0025544A012311680E2202FB041217
:10CBF000D2F82321AB401342594B5A495A4808BF37
:10CC000019460135FBF77EFA0E2DEBD1464801346B
:10CC1000FBF778FA082CE0D180E0304653490AF05F
:10CC200023FF2C4600284CD0022C4FD00AF018FFCE
:10CC300006AB43F824004D4900200AF015FF0134EB
:10CC4000F0E74A490AF010FF002460B1082C38D000
:10CC50000AF006FF06AB43F82400444900200AF01E
:10CC600003FF0134F1E7082C2BD1069B0F2B28D8AA
:10CC7000DDF81CE0BEF1070F23D8089F0D2F20D848
:10CC8000099E06F16402C82A1BD80A9DFF2D18D8F8
:10CC90000B98642815D80C99642912D8884210DAA8
:10CCA0000D9C032C0DD8324AC3EBC303134483F805
:10CCB00004E05F719E71DD71187259729C722D4C87
:10CCC000D1E60FB0BDE8F040FAF70EBA069B072B8D
:10CCD00020D807990D291DD80278722A0DD06E2A06
:10CCE00018D1154A0E20126800FB032301228A4046
:10CCF000D3F8231121EA020209E00F4A0E2012683C
:10CD000000FB032301228A40D3F823110A43C3F80E
:10CD1000232101E0FAF7E8F90D4CA4E60FB0F0BDCD
:10CD20001BCB0108B026002031D4010846CB0108F6
:10CD3000D2C80108842700205C100020FDC801082B
:10CD4000ACAC010802C90108CCAA010811C901084C
:10CD500013CB0108F4C9010862CB01084CDF0108BC
:10CD60006CD70108B2D6010867CB01086BCB01086C
:10CD70008027002058C601082DE9F74304780546AE
:10CD80008CB9324D95F89F12B5F89C2295F89E32D9
:10CD90002F48009121460134FBF7B4F9102C05F11E
:10CDA0000405EFD14FE00AF05BFE0F28044636DCA5
:10CDB000284620210AF0F1FD264EE4B2D6F8448040
:10CDC000451CA400002728460AF04AFE5FFA87F9AE
:10CDD000B9F1010F83B208D0B9F1020F0BD0B3F54E
:10CDE000B47F25D2726C13530AE0FF2B20D8736CEA
:10CDF0002344987004E0FF2B1AD8736C2344D87036
:10CE000028462C210AF0C9FD054608B1013502E08B
:10CE1000B9F1020F0CD10137032FD4D113E00E4822
:10CE20000E4900220F2303B0BDE8F043FBF76AB9B7
:10CE300008EB0400002104220AF079FD03B0BDE8EC
:10CE4000F043FAF751B903B0BDE8F083B0260020F3
:10CE50006DCB0108841C002071C8010890C801082E
:10CE60002DE9F04FAC498BB004460AF069FDAB499F
:10CE7000002820460CBF012507250AF061FDA849BE
:10CE80000028204608BF02250AF05AFD002808BFE6
:10CE90000425E90740F1FB80A24802F043FF00208F
:10CEA00002F04CFDA04CA14802F03CFFA04802F06B
:10CEB00039FF62799F4BA04803EB8203D3F8DC1162
:10CEC000FBF720F99D48FBF71DF926460027D6F809
:10CED00014800021404607F031F920B19848FBF753
:10CEE00011F9002669E039469648D6F818B0D6F808
:10CEF0001CA0D6F82090FBF705F94046002107F06A
:10CF000027F910B1202002F005FF06A94046FAF7E4
:10CF10007FFF01468C48FBF7F5F85846002107F0E3
:10CF200017F910B1202002F0F5FE06A95846FAF7CD
:10CF30006FFF01468448FBF7E5F85046002107F0F3
:10CF400007F910B1202002F0E5FE06A95046FAF7D5
:10CF50005FFF01467C48FBF7D5F84846002107F003
:10CF6000F7F810B1202002F0D5FE06A94846FAF7DE
:10CF70004FFF013701467548FBF7C4F80C2F06F147
:10CF80001006A4D1AAE749B294F8D42094F8D53079
:10CF9000009194F8D7106E48019194F9D810073495
:10CFA000029194F9D210039194F8D3100491314670
:10CFB0000136FBF7A7F8102E03D094F8D6100029FD
:10CFC000E1D100260E2777430024624A0123926CA8
:10CFD000A3403A44D2F80A20134240F0948001342E
:10CFE0000E2CF2D10136082EECD15B4802F09AFEED
:10CFF0004D4B5A4C9F6854F8041F19B15848FBF721
:10D0000081F8F8E70E46574B53F826404CB1012300
:10D01000B3403B4203D054482146FBF773F8013636
:10D02000F1E7524802F07EFE21463F4B0AAA0B442C
:10D0300093F88A3113444E4A8A5C0131082903F877
:10D04000102CF2D1002306A94A488DF82030FBF7B6
:10D0500059F8494802F066FE4848FAF781FB48480B
:10D0600002F060FE4548FAF745F8464802F05AFEDD
:10D070004248FFF781FE4448FBF744F84020FFF7A1
:10D08000FDFB424802F04EFE3C48FAF70BFCAA07B3
:10D0900026D53F4802F046FE3E4802F043FE3748A0
:10D0A00002F08CFC3C4802F03DFE3448F9F7A3FF47
:10D0B0003A4802F037FE3148FAF7A2FA3848FBF74F
:10D0C00021F82E48FAF724F9364802F02BFE2B48B7
:10D0D000FFF726FC2C48FBF715F88020FFF7CEFB66
:10D0E0006B0716D5304802F01DFE304802F01AFEDC
:10D0F000224802F03DFC2448FBF704F84FF480700E
:10D10000FFF7BCFB05E0314622462948FAF7FAFF53
:10D1100065E70BB0BDE8F08F81CB0108F6CF0108C1
:10D1200088CB01088ECB0108B02600209CCB0108DB
:10D13000AECB0108CCAA0108BACB0108C5CB0108C7
:10D14000D2CB0108DFCB0108F3C90108D5D2010811
:10D15000E7CB0108841C002006CC010810AD0108B3
:10D1600016CC010814AD010824CC010831CC01080B
:10D17000B4DF01083DCC010846CC010858C60108BF
:10D1800055CC010861CC010831D401086FCC0108ED
:10D190007CCC01088FCC01089DCC0108A7CC0108EC
:10D1A000B6CC0108C4CC0108D0CC0108E1CC010800
:10D1B000F3CC010810B5204A18B9136802221A826C
:10D1C00010BD1E481468002303802178024611F028
:10D1D0007F010DD1637A990644BF0221017013F0DB
:10D1E000400F037814BF43F0010323F0010314E060
:10D1F000012920D002291DD1617901F00F039B0084
:10D2000003F1804303F5B84311F0800F1B6806D08B
:10D2100003F03003102B07D10123137004E003F453
:10D220004053B3F5805FF6E7054B1B681B699847D1
:10D23000024810BD184610BD0C250020D01C00204F
:10D24000B81F002010B5064C18B9236801221A82B5
:10D2500010BD044B1B689B68984720680C3010BDBC
:10D260000C250020B81F002010B5064C18B9236803
:10D2700001221A8210BD044B1B681B689847206866
:10D280000A3010BD0C250020B81F0020084BDA68BA
:10D29000D10709D4DA68520708D4DB6813F0100FFD
:10D2A00014BF0320042070470120704702207047FC
:10D2B0000020024003788B4283BF034B03EB410104
:10D2C00048880020704700BFD01C002070B505467C
:10D2D00000F0FCFD324CE369E061C31AB3F5FA5F7C
:10D2E000236282BF002384F8243084F8253094F828
:10D2F00024302BB9A12D02BF294A012182F8251023
:10D3000094F82510264A31B1D118EDB2013381F8D5
:10D31000265082F8243094F8245094F84730AB42D9
:10D320003CD11F4B93F84830052B02D0062B03D07D
:10D330002FE0002006F0B8F994F827301E2B28D1F2
:10D3400000200246C1B26B1E99421ADA214491F8BC
:10D3500026300821DBB283EA0206F60744BF83F0D9
:10D360001803C3F3460301F1FF3154BF5B0843F0D8
:10D37000800311F0FF01C2F34702ECD101301A46DD
:10D38000E0E7234493F826309A4202D1032006F0C6
:10D390008BF9002384F8253084F8243070BD00BF59
:10D3A000D01C00202DE9F843324F3D682A8A2E7A9E
:10D3B000B2B9042E14D1304C30482378012B0BD154
:10D3C0002F4B19682F4B89B20B445B0019681A6008
:10D3D00030230380227048E010230380072644E0B6
:10D3E000AC8AAB69A24294BF04260226944228BFAD
:10D3F00014461FFA84F840469847214A04F1010E6A
:10D4000013684FEA6E0E9BB203F1005303F54053CD
:10D410005B001B6800219BB203F1005303F54053EE
:10D420005B00714500F1020009D010F8019C10F872
:10D4300002CC4CEA092C23F821C00131F1E7126833
:10D44000104B92B213445B001A681C602B8A302286
:10D45000C8EB03032B826B8A9844084BA5F8128013
:10D460001A80094B4FF440521A803B681E72BDE887
:10D47000F88300BF0C250020A5300020B21F00203B
:10D48000505C004002300020B01F00200E4B0F4ABD
:10D490001B683E299BB203EBC00002444FEA4202E4
:10D4A00009D94B09C80604BF03F1FF339BB29B02A5
:10D4B00043F4004304E04B08C90748BF01339B0213
:10D4C00011681360704700BF505C004006300020B8
:10D4D0008A6810B50C6A036814430A6923F4FF4391
:10D4E00014434A6923F0700314438A691443CA69D8
:10D4F00014434A6A14438A6A224313430360CB6885
:10D5000043600B6883604B68C36010BD4FF6FE73C9
:10D510000268134003600023036043608360C360BC
:10D52000284B984201D1284A27E0284B984201D144
:10D53000254A2AE0264B984201D1234A2DE0254B6B
:10D54000984201D1204A30E0234B984201D11E4A33
:10D5500033E0224B984204D11B4A536843F47003D2
:10D560002EE01F4B984204D1174A536843F0706372
:10D5700026E01C4B984204D11B4A536843F00F032A
:10D580001EE01A4B984204D1174A536843F0F00347
:10D5900016E0174B984204D1134A536843F4706362
:10D5A0000EE0144B984204D10F4A536843F4704381
:10D5B00006E0114B984204D10B4A536843F47023A0
:10D5C0005360704708000240000002401C00024007
:10D5D0003000024044000240580002406C0002400B
:10D5E0008000024008040240000402401C04024083
:10D5F0003004024044040240580402401F4A10B55F
:10D60000536803F00C03042B03D0082B04D01C4BED
:10D6100014E01C4B1B6811E053685168C3F383434B
:10D62000C90303F1020301D4174906E0516811F45C
:10D63000003F1449096818BF49084B430360536809
:10D640001249C3F30313CC5C0368E340436054689E
:10D65000C4F302240C5D23FA04F484605468C4F318
:10D66000C2240C5DE340C3605268C2F381320A44B5
:10D67000127CB3FBF2F3036110BD00BF0010024047
:10D6800000127A004800002000093D00FCAE0108AD
:10D6900010B50446FFF7FAFD012806D11CB1FFF7CB
:10D6A000F5FD013CF8E7052010BD002C08BF052062
:10D6B00010BD0A88F0B54B888E88B1F808E0CC8898
:10D6C000002A3AD1028C43F0010322F00102120435
:10D6D000120C0284058B078CADB225F0F30545EAE8
:10D6E0000E1189B241EA06027A49BFB2884212D0CD
:10D6F00001F5006188420ED0B0F1804F0BD0A1F54A
:10D700009831884207D001F58061884203D001F545
:10D710008061884202D127F0020701E027F00A0762
:10D720001F4302830784038B23F00C031B041B0C91
:10D730000383038B9BB21C4344E0042A44D1028C34
:10D7400022F010021204120C0284018B058C21F4C9
:10D7500040721205120D42EA0E325E4992B242EA5E
:10D7600006228842ADB292B212D001F50061884221
:10D770000ED0B0F1804F0BD0A1F59831884207D080
:10D7800001F58061884203D001F58061884207D1AC
:10D7900025F0200141EA03139BB243F0100304E09B
:10D7A00025F0A00143F010030B4302830384038B95
:10D7B00023F440631B041B0C0383038B9BB243EADB
:10D7C0000424A4B20483F0BD082A028C3ED122F4C2
:10D7D00080721204120C0284828B3E4D92B222F0AF
:10D7E000F307018C47EA0E1292B2A84289B242EACC
:10D7F000060212D005F50065A8420ED0B0F1804FA8
:10D800000BD0A5F59835A84207D005F58065A8424C
:10D8100003D005F58065A84207D121F4007141EAE3
:10D8200003239BB243F4807304E021F4206143F4AA
:10D8300080730B4382830384838B23F00C031B04CC
:10D840001B0C8383838B9BB21C4341E022F48052E8
:10D850001204120C0284858B018C25F440752D0571
:10D860002D0D45EA062545EA0E321A4D89B2A84229
:10D8700092B212D005F50065A8420ED0B0F1804FEB
:10D880000BD0A5F59835A84207D005F58065A842CC
:10D8900003D005F58065A84207D121F4005141EA83
:10D8A00003339BB243F4805305E047F6FF5543F43E
:10D8B00080530D402B4382830384838B23F4406386
:10D8C0001B041B0C8383838B9BB243EA0424A4B206
:10D8D0008483F0BD002C0140CA78F0B5D40648BF5F
:10D8E0008C780D8802F00F0348BF234315F0FF0F1B
:10D8F0001DD0016800240126A64006EA0507B742AC
:10D9000011D14FEA840E0F2606FA0EF621EA06011F
:10D91000282A03FA0EF641EA060101D1476102E026
:10D92000482A08BF07610134082CE4D10160FF2DAB
:10D930001FD94168002404F108070126BE4006EA09
:10D940000507B74211D14FEA840E0F2606FA0EF6EC
:10D9500021EA0601282A03FA0EF641EA060101D15E
:10D96000476102E0482A08BF07610134082CE2D170
:10D970004160F0BD0F4B1A6842F001021A6059680D
:10D980000D4A0A405A601A6822F0847222F48032EA
:10D990001A601A6822F480221A605A6822F4FE0281
:10D9A0005A604FF41F029A60044B4FF000629A6075
:10D9B000704700BF001002400000FFF800ED00E0DB
:10D9C0002DE9F843564C0368013AC4F84A3083887D
:10D9D0000D46A4F84E30072A42D8DFE802F0040AC8
:10D9E000101822292F35B4F84A300B80B4F84C3087
:10D9F00013E0B4F84C300B80B4F84A3005E0B4F8CA
:10DA00004A305B420B80B4F84C305B4205E0B4F81E
:10DA10004C305B420B80B4F84A306B80B4F84E3027
:10DA20001DE0B4F84A305B420B80B4F84C3012E091
:10DA3000B4F84C300B80B4F84A300CE0B4F84A30FB
:10DA40000B80B4F84C3005E0B4F84C305B420B80EE
:10DA5000B4F84A305B426B80B4F84E305B42AB8026
:10DA6000304B1B79002B59D1B5F9000006F07EF937
:10DA70008046B5F9020006F079F90746B5F90400C9
:10DA800006F074F9216D0646404606F0C3F9E16DD3
:10DA90008146384606F0BEF90146484606F0B2F81F
:10DAA000A16E8146304606F0B5F90146484606F0BB
:10DAB000A9F80AF049F9616D2880404606F0AAF9F4
:10DAC000216E8146384606F0A5F90146484606F023
:10DAD00099F8E16E8146304606F09CF901464846C9
:10DAE00006F090F80AF030F9A16D6880404606F023
:10DAF00091F9616E8046384606F08CF90146404641
:10DB000006F080F8216F0746304606F083F901469B
:10DB1000384606F077F80AF017F9A880BDE8F883D0
:10DB2000D01C00204800002038B50F4B1B689C8992
:10DB30000E4B186880F31000201A06F017F90C49F4
:10DB400006F068F90546204606F010F90146284619
:10DB500006F014FA06F024FB6428A8BF642020EA2B
:10DB6000E070C0B238BD00BF0C1100201C110020B5
:10DB70000000C84244F6FB71084B1A68137803EBA7
:10DB8000431300FB03135078C0EB0030B3FBF0F3FA
:10DB90009078B3FBF0F080B2704700BF0C1100200A
:10DBA00008B50A480A2290F8753000EB4303B3F831
:10DBB0008410903089B220F8041C00F05DFA80B225
:10DBC000FFF7D8FF024B188008BD00BFD01C002013
:10DBD00010110020034B4FF4004208B11A61704746
:10DBE0005A61704700080140034B4FF4004208B1EE
:10DBF0005A6170471A617047000801402DE9F74FDC
:10DC00002F4C054627683846FAF71EFB064638466D
:10DC1000FAF7A7FA676881463846FAF715FB0190CC
:10DC20003846FAF79EFAD5F804A007463146504622
:10DC300006F0F0F8D5F8088083464946404606F0DD
:10DC4000E9F80146584605F0DBFF019B2968834649
:10DC5000184606F0DFF849460546504606F0DAF861
:10DC6000394606F0D7F80146284605F0CBFF39467D
:10DC70000546404606F0CEF8314606F0CBF80146A0
:10DC8000284605F0BFFF014658460AF035F90D4910
:10DC900006F0C0F80C4906F071F9A16805F0B2FF72
:10DCA0000A4906F06BF90AF04FF883B21A0444BF30
:10DCB00000F5B47083B218B203B0BDE8F08F00BFB6
:10DCC000E81D00200000E144DB0F49400000204136
:10DCD00010B5084B0022196801EBC20393F902400A
:10DCE000844201D1981C10BD0132042AF4D10020D5
:10DCF00010BD00BF0C26002038B1438811EA030094
:10DD000003D08B420CBF01200220704730B50A4B74
:10DD10000A491C680A7B032A0AD81346551C04EBDF
:10DD2000C303EAB29D882842F5D00A73981C30BD1F
:10DD30000A73002030BD00BF0C260020E81D002023
:10DD4000014B00221A73E1E7E81D00202DE9F0479E
:10DD5000877890F803C0BBB2C7F1640E03EB83066B
:10DD60005C42C3F178001C4D5FFA8EFE7600CCF168
:10DD70006408A4B280B2A3B20FFA83F9B9F1000F1C
:10DD800004DC002B14BF3B46012300E0734609FB73
:10DD900009F25B4302FB0CF292FBF3F3434403FBF7
:10DDA00009F30A2293FBF2F333449BB225F8023FB6
:10DDB000B1F800904A880A34C9EB020A1AB202FB91
:10DDC0000AF24FF47A7392FBF3F3A4B24B44844209
:10DDD0002B80D0D1BDE8F087F41D002010B5447829
:10DDE0000078002240F6C41102FB02F3193B6343A2
:10DDF00003F6C4135343434393FBF1F3034921F860
:10DE000012300132072AEDD110BD00BF0E1E0020D6
:10DE1000104B043033F91000B0F5617F05DB40F69C
:10DE200033039842A8BF184601E04FF461700A78A6
:10DE300019235A4302F28332824208DA4A78534362
:10DE400003F283338342B4BF0020012070470020D7
:10DE5000704700BF8C26002010B500F150030278F7
:10DE60008A4203D18478C278944204D30430984221
:10DE7000F5D1002010BD012010BD1FB5084B1B6857
:10DE80001B0309D58DF80400039101230D2001A97E
:10DE90008DF80530FBF768FB05B05DF804FB00BFAB
:10DEA000502600201FB5084B1B681B0309D58DF8B1
:10DEB0000400029100230D2001A98DF80530FBF725
:10DEC00053FB05B05DF804FB5026002010B5094A4D
:10DED000094B11689B6812689142F8D1074A4FF4C8
:10DEE0007A70546B00FB04F2D31AB3FBF4F300FB1B
:10DEF000013010BD7426002010E000E0E81D002075
:10DF000038B50446FFF7E2FF0546FFF7DFFF401B89
:10DF1000A042FAD338BD10B504462CB14FF47A7044
:10DF2000FFF7EEFF013CF8E710BD024A136801332A
:10DF30001360704774260020024B9B6B03B1184797
:10DF4000704700BFE81D0020014B1B68184700BF49
:10DF50008430002010B50020FFF7F6FF064B0024A8
:10DF60001C7005F0B9FC054B83F83C401C64A3F819
:10DF700044409C6410BD00BF6E300020E81D0020AE
:10DF800010B510B9BDE81040E4E700230C225A4355
:10DF90000A4C1119125D824203D00133102BF5D1C6
:10DFA00010BD074B986C18B14A784078824204D271
:10DFB00000229964A3F844201A6410BD18B2010825
:10DFC000E81D002010B540001428A8BF142000232D
:10DFD000074A022199540B4499181424834201F8EA
:10DFE000014CF5DBFF21D1540F20BDE81040C7E7FD
:10DFF0005020002038B540F2DB156843104B082252
:10E000001A61851E0B24013C14F0FF0411D00C4A48
:10E010002846D36883F00803D360FFF77CFF012014
:10E02000FFF792FF1920FFF776FF0020FFF78CFF24
:10E03000E9E7044A044B1A60044A054BDA6038BD2C
:10E04000000C0140EFBEADDEF04F00200400FA05E9
:10E0500000ED00E003685B69184703681B69184717
:10E060000368DB68184703689B68184703685B68A8
:10E07000184703681B681847B0F902302DE9F74FBD
:10E0800093421CBF0023037090F800A004460E4684
:10E090009146BAF1000F40F0AB80104605F066FEE5
:10E0A000864905F0B7FE864905F0B4FE4FF07C5175
:10E0B00005F0B0FE09F0A8FE0146054605F0AAFEEF
:10E0C00080498346284605F0A5FE03465846194672
:10E0D000019305F097FD4FF07E5105F093FD014649
:10E0E0004FF07E5005F04AFF2946804605F092FE2B
:10E0F000294605F08FFE07460146606005F082FD67
:10E10000E7604FF07E572946A0602761284605F05A
:10E1100079FD294605F07EFE4FF0804105F070FD47
:10E120000146404605F076FE019B6061194658465F
:10E1300005F066FD394605F065FD0146404605F0EF
:10E1400069FE40F2DC53A04627465546636510231E
:10E15000A4F852301823A061A4F850304FF0974132
:10E16000D8F8100005F056FE0021824605F0F0FFB9
:10E1700028B150464FF07C5105F042FD04E0504676
:10E180004FF07C5105F03EFD06F06CF8C7E90E013A
:10E190004FF09741D8F8040005F03CFE002182467C
:10E1A00005F0D6FF28B150464FF07C5105F028FD10
:10E1B00004E050464FF07C5105F024FD06F052F883
:10E1C0000135032DC7E9080108F1040807F1080724
:10E1D000C4D1A6F2DC531B042367E3676367C4F86A
:10E1E0008030A367C4F884300123A4F80290237020
:10E1F000D4F85490B4F95280C9EB0606636A06FA63
:10E2000008F67343276A4FEAE67B206F07FB0B3360
:10E210002667A7FB0667E26F1F44636CD4F840C013
:10E2200053434FEAE27B0CFB0B3ED4F88010C4F85A
:10E230008020ACFB02237344B61A67EB0307E36A42
:10E24000A26A43434FEAE07B02FB0B3EA2FB0023A2
:10E250007344B6185F41E36C656F4B436067A06C15
:10E260004FEAE17B00FB0B33C4F88410A0FB0101F3
:10E270001944636B361A05FB03F3206B4FEAE57B09
:10E2800000FB0B3367EB0107A0FB05018019194464
:10E290007941B4F95020A56705F0A0FC08F1FF32E0
:10E2A00001239340E067C01841EBE371424605F05B
:10E2B00095FC484403B0BDE8F08F00BF6F12833A6D
:10E2C000DB0F4940F404B53F2DE9F0410024234B16
:10E2D000E0B21E78B0420CD2214B33F81010214B23
:10E2E00053F820301BB10B2801D8DB689847013464
:10E2F000EDE71D4B1B685B032DD500242346E2B2DE
:10E30000B24228D2174F4FEA840857F824205568A4
:10E310009D4218D02846FDF70BFFEFF312835022E1
:10E3200082F3128811494FF0280EAA8C0EFB0010C0
:10E3300092B201320267AA8ADBB292B242F00102C3
:10E34000AA8283F3118857F8083000221B68013431
:10E350001A802B46D3E7BDE8F08100BF00200020E3
:10E36000601000200420002050260020E81D00201E
:10E3700008B50E4B1B6813F4805F0D4B14BFD3F828
:10E38000EC30D3F8F0309A880A4B19780023D8B2D1
:10E39000884204D2084820F813200133F7E7FFF73A
:10E3A00093FFBDE808403220B5E500BF50260020AD
:10E3B000E81D002000200020601000200A4B30B52E
:10E3C0001A680A4B02F48052D3F8EC40D3F8F050AC
:10E3D00000230AB1A18800E0A988054820F813109D
:10E3E00001330C2BF5D130BD50260020E81D002054
:10E3F000E21F002070B5124D0024214605F1F50002
:10E40000702285F8F44009F092FA2146D5F8683177
:10E410000B4A0B4493F9020088B11E6802F1F5041F
:10E420000E5108199C88073184809B79702983716B
:10E4300092F8F43003F1010382F8F430E6D170BDB4
:10E44000E81D0020094B1A680E2303FB0020437AC5
:10E45000FF2B07D0064A12789A4203D9054A32F8B0
:10E46000130000E0808800B2704700BFCC1C002081
:10E47000083000208C2600202DE9F04F91B0FFF7E6
:10E4800025FD8C4C0546D4F86C614FF00008831BC9
:10E490001846019305F066FCD4F87011029005F05F
:10E4A000B9FCC4F86C514546D4F87471824E97F8A3
:10E4B00000B00390814A0DF11C0A32F9150005F0F5
:10E4C00055FC039905F0A6FC4AF82500BBF1000FA6
:10E4D0002BD0584605F04AFC01464FF07E5005F01F
:10E4E0004DFD0246DFF8009211464FF07E50059236
:10E4F00005F086FB59F8251005F08CFC09F10C019C
:10E50000049031F9150005F031FC059A114605F02B
:10E5100081FCDDF810C00146604605F073FB49F848
:10E52000250005F03DFE708003E0654A32F81520B5
:10E53000728036F9022F0135032D02FB0288B9D112
:10E54000642303FB08F85F4B5F481B8807A95B4304
:10E5500098FBF3F8A8F149081FFA88F8F9F7F2FEDA
:10E56000B8F13B0F7D6810D9524BB3F99801D3F83D
:10E57000945105F0FBFB0146284605F007FE534B7E
:10E5800068B31A7842F008022CE04FF07E5128461A
:10E5900005F038FB01464FF07E5005F0EFFC814658
:10E5A0004FF00008DFF820B128465BF8281005F08E
:10E5B00031FC474A039032F9180005F0D7FB039B62
:10E5C0000146184605F01EFB494605F023FC4BF8B2
:10E5D000280008F10108B8F1030FE3D1C4E71A7865
:10E5E00022F008022946D4F890011A7009F084FC40
:10E5F00081462060D4F88C01D4F894B100F1004534
:10E60000D4F89001014605F005FC5946804658466D
:10E6100005F000FC0146404605F0F4FA09F0F8FD6B
:10E620000146284609F068FC2A4980466060484651
:10E6300005F0F0FB09F088FB274D2649288040466D
:10E6400005F0E8FB09F080FB244B68801B681B0782
:10E650004CD5234807A9F9F775FEBD684FF07E51E8
:10E66000284605F0CFFA01464FF07E5005F086FCB3
:10E6700082464FF0000B1A4B284653F82B10049398
:10E6800005F0C8FB1749039031F91B0005F06EFB3C
:10E69000039A0146104605F0B5FA514605F0BAFB5B
:10E6A000049B43F82B000BF1010BBBF1030FE2D1EC
:10E6B000184652E0E81D0020EC1000204010002019
:10E6C0006C1F00201C000020741F0020241100205B
:10E6D000EE1000204C3D0F44462600202011002063
:10E6E000841F002046100020601F00206C4D514602
:10E6F0002846F9F727FE28686B680146039305F062
:10E7000089FB039B82461946184605F083FB0146A8
:10E71000504605F077FAD5F808B082465946584673
:10E7200005F078FB0146504605F06CFA09F070FDE3
:10E730000021824605F002FD70B92868514605F0B7
:10E740001DFC51462860686805F018FC5146686059
:10E75000A86805F013FCA8605148FFF74FFA514B29
:10E7600051491880029805F055FB4E4B08F10048BE
:10E77000054609F10049B3F90000CDF82C80CDF829
:10E78000289005F0F3FA494900F1004005F042FBFA
:10E79000DFF82C810C90B8F9000005F0E7FA0D9035
:10E7A000B8F9020005F0E2FA0E90B8F9040005F09D
:10E7B000DDFA0AA90F900DA8F9F7C4FD7B78012BAB
:10E7C0001AD13B4B3B4F1B7813F0040F0ED1D7F8F7
:10E7D000A801402390FBF3F3C01A05F0C7FA0F9984
:10E7E00005F010FA05F0DCFCC7F8A801D7F8A8017D
:10E7F000402390FBF3F001E02F4B188805F0B6FAA8
:10E8000001460F9805F0FCF9D4F8B0110F90284696
:10E8100005F0F8F90146284605F0B0FBD4F8AC71D4
:10E82000054639460F9805F0EBF90146284605F0F4
:10E83000F1FA0146384605F0E5F90746C4F8AC019F
:10E840000D9809F081FAD4F8B4512978F9F77AFCD7
:10E85000D4F8B8311844C4F8B8010E9809F074FA25
:10E860002978F9F76FFCD4F8BC311844C4F8BC011E
:10E87000384609F069FA6978F9F764FCD4F8C031D0
:10E880000E4A184401991368C4F8C0011944D4F819
:10E89000C43111600133C4F8C43111B0BDE8F08F48
:10E8A00050000020FC100020BD37863535FA8E3C24
:10E8B000A3300020E81D00201C0000208030002034
:10E8C000EE10002001380A4B042804D8DFE800F0DD
:10E8D0000507090B0D00074A08E0074A06E0074A4A
:10E8E00004E0074A02E0074A00E0074A1A6070475E
:10E8F000FC00002099230108C99D0008B5260108E5
:10E900002DA4000889A0000859A70008704708B581
:10E910000B4B002093F82C10FEF7B8FD094B1B6839
:10E92000187A082801BF084B4FF480521A80102231
:10E9300008BF5A80A0F109035842584108BD00BFE2
:10E94000C80000200C250020B01F00207047704731
:10E950007047FEE7FEE7FEE7704730B50024E3B2FC
:10E9600093420DD2030F092B94BF3033373301F894
:10E970001430002501EB440300015D700134EEE723
:10E9800030BD30B5002240F60F7102F1805303F51F
:10E99000B8539B001D6842F4004444F080042940B1
:10E9A00001322143042A1960EDD1024B40F080006E
:10E9B000186030BD4C5C00402DE9F347884D894C10
:10E9C0002B68894E9BB2A380A28831880A409705A4
:10E9D00007D54FF6FF53854A2B6013780133DBB21E
:10E9E0001370A3880B40180440F100830023ADF896
:10E9F00002302B687B4F9AB21804A28040F1F68255
:10EA0000BB8803F00F03BB71002B40F0C182784A32
:10EA100013689BB23B803B8803F030037B803B88CC
:10EA200003F440533B804BF6BF7311680B4083F4F3
:10EA3000005383F0200343F4004343F0800313604A
:10EA4000BB88D90621D448F60F7311680B40694979
:10EA500013600B6888461A7A022A01D0042A02D170
:10EA6000FEF7A0FC59E2062A40F06B825A78052A8C
:10EA700008D11A78520605D1D878FFF782FFBB6813
:10EA80001B6A9847E3689B685AE213689BB2ADF82B
:10EA90000230BDF802301F0540F1CF8140F68F7380
:10EAA0001168544F0B40544913600A68534B92B29B
:10EAB00013445B001A683B688846187A092817D007
:10EAC00092B2520002F1804202F5C04211781970F0
:10EAD000517859709188C8B2090A41EA00215980D9
:10EAE0001189C8B2090A41EA002199809289DA8025
:10EAF00001221A72DA8893F80190002A40F0DC8033
:10EB00001A7812F07F024AD1B9F1090F0FD1DA78E1
:10EB1000012A00F2B8809978002940F0B4809988E1
:10EB2000002940F0B0809A72A3685B68A9E0B9F14F
:10EB3000050F10D193F90320002A01DA0823B9E068
:10EB40009A78002AFAD19A88002AF7D19B7A002B6A
:10EB500000F0A280F2E7B9F1030F0ED1DA78012AB2
:10EB600040F091809A88002A40F08D805A7A42F0D5
:10EB700020025A72A368DB6983E0B9F1010F40F00B
:10EB80008280DA78012A7ED19A88002A7BD15B7A4A
:10EB9000980678D508F01EFE00287DD073E0012A83
:10EBA0002ED1B9F10B0F6ED1E26858799269D978FC
:10EBB00090473B689A7A002A65D0002863D11A7979
:10EBC000002A60D19B78002B5DD1064B9B68DB68E7
:10EBD0009847084B1B685A79DA72DA781A735BE047
:10EBE000445C0040B01F002074300020A63000209C
:10EBF000005C00400C250020505C004004300020E8
:10EC0000022A40D1B9F1010FC4D0B9F1030F3AD1B2
:10EC1000587920F0800E4FEA8E0202F1804101F512
:10EC2000B841096810F0800F14BF01F0300101F401
:10EC30004051BEF1030F26D8B3F802E0BEF1000F39
:10EC400021D101B39B7AF3B102F1804202F5B842BF
:10EC5000136801064BBF23F4E04323F4804323F001
:10EC6000400323F070034BBF9BB29BB283F01003B1
:10EC700083F4805343F4004343F080031360A3689C
:10EC80009B69984708E0E36848465B699847032812
:10EC90000FD000287FF452AFD8F80020A14B92B2D9
:10ECA00013445B001A6800221A6030236380062335
:10ECB00000E009233A6847E1B9F1060F12D11A784A
:10ECC000520677D19B78012B02D1E368DB6966E0BD
:10ECD000022B02D1E3681B6A61E0032B6AD1E3686F
:10ECE0005B6A5CE0B9F1000F37D15988002961D126
:10ECF0005A6822F47F42B2F5003F5BD11A7812F0D5
:10ED00007F0204D19B88002B00F0D58152E0012ABC
:10ED100008D1E26858799269904700284AD13B6847
:10ED20009B7A16E0022A45D15A7902F00F018B0036
:10ED300003F1804303F5B8431B6812F0800F14BF42
:10ED400003F0300303F44053032933D812F0700F5B
:10ED500030D1002B40F0AF812CE0B9F1080F04D185
:10ED60001B785B0600F0A98124E0B9F10A0F21D1DC
:10ED70001A7802F07F02012A1CD19A7AD2B15988FE
:10ED8000C1B95A6822F47F42B2F5803F12D1E268DD
:10ED9000587992699047002800F091810AE04BB1C0
:10EDA0003A684FF00008A2F81280936140469847F5
:10EDB00040460BE0E3683A681B695078984703289F
:10EDC00004D1594B09221B681A72BEE04FF6FF713D
:10EDD0003A68138A8B4201D10923B5E0022800D09A
:10EDE0000BB90823B0E092F9001000291FDAD1888E
:10EDF00001910198834202D9019B138210E08B425A
:10EE00000ED2E16891F82C00834201D2002105E086
:10EE100093FBF0F100FB113313B90121434B19703F
:10EE2000E36893F82C309382FEF7BCFA8DE003235D
:10EE300013724FF44053238087E0BDF802301BB2B9
:10EE4000002BBFF6D6AD40F68F7311680B401360F0
:10EE5000354A176890463B7A022B72D0042B70D04B
:10EE6000032B01D0052B67D1BB693A8A8BB9398A4C
:10EE700000293BD04FF4405323802D4B1A68294B77
:10EE800092B213445B001A6800221A603023638038
:10EE90002CE0002AEBD0B7F81490914528BF91469A
:10EEA0001FFA89FA504698473B8A4FF0000ECAEB8A
:10EEB00003033B827B8A53447B821D4B1A681D4BA4
:10EEC00092B213445B001B6809F101029BB203F18B
:10EED000005303F5405352105B009645C7D053F8DA
:10EEE0002E1020F81E100EF1010EF6E7BB8A8B42A1
:10EEF000D8F8003001D8032201E011B105221A72BE
:10EF00000BE006221A720A4B1A68064B92B213449F
:10EF10005B001A68196030236380D8F800301B7AD0
:10EF200010E000BF023000200C250020A53000209A
:10EF3000505C004004300020072B02D1E368DB68FE
:10EF400098470823D8F800201372FFF7E0FC5E4BC7
:10EF50001A684BF6BF7313402288D704228848BF33
:10EF600083F480539004628848BF83F40053D10631
:10EF7000628848BF83F01003920648BF83F02003E5
:10EF800043F4004343F080034F4A9BB213602DE0EB
:10EF90009A0002F1804202F5B842116889B2ADF8D8
:10EFA0000210BDF8021009B2002909DA40F68F718B
:10EFB0001068013B01401160444A52F823309847E1
:10EFC000BDF802301F067FF514AD48F60F72A17927
:10EFD0008B0003F1804303F5B843186802401A60C0
:10EFE0003A4B03EB81039B69984702E5A28833887B
:10EFF0001340590505D54FF6FF332B60344B5B6842
:10F000009847A28831880A40920444BF4DF6FF73A6
:10F010002B60A3882F4A0B40DB0452D54EF6FF73BA
:10F020002B6000231374137C052B41D8DFE803F019
:10F03000030D1418222D6369264D1BB903F05CFFE4
:10F04000062300E005232B743BE003F055FF042367
:10F0500023740123636134E002236374032328E0F3
:10F06000637C013BDBB26374637C53BB194B0422AA
:10F070001A7426E0184A13689BB243F01003136019
:10F08000052323740A2363741BE0637C114A013B4C
:10F09000DBB26374637C03F0FF0093B94FF6EF7348
:10F0A0000D490C6823400B6006231374506108E07F
:10F0B0000623237405E0094B72E6094B70E6094B01
:10F0C0006EE602B0BDE8F087005C004010AF0108BA
:10F0D000C8000020B01F0020405C0040B5D10008EF
:10F0E00069D2000845D2000837B50622044603213C
:10F0F0006B461E20F5F7FEFF9DF801309DF80000DD
:10F10000154D43EA002000B204F030FE296804F0F7
:10F1100081FE05F045F89DF8033020809DF802003F
:10F1200043EA002000B204F021FEA96804F072FE58
:10F1300005F036F89DF80530A0809DF8040043EAFC
:10F14000002000B204F012FE696804F063FE05F0CE
:10F1500027F8608003B030BD5C0000202DE9F04747
:10F16000664D2B686649581C0A788E4602F0FF06E9
:10F170000AB10346F6E737462B60687BAB6895F823
:10F180000C80AA7B39B2202900F09C80DFF880C176
:10F190000CEB8103DC789B783CF82110C3F1FF0372
:10F1A0009BB2002B65D04FF03C0CB1FBFCF9C3F1D6
:10F1B000FF0363431B12B9F1050F5DD8DFE809F0C7
:10F1C000030B1A293A4AE01A4143B1FBFCF0DAB2C8
:10F1D0001044C0B251E0B1FBFCF00CFB101189B23D
:10F1E000DAB2C1F13C01E31A4B43B3FBFCFC20460D
:10F1F00094442CE0B1FBFCF00CFB1011E21A89B234
:10F200004A43B2FBFCF25FFA83F84244D2B2204692
:10F2100032E0B1FBFCF90CFB191189B2E01AC1F123
:10F220003C014843B0FBFCF05FFA83F84044C0B2B5
:10F23000224621E0B1FBFCF80CFB1811D8B289B2D0
:10F24000E31A01FB03F2B2FBFCFC224684445FFAA2
:10F250008CF412E0B1FBFCF80CFB181189B2D8B2A7
:10F26000C1F13C01E31A4B43B3FBFCF20244D2B2BE
:10F2700003E02246204600E044464FEA042C4CEAD4
:10F28000004C4CEA020C17234FF0010808FA03F86F
:10F2900006F1170118EA0C0FA1EB0301DFF87480E7
:10F2A00014BF4FF011094FF0090989B213F1FF3370
:10F2B00008F80190E8D218360137B6B2BFB2114B48
:10F2C000A0465FE7AB6001238EF8003040F22A339E
:10F2D000AA730D4AE9800D4985F80C806873AE80E9
:10F2E000536000238B840B889BB243F001030B8097
:10F2F000136843F001031360BDE8F087C81F0020C6
:10F30000A2300020D41F00206C0002400004004006
:10F31000FA0D002085030020F0B5B1F800E00023CD
:10F320004EFA03F2D50725D58E784FEAD30CF406B2
:10F3300048BFCC7806F00F0203F0070748BF22430E
:10F34000BF0050F82C500F24BC4025EA0404BA40FA
:10F350002243282E40F82C2005D1C46801229A406F
:10F3600024EA020205E0482E04D1C46801229A4032
:10F370002243C2600133102BD2D1F0BD2DE9FF41F1
:10F380005B4B1B689BB11A681AB15A4988690243E2
:10F390008A619A889868ADF8042002228DF80720C7
:10F3A00004220DEB02018DF80620FFF7B5FF322095
:10F3B000FEF7B1FD002111221E20F5F75BFF0121B0
:10F3C00060221E20F5F756FF6420FEF7A4FD0024FE
:10F3D00002A8FFF789FE274626460A2502210122B8
:10F3E0001E20F5F747FF3220FEF795FD02A8FFF734
:10F3F0007BFEBDF90820BDF90A1014448A42A8BF5B
:10F400000A46BDF90C300F4493421E44A8BF134670
:10F4100013F5805F04DD013DE0D14FF0010801E00C
:10F420004FF000081E2000211222F5F723FF0A25C5
:10F43000022101221E20F5F71DFF3220FEF76BFD91
:10F4400002A8FFF751FEBDF90820BDF90A10A41A61
:10F450008A42A8BF0A46BDF90C307F1A9342A6EB38
:10F460000306A8BF134613F5805F02DD013DDFD11F
:10F4700001E04FF00008204604F078FC01461E48E9
:10F4800004F07CFD1D4D20F000402860384604F05B
:10F490006DFC0146184804F071FD20F000406860E2
:10F4A000304604F063FC0146154804F067FD20F087
:10F4B0000040A860002170221E20F5F7DBFE01212C
:10F4C00020221E20F5F7D6FE1E2002210022F5F78D
:10F4D000D1FE6420FEF71FFDB8F1000F04D14FF0FC
:10F4E0007E532B606B60AB6004B0BDE8F08100BF61
:10F4F000640300200010024000406F465C000020C2
:10F5000001C05E46104B73B518781C46A0B10523A8
:10F510000E4D8DF800304FF4805600238DF80130E9
:10F520000B486E6101A96A460223F5F70BFF2E61B5
:10F530009DF8050000F0010000F00100207080F04F
:10F54000010002B070BD00BFD9060020000C0140D0
:10F5500000380040064B70B506461C461D68FFF794
:10F56000D1FF18B923685B1BB342F8D970BD00BF47
:10F5700074260020F7B503238DF80430030C8DF8B2
:10F5800005308DF80700030A06200F4614468DF853
:10F590000630FFF7DFFF88B1094D4FF48056002198
:10F5A00001AA04236E610748F5F7CCFE05483946E9
:10F5B00000222346F5F7C6FE20462E6103B0F0BDBB
:10F5C000000C014000380040024640213C20F5F785
:10F5D00051BE70B500EB8000094CA0F1A1059C382C
:10F5E00025440444074B15F8010F1E787040FFF7BF
:10F5F000EBFFA542F6D13046BDE87040E4E700BF1E
:10F600004CAF0108A730002010B5441E14F8010FBC
:10F6100010B1FFF7DEFFF9E710BD024680213C2064
:10F62000F5F728BE10B5D420FFF7F7FF8020FFF7CD
:10F63000F4FFA820FFF7F1FF3F20FFF7EEFFD320F4
:10F64000FFF7EBFF0020FFF7E8FF4020FFF7E5FFA3
:10F650008D20FFF7E2FF1420FFF7DFFFA120FFF767
:10F66000DCFFC820FFF7D9FFDA20FFF7D6FF122012
:10F67000FFF7D3FF8120FFF7D0FFCF20FFF7CDFFAB
:10F68000D920FFF7CAFFF120FFF7C7FFDB20FFF704
:10F69000C4FF4020FFF7C1FFA420FFF7BEFFA62054
:10F6A000FFF7BBFFAF20FFF7B8FFA620FFF7B5FFBE
:10F6B000AE20FFF7B2FF2020FFF7AFFF0020FFF7DB
:10F6C000ACFFB020FFF7A9FF4020FFF7A6FF002006
:10F6D000FFF7A3FF1020FFF7A0FF4FF48064013C69
:10F6E0000020A4B2FFF770FF002CF8D18120FFF7B3
:10F6F00094FFC820FFF791FFAF20FFF78EFF012096
:10F7000010BD08B55038C0B2FFF787FF0020FFF7E3
:10F7100084FFBDE8084010207FE710B5044650394B
:10F72000C8B2FFF77AFF04EB4400400000F00E007F
:10F73000FFF773FF06206043BDE81040C0F30310DD
:10F7400010306AE7012828BF01202DE9F04F064656
:10F75000734F142000FB0671724BD1F8A4421E7542
:10F760001C61714BD1F8B422DD69B1F8AC822A4337
:10F77000DA61A288B1F8AEA222F44072D1F8A852A0
:10F78000120489B0120C4AEA0809A28003A9C5F83C
:10F79000109002228DF80E0028460193ADF80C90CF
:10F7A0008DF80F20FFF7B8FD019B00971F464FF023
:10F7B000080BAA6818EA020F03D10A20FEF7A0FB83
:10F7C000F7E70A20C5F81480FEF79AFBC5F8108009
:10F7D0000A20FEF795FBBBF1010BEAD1C5F814A096
:10F7E0000A20FEF78DFBC5F814800A20FEF788FB7F
:10F7F000C5F810800A20FEF783FB0222C5F810A08E
:10F80000284603A98DF80F201C228DF80E20ADF894
:10F810000C90FFF781FD454A03A894423A690BBF5B
:10F8200042F4001242F480023A613A610BBF3A6935
:10F830003A6922F4001222F480023A61A38823F488
:10F8400040731B041B0CA38023889BB243F001036D
:10F850002380A588FDF7D2FE0599354B25F03F059D
:10F86000B1FBF3F32D042D0C1D43ADB2A58022880E
:10F87000002522F001021204120C22802D4A03A856
:10F88000B1FBF2F100298AB208BF012242F4004123
:10F890004FF4967253434FF47A7293FBF2F30133B1
:10F8A0009BB22384A1832388009A9BB243F0010377
:10F8B0002380238823F4816323F002031B041B0CA1
:10F8C00023804FF480432381142303FB062696F8FC
:10F8D000B13201248DF80C308DF80D508DF80E509A
:10F8E0008DF80F4003F024FB96F8B0329DF80F20FE
:10F8F0008DF80C308DF80D508DF80E501AB103A80C
:10F9000003F016FB08E05A0903F01F039C4002F1C4
:10F910002003094A42F8234009B0BDE8F08F00BF38
:10F920004CAF0108C81F00200010024000540040E6
:10F9300040420F00804F120000E100E007B5064B87
:10F9400006490093064B074A01930748074BF8F70F
:10F95000D9FB03B05DF804FB88C3010878D2010825
:10F960005DC301087DD2010858D201087CC301089B
:10F9700008B5037833B90C4B0C481978BDE808403A
:10F98000F8F7C0BB08F06CF802280CD8064B0C2224
:10F990001870074B02FB0030064B0630186001F070
:10F9A00087FF0548E5E708BDE01F002084D2010875
:10F9B000502E00208410002058C6010808B5037896
:10F9C0003BB90B4B0B4893F8A417BDE80840F8F778
:10F9D00099BB08F045F8022808D8054B83F8A4071E
:10F9E000F8F756FDF8F7F6FD0348E8E708BD00BF55
:10F9F000B026002088D2010858C6010838B503781F
:10FA000003BB214B1B6801330F2B07D81F490C2266
:10FA100002FB031295681C462DBB00E01C46013416
:10FA20000F2C01DD002400E005D818490C2202FB50
:10FA300004129568BDB99C42F1D11548BDE8384023
:10FA4000F8F760BB08F00CF80F28044605D80F4AF9
:10FA50000C2303FB00239D682DB92146BDE83840E7
:10FA60000C48F8F74FBB084B1C60FEF773FA2146B1
:10FA70002A460948F8F746FB0C235C43034B185D04
:10FA8000BDE83840FEF77CBA6800002018B20108D3
:10FA900095D20108ABD20108C3D2010873B503782F
:10FAA00013B9F7F721FB3FE001AA204908F039F824
:10FAB00000240246264625469AB134B1012C08D1CD
:10FAC000104607F0CDFF064603E0104607F0C8FFDA
:10FAD000054601AA0020154908F023F80134024622
:10FAE000EAE70B2D03D9124812490C230CE0022C33
:10FAF00011D1A6F57A73B3F57A7F08D90C480E496F
:10FB00004FF47A724FF4FA63F8F7FCFA0CE00B4BFF
:10FB100003EB45035E80094B094803EB4503294687
:10FB2000B3F90220F8F7EEFA02B070BD6BCB010812
:10FB300071C8010890C8010818CF0108E01F002013
:10FB4000DAD2010838B50D4C05462368834206D148
:10FB5000F7F719FF204600214C2207F0E8FEE36C7E
:10FB6000AB4209D12846F7F70EFFBDE838400448FC
:10FB700000214C2207F0DBBE38BD00BF70250020FD
:10FB8000BC250020034B1A68D379591C1344D1714A
:10FB9000187A7047C411002010B5FFF7F3FF84B244
:10FBA000FFF7F0FF04EB002080B210BD10B5FFF7A7
:10FBB000F3FF0446FFF7F0FF04EB004010BD10B563
:10FBC0000446054B21461868FEF753FA034B1B68A1
:10FBD00098796040987110BDC8110020C4110020B0
:10FBE00038B504460D462420FFF7E9FF4D20FFF706
:10FBF000E6FF002C084C14BF21203E20FFF7DFFF5A
:10FC00002368002228469A71FFF7D9FF236893F8EA
:10FC10004900BDE83840D2E7C41100200146002069
:10FC2000DEE710B50446C0B2FFF7C9FF200ABDE801
:10FC30001040C4E710B5044680B2FFF7F2FF200C75
:10FC4000BDE81040EDE737B58288836804461006AA
:10FC50000D4641BF29494FF4CC7091F8A41700FB21
:10FC60000133D10542BF26490C20097802F03F023A
:10FC700048BF00FB0133042A12D006D8012A0DD058
:10FC8000022A2FD193F900102DE0102A0AD0202A41
:10FC90000AD0082A26D1B3F9001024E0197822E00E
:10FCA000198820E019681EE069461868F8F7B0F86E
:10FCB00001461448F8F726FAF5B1E06804F056F862
:10FCC0006946F8F7A5F801460F48F8F71BFA2069CE
:10FCD00004F04CF86946F8F79BF801460A48F8F733
:10FCE00011FA09E000210948F8F70CFA25B1084893
:10FCF000E1682269F8F706FA03B030BDB0260020AB
:10FD0000E01F0020F3C90108ECC901084CDF01081D
:10FD1000E9D20108024B0146D869FEF7AAB900BF33
:10FD2000E01F002010B5441E14F8011F21B1034B41
:10FD3000D869FEF79EF9F7E710BD00BFE01F00206D
:10FD40002DE9F04F037885B01BB96C48FFF7EAFF47
:10FD5000D1E007F085FE05460628694C99BF694841
:10FD6000294669480621F8F7CDF994F820200023A8
:10FD7000D9B2914207D26549002051F823100133CE
:10FD800009680880F4E7013DEDB272B6604F6DB2CC
:10FD900007EBC50149684FF001085E4B5E4E57F80E
:10FDA0003590042208FA01FA5A611FFA8AF14FF4D9
:10FDB00080624FF4007372614FF0480B73613046FC
:10FDC000C9F8141003A9ADF80C2001938DF80EB0FA
:10FDD0008DF80F80FFF7A0FA019B3046ADF80C308C
:10FDE00003A910238DF80E30ADB28DF80F80FFF708
:10FDF00093FA484603A9ADF80CA08DF80EB08DF823
:10FE00000F80FFF789FAE9007B185A6857F83530F8
:10FE1000D00803EB800E53F8203002F00702A365F0
:10FE20009200E36523660F239340DB43E06DC4F843
:10FE300054E01840E065A06D0340A365E06D082321
:10FE400093400343E365A06D08FA02F30343384689
:10FE5000A365B3685F05FCD4676DA36D08223B60A2
:10FE60004FF40073C9F814A073612A4B1A6140F66D
:10FE7000B833B268520516D4013BFAD14FF400737F
:10FE8000ADF80C3018238DF80E302348012303A958
:10FE90008DF80F30FFF740FA236E04223B601D4BB4
:10FEA0001A6162B627E0C9F810A0E36D50F835E09A
:10FEB0003B604318D3F804C0DEF80C20012303FA9A
:10FEC0000CF31343CEF80C30B268134B5205C4D573
:10FED000D9F808204FF4007C1AEA020F0D4A4FF0BF
:10FEE000080E15BFC3F810C0C3F814C0C2F810E064
:10FEF000C2F814E0E8E705B0BDE8F08FF0D20108E1
:10FF0000E01F002037D3010863D30108042000203C
:10FF100028D20108000C014000080140F7B52A4929
:10FF20002A4B08782A4D1C682A4B05EB80001A885A
:10FF3000D0F8C010284B29481B7800914FF47A71F3
:10FF4000B4FBF1F1F8F7DEF8254B26481968264B8B
:10FF50000026B1FBF3F1F8F7D5F8244B1F68F3B294
:10FF600005EB8302D2F8D010E9B101249C403C4259
:10FF700017D0220715D01E4A0B20D25C00FB0323AA
:10FF8000134A1C4802EB8303D3F8F020F8F7BAF8C1
:10FF9000022C06D1184B93F86C1011B11748F8F7E2
:10FFA000B1F80136DBE71648FFF7BCFE154B1648E3
:10FFB0001A88164B92B219884FF4FA6303B0BDE861
:10FFC000F040F8F79FB800BF7011002074260020A1
:10FFD00018B2010810110020F80000208ED301088B
:10FFE00004010020D1D3010840420F00201100205D
:10FFF00000010020E1D30108E01F0020E9D301083F
:020000040801F1
:1000000031D401081E100020EDD301081C1000207F
:100010002DE9F0410024804625460F4E4146A75960
:10002000384607F005FD58B139460C48F8F76AF82C
:1000300030190021FFF707FE0948FFF773FE01356D
:1000400040F6944314349C42E7D11DB9BDE8F04119
:10005000044867E6BDE8F081B8B301087BCA01082F
:1000600031D4010802C901082DE9F74F824607F093
:10007000A2FC054628B1012819D19AF800302A2B94
:1000800015D15948FFF74EFE0024584E5848A15943
:10009000F8F738F830192946FFF7D5FD5548FFF72E
:1000A00041FE40F6944314349C42EED198E0504611
:1000B0003D2107F072FC002800F08D8003461D46AC
:1000C00013F8012D202AFAD0441C204607F0C8FC62
:1000D00081462046F7F706FE0746CAEB05054FF0B6
:1000E000000B142404FB0BF4DFF8208108F5D07317
:1000F000E6580193304607F05EFC8446314662467E
:100100005046CDF800C007F05FFCDDF800C0019B51
:10011000002856D1EAB2624553D11D194444D4F89F
:10012000AC0103F023FE0146384604F025F8002810
:1001300045D0D4F8B00103F019FE0146384604F06A
:1001400011F800283BD0B4F8A4319A0658BF4F46A6
:10015000142202FB0B881C0648BF2748D8F8A821A8
:1001600042BF90F8A4074FF4CC7404FB0022D805DA
:1001700042BF22480C24007803F03F0348BF04FB31
:100180000022042B39460BD004D8013B012B0CD89C
:1001900017700AE0102B05D0202B05D0082B04D1B6
:1001A000118002E0176000E0176031461448F7F74D
:1001B000A9FF2846002103B0BDE8F04F43E51148F0
:1001C00005E00BF1010BBBF1A10F8AD10E4803B082
:1001D000BDE8F04FA6E5504603B0BDE8F04F17E785
:1001E00003B0BDE8F08F00BF1FD40108B8B3010809
:1001F0007BCA010831D40108B0260020E01F00208E
:1002000034D401083FD4010802C9010818B201081A
:1002100008B50748FFF786FD064BD869F7F7A8FB36
:10022000FEF7A6F8F8F70AF9034A044BDA6008BDAE
:100230005FD40108E01F00200400FA0500ED00E093
:1002400008B50548FFF76EFD01F078FBF8F720F9D7
:10025000BDE80840DCE700BF6BD4010808B50448DE
:10026000FFF760FDF8F714F9BDE80840D0E700BFDC
:1002700081D4010810B54B88DC0641BF2F4B14799F
:100280001B6853F8244044BF2D4B43F820404B8853
:100290009B0641BF294B54791B6853F8244044BF47
:1002A000274B43F820404B881C070ED5254B0C7874
:1002B0001B78B3EB141FA1BF204BD4781B6853F8F5
:1002C0002440A4BF1E4B43F820404B889B070ED50B
:1002D0001D4B0C781B78B3EB141FDFBF174B547802
:1002E0001B6853F82440DCBF154B43F820404B8873
:1002F000DC070FD5154C0B78247803F00F03A342CD
:10030000DFBF0E4B14781B6853F82440DCBF0C4B46
:1003100043F820404B885B070FD50B780C4903F05E
:100320000F0309788B42A1BF044B92781B6853F8E6
:100330002220A4BF024B43F8202010BDC81C00207F
:10034000FA0D00205B1600205916002058160020D8
:100350005A160020254A0023F0B515681C461A4697
:100360002348244903700B702E1976884EB92F5DEF
:100370003FB9037000230A704B7007781C461A4679
:100380000CE0360548BF013204F1040403F1010317
:1003900048BFD2B2802CDBB2E6D1EAE7E0B2B84285
:1003A0000CD215F82400013406099E4200F00F001B
:1003B000A8BF731C9042A8BF421CEFE78A704B7025
:1003C000C2F3470102F001020A444C1E0A490B48DD
:1003D0000A70C3F3470203F0010313440470084991
:1003E000501E084A08701370F0BD00BFE8110020CD
:1003F00050160020682000205A16002058160020B1
:100400005B16002059160020924B2DE9F04FDA6858
:10041000914D1A612A6891B0DA60904A029513688A
:1004200043F0200313608E4B1A78012A0CBF002280
:1004300001221A708B4B1A78910740F14D838A493B
:100440000978042940F248838849097801F00401B9
:1004500001F0FF0011B922F001021A701B78DB07CE
:1004600002D408B1FBF7E8FA8149CA78531C052287
:1004700093FBF2F202EB82029A1A7E4BCA701F784B
:1004800092000023DFF81082DFF8109258F8231052
:10049000794C91FBF9FE04F1080040F823E077481D
:1004A00044F8231000FB0E1142F2107091FBF0F0A3
:1004B00004F1100680B226F813004FF0140C04F17A
:1004C00014060CFB036C04F13C0A5AF823605CF838
:1004D00002504CF80210761B314405264AF82310CE
:1004E00091FBF6F109FB0E114434012F44F823105F
:1004F0004FEA830B444605D10238B0F5797F98BFA7
:100500004BF808100BB90123BCE7594E029BB246C9
:100510001868336DC01A03F025FC594903F02EFD0D
:10052000029B4FF07E511B680746336503F010FEB7
:1005300008B94FF07E574B4BCAF854701B78514E98
:1005400013F00103504D12D00DAA00924F4B0EAA8A
:1005500001920CCB94E80300FBF784F90D9A642117
:10056000B2FBF1F20E9B328093FBF1F300E033809B
:100570002B809AF858303E4D002B35D0696D4FF0E6
:100580007E5003F0FBFC0746EB6D2068C01A03F0B9
:10059000EDFB394603F03EFC03F002FE2B6E86B203
:1005A000606836B2C01A03F0E1FB394B196803F0FA
:1005B00031FC394603F02EFC03F0F2FDB5F966205C
:1005C00000B28118B5F964200220B31891FBF0F154
:1005D00093FBF0F389B29BB2A5F86A10A5F86830D6
:1005E000A5F86610A5F8643001238AF85830294B25
:1005F00061681B88206803F030031D4E264DCAF841
:100600006010CAF85C00002B00F0668206F17403EB
:10061000009306F178030193F26E336FFBF722F932
:100620006B68306FC01A03F0A1FB194B196803F017
:10063000F1FB03F0B5FDF36E2A68C6F880009B1A43
:10064000F3670C4B1B78012B2AD0022B00F0E680BD
:1006500042E200BF6807002074260020201100201D
:100660008A100020241100202A110020A33000202D
:1006700068200020340F00206C200020806967FF74
:1006800000007A449E110020A01100208C10002050
:100690006C000020E41100202C11002080969800AE
:1006A000D6F88430D6F8A0400293D6F8943004F1FE
:1006B00000400393D6F89830776D059303F070FDF2
:1006C0008146204603F06CFDD6F89C30BB4C049369
:1006D000BB4B06901B684FF0000B0793B94E4FEAD7
:1006E0004B0356F82B80A6F11402404632F81B50FB
:1006F000089303F03BFB029903F08CFB03F050FDE1
:10070000401B1FFA80FA283626F81BA00FFA8AFA37
:10071000504603F02BFB039903F07CFB03F040FDF4
:1007200086B20AEB080003F021FB059903F072FB87
:10073000394603F06FFB216803F064FA03F030FDE3
:10074000484504DB069B9842A8BF184600E048468F
:1007500003F00CFB206003F023FD079B304486B2BE
:10076000987803F0FFFA984903F054FB01464FF0E4
:100770007E5003F003FC394603F044FA0146384644
:1007800003F0FCFB09906068D4F808A0C0EB0800F7
:1007900003F0ECFA394603F0F1FB514603F030FA6E
:1007A000099A0146104603F035FB0146504603F016
:1007B00029FA3135ADB2622D01462061C4F80480BA
:1007C000A0600ED9049803F025FB03F0E9FC7F4AF2
:1007D000B0F5FA6FA8BF4FF4FA609042B8BF104668
:1007E00000E0002040F6B832064436B29642A8BF78
:1007F0001646774A089B9642B8BF1646754A54F883
:10080000140B9E52142202FB0BF273495050BBF1A1
:10081000000F40F061814FF0010B5FE7684BB6F8C5
:10082000A8401F68736F3D8902935B089D4228BFF3
:100830001D4623B29D4202DC1FFA85F90AE0674992
:10084000706D03F0E7FA03F0ABFC20441FFA80F967
:10085000A6F8A890DAF87860DAF8AC40341B2046A5
:10086000FBF742F841F293130028D8BF4042984268
:10087000CCBF0020012078B3204603F077FA584916
:1008800003F0C8FAF7F76DFC0446029803F06AFA21
:100890000146204603F0BEFA03F082FC40F6B8336E
:1008A00080B2AAF8B00000B29842A8BF1846484BE0
:1008B0009842ACBF3018F01848F6A043984203DDC8
:1008C000A0F50C40A03804E00028BCBF00F50C40A7
:1008D000A030CAF8B40001E0CAF8B460DAF8B43065
:1008E0000026C3F50C502830039303F03FFA3C492F
:1008F00003F090FA0446F7F7A7FC0F902046F7F7AD
:1009000030FCDAF8B830DAF8C4400593DAF8BC30D5
:100910000E9004F10040089303F042FC049020463E
:1009200003F03EFCDAF8C030DAF854802A4C099023
:100930000793730048460A9303F018FA0EAB53F876
:10094000261003F067FADFF8A0A005463AF9160072
:1009500003F00CFA0146284603F052F903F020FC9C
:1009600005B2204BB5F57A7FA8BF4FF47A759D424A
:10097000B8BF1D460AF13C0AA8B22AF8160000B218
:1009800003F0F4F90599824603F044FA03F008FCF9
:10099000089983B25046069303F03CFA414603F0AF
:1009A00039FA216803F02EF903F0FAFB049B984210
:1009B0001CDB099B9842A8BF184618E0700F002066
:1009C000380F0020E4200020DB0FC94030F8FFFF83
:1009D00048F4FFFF420F0020980F00200000C8429B
:1009E000D302373918FCFFFFD0200020049803F011
:1009F000BDF920608346B87803F0B4F9384903F0B4
:100A000009FA01464FF07E5003F0B8FA414603F070
:100A1000F9F80146404603F0B1FA0B906068D4F84B
:100A200008A0281A03F0A2F9414603F0A7FA51469C
:100A300003F0E6F8DDF82CC00146604603F0EAF961
:100A40000146504603F0DEF8656001462061A06073
:100A5000079803F0DFF903F0A3FB069B143403446B
:100A600058469A4603F09CFB40F6B832504400B218
:100A70009042A8BF10461B4A0A9B9042B8BF10463E
:100A8000194A1A4998521422724342F801B00EB919
:100A900001264EE73B792BB1039A642392FBF3F3D3
:100AA000134A13803B88029A124C9A420DD9D4F80B
:100AB000AC30A06FC01AFAF717FF42F2107380EA49
:100AC000E072A2EBE0729A4206DD0B4B01221A7033
:100AD000B4F8C820064B1A8011B0BDE8F08F00BFF3
:100AE000DB0FC94048F4FFFF420F0020700F0020C9
:100AF000300F002068200020340F002008B508487F
:100B000006F059FFC0B209280246054B04DC01304B
:100B10002021C0B29954F6E700221A5408BD00BF44
:100B20003421002008B5074806F045FFC0B214285C
:100B3000044B04D8421C20211954D0B2F7E70022FC
:100B40001A5408BD34210020642928BF6421F8B557
:100B500001FB00F5642495FBF4F40646E4B200279B
:100B6000FBB2A34204D29F20FEF733FD0137F7E723
:100B7000B4420BD2142195FBF1F5C4EB8410663D11
:100B8000C4EB80002844C0B2FEF723FD0134E4B278
:100B9000B44201D29A20F7E7F8BD2DE9F743FDF7FB
:100BA00095F9924CA369C31A002BC0F2588300F543
:100BB000433303F5A073A3618D4B1E78237FC6F3E7
:100BC0008006F31A18BF012326774EB1002B00F0E0
:100BD0004683884B5A789A7001225A701A702BE01B
:100BE000844A2BB1D37843F00203D37093785370C7
:100BF000D57805F0020101F0FF0339B97D49896814
:100C0000411A002903DB05F0010300E0012303F092
:100C10000107784917707BB1EA070DD50A790523DA
:100C20000132D2B2B2FBF3F303EB8303D31A724A5D
:100C3000DBB20B71D35C4B706E4DDFF804822B7806
:100C40007BB3EB7823F00203EB706C4B0344AE20D4
:100C5000AB60FEF7E2FC08B1FEF7E4FC88F80000A8
:100C6000002800F0FC82B020FEF7D7FC4020FEF701
:100C7000D4FC0020FEF7D1FC1020FEF7CEFC4FF490
:100C80008067013F0020BFB2FEF79EFC002FF8D125
:100C90003846FEF736FD6A78594B53F82200FEF7C6
:100CA000B3FC98F80030002B00F0D9826B78062B4B
:100CB00000F2AA82DFE813F00700A802180078000B
:100CC00061017E01E4014F494F4A504B4748F7F715
:100CD00004FA0120FEF715FD4448FEF795FC0220BA
:100CE000FEF70FFD4A48A3E14A4F3B689B0735D505
:100CF000DFF850810A23B8F80010DFF84C91B1FBFF
:100D0000F3F203FB121399F8001092B29BB2009118
:100D100036484149F7F7E1F9FFF704FF0120FEF7F4
:100D2000F0FC3248FEF770FC3C4B99F80020186844
:100D3000B8F80030057902FB153164234B43C178C4
:100D400002204D1B5543B3FBF5F5EDB2FEF7D9FC80
:100D500029461520FFF7F8FE032500E001253B6832
:100D60001F0540F151822E4B2E491F68642397FBCB
:100D7000F3F2096803FB127300911C482A49F7F744
:100D8000ACF9FFF7CFFE2846FEF7BBFC1748FEF78D
:100D90003BFCFCF7C9FE0746681CFEF7B2FC1520B9
:100DA0003946FFF7D1FE2FE20120204FFEF7A9FCC4
:100DB0001F48FEF729FC3B68980747D51D4A0B489A
:100DC000B2F90210B2F900300091B2F904201A49C8
:100DD00001921A4AF7F781F9FFF7A4FE0220FEF705
:100DE00090FC0248FEF710FC032530E0342100207F
:100DF000A3300020881C002075DE0108404B4C0009
:100E0000A8C001087ADE01087DD201085DC301088F
:100E100078D201085026002083DE01080C11002042
:100E2000181100201C1100209BDE01082011002059
:100E3000B0DE0108EE100020C6DE010864DE010805
:100E4000E902002010110020F800002002253B6874
:100E5000D9071AD5784A7948B2F90210B2F90030A8
:100E60000091B2F9042076490192764AF7F735F9F4
:100E700005F10108FFF756FE2846FEF742FC5FFA2F
:100E800088F86E48FEF7C0FB45463B681A0718D540
:100E90006D4A6A48B2F90210B2F900300091B2F915
:100EA000042067490192694AF7F717F96F1CFFF7A9
:100EB00039FE2846FEF725FCFFB26048FEF7A4FB8A
:100EC0003D46634A5E49B2F90030B2F902205B4800
:100ED0000092604A604FB2F9002005F101080192CA
:100EE0005E4AF7F7FAF8FFF71DFE2846FEF709FC01
:100EF0005248FEF789FB51493868F6F789FF4F4899
:100F000006F059FD5FFA88F8C1B2092908D84B1CD0
:100F1000DBB2202262540021E21851701946F4E736
:100F200021447868F6F774FFFFF7FCFD4046FEF7B2
:100F3000E8FB4248FEF768FBB8684049F6F768FFEF
:100F40003E4806F038FD0235EDB2C7B2092F08D889
:100F50007B1CDBB22022E2550021E21851701F46B3
:100F6000F4E73F4BB3F9000002F000FFE119F6F798
:100F70004FFFFFF7D7FD284657E00025394F3B7854
:100F8000AB4240F241810E2D00F03E8168080130F5
:100F9000FEF7B7FB284602F011FA3B78AB4206D9C0
:100FA0002020FEF716FB681CC0B202F007FA0235DB
:100FB000EDB2E3E72C4D2D4995F8A4271F48F7F72C
:100FC0008CF80120FEF79DFB1C48FEF71DFB284B0B
:100FD00028491F7819483A46F7F77FF80220FEF7AC
:100FE00090FB1648FEF710FB0C2303FB0755224924
:100FF00095F8A72795F8A6371048F7F76EF8FFF78A
:1010000091FD0320FEF77DFB0C48FEF7FDFA95F8F5
:10101000AC1795F8AA2795F8AB37084800911749FF
:10102000F7F75BF8FFF77EFD0420FEF76AFB034845
:10103000FEF7EAFAE8E000BF40100020342100206B
:10104000C6DE0108D5DE01084610002071DE010869
:1010500046260020FC100020741F0020D9DE010865
:10106000801F002008300020B0260020DDDE0108AF
:10107000E01F0020E9DE0108FADE01080BDF0108AD
:10108000784B1B681B0640F1BB80236A616A764A75
:101090008B421CBF536292F828304FF001011CBFF5
:1010A000013303F003034FF0000018BF82F828302B
:1010B000FEF733FB94F828306C4A0025D05CFEF72D
:1010C00088FA02200121FEF728FB694B3620EB5CF1
:1010D0000135C3EBC30393FBF0F0C0B2062828BF71
:1010E00006206038C0B2FEF774FA102DEDD1614BC6
:1010F00061491B785C4813F0020F604B1A7814BFEB
:1011000059234E23F6F7E9FFFFF70CFD0220FEF707
:10111000F8FA5548FEF778FA59495A4B4D680A686B
:10112000514892FBF3F2584995FBF3F3F6F7D5FFDC
:10113000FFF7F8FC0320FEF7E4FA4B48FEF764FAE9
:10114000524B53491A884848F6F7C7FFFFF7D6FCB9
:101150000420FEF7D6FA4448FEF756FA4D4B4E49A6
:101160001A884148F6F7B9FFFFF7C8FC04210A20A6
:10117000FEF7D3FA3C48FEF747FA4849E26A3A4894
:10118000F6F7ABFF464DFFF7B9FC0520FEF7B9FABD
:101190003548FEF739FA6A68AB6842493248F6F7D3
:1011A0009CFFFFF7ABFC05210A20FEF7B6FA2E489C
:1011B000FEF72AFA2B69EA683B49D21A2A48F6F761
:1011C0008CFFFFF79BFC0620FEF79BFA2648FEF7F4
:1011D0001BFAAA6835492448F6F77FFFFFF78EFC13
:1011E00006210A20FEF799FA1F48FEF70DFA30494A
:1011F00015221D4806F00AFCFFF780FC072014E7C3
:10120000EB7843F00203EB704EBB2A4B00219B7935
:101210001220032B97BF284A3F259B181D7FFEF7FE
:101220007CFA2846FEF7D5F913200021FEF775FA5F
:10123000224B1B78002B14BF52202120FEF7C9F946
:1012400014200021FEF769FA94F83050074B585DDE
:10125000013505F00305FEF7BCF984F8305003B002
:10126000BDE8F08350260020342100201DDF010856
:10127000D11000202411002022DF01082A110020B3
:101280002C1100208096980033DF010826110020E1
:1012900040DF01088810002048DF01084FDF010807
:1012A0006807002056DF01085FDF010866DF0108DC
:1012B00070030020FC240020A8C001080A30002090
:1012C0000028114AB8BF404290FBF2F330B50F4CF2
:1012D0003C2504FB030068430D4D90FBF2F22D68A2
:1012E0002D7B25B903EB830303EB830301E0C3EB01
:1012F000031302EB830304FB02020B804FF47A73A7
:1013000092FBF3F24A8030BD80969800806967FFB7
:1013100014110020022803D0431E58425841704740
:10132000064B1B681B7823B1054B1868C0F3C040FF
:101330007047044B1878C0F380007047B006002057
:1013400020100020A3300020A0F17D03012B70B5F8
:1013500004460D460A4E05D830687D21FCF789FE0B
:1013600084F0200430682146FCF783FE35B12B88D9
:101370001C4404EB142404F0FF042C8070BD00BF57
:10138000D411002010B50A4C5E280146206805D112
:101390005D21FCF76EFE20683E2105E05D2903D14A
:1013A000FCF767FE20683D21BDE81040FCF761BEF8
:1013B0006821002037B51A4B1A4C1B491B4A20B133
:1013C0001B480088B0F5805F21D209881278154D3E
:1013D0009B79ADF804108DF8062001A8291D042280
:1013E0008DF8073006F088FAC0B101986860532084
:1013F00000F09CFDA08800F0CBFDA07900F0C8FDB6
:10140000E07900F0C5FD0A4B00221A8006E0098849
:1014100012789B79A180A271E371E8E703B030BD37
:10142000FC24002068210020E41100202411002069
:10143000A02400202DE9F84305460E460D4B00245C
:1014400093E88003B44213DA7B1933F9140008EBF4
:10145000050333F9142009EB050333F91430013483
:101460001344022293FBF2F3C01A00F0A0FDE9E757
:10147000BDE8F883FC220020F8B5374CA368C01AF9
:10148000002867DB237B0021012BA1600FD002D352
:10149000022B1DD059E0314DAB689847EB68984757
:1014A000012323736A88A3681344A3604DE02B4D86
:1014B0002B6998476B689847A3682A8804F1100045
:1014C0001344A36026496B699847022323733CE0C9
:1014D000244E62693668551C36782173B54201BFC7
:1014E000214D01262E700D46A16923694E1C032E45
:1014F00002BF194E4FF0010E86F81CE004EB81018B
:101500001A480B62217F08BF00260768DFF848E011
:10151000A66181B1DEF82060DEF82410DEF8283004
:101520008E42DEBF8E4631467646B342A8BF334672
:101530008B42B8BF0B4604EB8202D36204EB8502F8
:10154000D26A6561BA1A13440360FCF7BFFCA36852
:101550001844A060F8BD00BF682100202C030020C3
:101560000011002038070020290700203407002040
:1015700030B585B004AC002524F8025D0091ADF8CB
:10158000060021461020FFF7DFFE9DF806002146E9
:10159000FFF7DAFE9DF807002146FFF7D5FE9DF81C
:1015A00000002146FFF7D0FE9DF801002146FFF71D
:1015B000CBFE9DF802002146FFF7C6FE9DF8030012
:1015C0002146FFF7C1FE9DF80E002946C043C0B278
:1015D000FFF7BAFE05B030BD10B5054C2068FCF72A
:1015E00045FD18B12068FCF73EFDF6E710BD00BFD1
:1015F000A811002010B50446C0B2FFF7C3FEC4F323
:101600000720BDE81040BDE6024B5E211868FCF7DC
:1016100030BD00BF6821002038B50546054C5E216D
:101620002068FCF726FD20682946BDE83840FCF715
:1016300020BD00BF6821002013B5044601A9006841
:10164000FFF73EFE1320FFF7E7FFBDF90400FFF7A9
:10165000D1FF1B20FFF7E0FFBDF90600FFF7CAFF2F
:101660002320FFF7D9FF2368002BB4BF53204E205F
:10167000FFF7C0FF01A96068FFF722FE1220FFF705
:10168000CBFFBDF90400FFF7B5FF1A20FFF7C4FF39
:10169000BDF90600FFF7AEFF2220FFF7BDFF63682C
:1016A000002BB4BF57204520FFF7A4FF02B010BDA8
:1016B000674B73B51878FFF72DFE664D04462B78FF
:1016C000834220D0C8B1644B1B68E3B193F900009A
:1016D00002230093614B04211B6800225B780033D6
:1016E00018BF012301934FF41653F6F75FF95C4BD3
:1016F000186040B101232B7005E0594E3068F6F7B1
:1017000042F934602C70574B574D1878FFF702FEA2
:101710002B780446834218D088B1544B1B68A3B180
:101720000022012493F9000008214FF4964300940D
:101730000192F6F73BF94E4B186028B905E04C4E84
:101740003068F6F720F934602C704A4B4A4D18780F
:10175000FFF7E0FD2B78044683422E4643D0002855
:1017600038D0464B1A68002A3DD0D37992F9000050
:10177000002B4FF00202424C08BF022300920022CD
:1017800054F8233001921021F6F710F93D4B05462D
:10179000186040B33C4C94F84A30022B0BD094F8BC
:1017A0009620022A01D14C3405E023B1002A04F12D
:1017B0004C0418BF0024354B1C6044B12046002166
:1017C0004C2206F0B4F80223256084F84A30012345
:1017D000337008E02B4E3068FEF7B4F93068F6F746
:1017E000D2F834602C702A4B2A4D1878FFF792FDFE
:1017F0002B780446834229D000B3274B1B682BB3B8
:10180000264A93F900001268032352782021002A07
:101810000CBF08220922009301924FF46143002279
:10182000F6F7C4F81E4B186080B11E4A01231370EE
:101830002B701D4B1A681D4B1A6007E0184E30685C
:10184000F6F7A1F8174B34601C702C7002B070BD15
:10185000B8060020E4100020B40600201411002077
:1018600068210020C006002034110020BC060020A2
:10187000A8110020CC060020BA110020C8060020C4
:10188000A0C10108BC11002070250020C01100205B
:10189000D8060020D0110020D4060020D006002059
:1018A000D4110020D811002074260020DC11002063
:1018B00010B50E4C2068FCF791FA20680022047ADB
:1018C00002FB02F3193B634303F6C413534319218C
:1018D00093FBF1F3064921F812300132072AEFD1C8
:1018E000BDE810400349FCF731BA00BF8410002066
:1018F000800E0020F42700200E4B1A78692A15D19B
:101900005A88B2F5FA6F11D11A79BE2A0ED193F81E
:10191000CD270020EF2A0BD113F8012B5040064AA7
:101920009342F9D1B0FA80F0400970470020704727
:10193000704700BF00F80108D0FF01082DE9F74FFC
:10194000EA4C00214FF4FA62204605F0F0FFE84B24
:1019500004F537721A60E74B00221A70E64B04F266
:10196000A671196069232370032363714FF4807398
:10197000A3604FF41673A4F86631FA23A4F8683113
:10198000BC23A4F864314FF4FA73A4F86E31012338
:1019900084F8623184F87E3184F88631052384F836
:1019A0001B3240F2DC53A4F8983140F24C43A4F8C7
:1019B0009A3140F26C73A4F89C3140F27533A4F86C
:1019C0009E3140F64303A4F8A0312346202184F839
:1019D0006A116E2184F87C110A2184F87D112B2173
:1019E00084F87F11212184F88011232184F881114A
:1019F0004FF4C871A4F882119918023200254FF0F3
:101A00001E0A1C2AB94C81F8A25181F8A3A1F3D176
:101A100040F27E41A4F8441140F23A71A4F8461114
:101A200040F27E51A4F84C1140F2EA5140F2DC50F1
:101A3000A4F84E1140F2B4514FF4FA63A4F8C03147
:101A4000A4F8C431A4F8C831A4F8CC31052384F833
:101A5000D631C82301264FF47A784FF0320BA4F820
:101A6000DA31DFF88C924FF4C8731922A4F8DE3112
:101A7000A4F84A01A4F85011A4F8BE81A4F8C281C8
:101A8000A4F8C681A4F8CA8184F8D86184F8D96121
:101A900084F8DC61A4F84881A4F852B184F895A1D7
:101AA00084F8D72100920190A4F8543184F8D561CC
:101AB00084F8E261A4F856B184F8E56101F09CF97C
:101AC000D9F80030009A4FF00F0E2674E673A57314
:101AD000A58183F805E04FF0220E172183F806E078
:101AE000DA714FF00E0E21225975997583F810E0C6
:101AF0005A7455214FF0350E53224FF0640C2827AD
:101B0000D97083F81AE02D21DA764FF05A0E0A22A6
:101B100083F81CC04FF0780C83F80BA083F80CA05E
:101B2000597383F808E09A7483F80AC01D705F70D7
:101B30009F70DD7583F804B09D731D76DD735D764F
:101B40005F7219754FF4FA71A3F84E106B49DFF804
:101B5000CCC19963D9636A49C3F82CC0C3F830C0BB
:101B60009962DFF8BCC14FF07E5159634FF07F5A44
:101B700064490198C3F820A0C3F824A0C3F848C062
:101B80004FF0000A4FF04B0C83F8502059649E77B9
:101B900083F8525083F85170C3F840A083F84CC0CA
:101BA00084F8A6E7A4F8B0074FF0410E042084F8AB
:101BB000A7E784F8A8B784F8A95784F8AD5784F844
:101BC000AE5784F8AA5784F8AB5784F8AC57009204
:101BD00083F85C00A3F85850A3F85A50A3F8565065
:101BE0001966152183F8681047494848D96648495D
:101BF00083F864701967474983F86570596783F8FB
